:020000040000FA
:040000006FD00400B9
:101000006F00507B000000000000000090200020D6
:10101000AA220020A9BDF9F56C23002000000000E1
:10102000000000006C230020902000200000000041
:101030000000000090200020000000009020002010
:101040000000000090200020902000209020002030
:101050009020002090200020242F00205E240020DB
:101060000000000090200020902000200424002098
:1010700090200020D22300209020002090200020EB
:101080009020002090200020902000209020002020
:101090009020002001A04111B7170040985F3AC688
:1010A000945F3247E39CE6FE3245410182800111A4
:1010B00013078008F337078093F787083EC20100C3
:1010C0000100B7170040930570052380B70413068D
:1010D00080FA2380C7040100010083C6B70493F699
:1010E000F60DA385D704238007049246F3A6068055
:1010F0000100010093760502D5CEF336078093F602
:10110000860836C4010001002380B7042380C70489
:1011100001000100B70614007D89558D88C70100C4
:1011200001000100010023800704A246F3A6068007
:101130000100010073370780137787083AC6010062
:1011400001002380B7042380C704010001000100CF
:1011500001003727004093061005A303D7802380A2
:101160000704B247F3A70780010001009307800836
:10117000F3B7078093F787083ECE01000100B71749
:101180000040130770052380E704130780FA2380CB
:10119000E7040100010003C7B70413670708A3852C
:1011A000E70423800704F247F3A70780010001004A
:1011B0000561828093760504BDC6F336078093F6F9
:1011C000860836C8010001002380B7042380C704C5
:1011D00001000100B7061400938606047D89558D31
:1011E00088C7010001000100010023800704C246F6
:1011F000F3A6068001000100733707801377870884
:101200003ACA010001002380B7042380C70401000B
:1012100001003727004093062005A303D7802380D1
:101220000704D24781B773370780137787083ACC12
:10123000010001002380B7042380C70401000100DE
:1012400098471367070C98C723800704E24719BF24
:101250000111814601468145114506CE97000000E7
:10126000E780005593078008F3B7078093F7870856
:101270003EC601000100B717004013077005238028
:10128000E704130780FA2380E7040100010003C785
:101290006704136717002383E70423800704B2471A
:1012A000F3A7078001000100F2400561828041112F
:1012B000814601468145114597000000E780404F77
:1012C00013078008F337078093F787083EC40100AF
:1012D0000100B7170040130670052380C70493066A
:1012E00080FA2380D70401000100FD552396B70240
:1012F00023800704A245F3A5058001000100733790
:101300000780137787083AC6010001002380C704CD
:101310002380D7040100010003C767041367170087
:101320002383E70423800704B247F3A70780010063
:10133000010001A0BD473305F50201007D1575FDD3
:101340008280411122C426C206C6AA8401446317C2
:101350009400B24022449244410182800504130566
:10136000803E420497000000E78000FD4180C5B741
:101370009305000273A04580824573901534924016
:101380002242B2424243D2436244F2440255925551
:101390002256B2564257D2576258F25806499649D9
:1013A000264AB64A464BD64B664CF64C065D965DD1
:1013B000265EB65E465FD65F09617300203041113C
:1013C000B7170040985F3AC6945F3247E39CE6FE49
:1013D000324541018280B71700401307000323887C
:1013E000E702854717170000232EF74273002030CD
:1013F000411122C406C637040020976000E0E78050
:10140000E0E21C408297D5BF373700408347470052
:101410009146BD8B6389D70099466394D700834773
:101420005740730020309736000083C6662C9387A0
:10143000160017360000230DF62A0347870097375A
:1014400000009387E71AB6972380E700B7E7040008
:10145000BC4F0946894517150000034565F482977E
:10146000C9B7B787004003C76700098B6309071036
:1014700003C777009306000313770703630DD708AC
:10148000173800000348586217360000130606613B
:101490000547B30606012380E60083C577001737AA
:1014A000000013072760429793F5F50F2300B7005C
:1014B00003C58700973500009385855EC295137537
:1014C000F50F2380A5000347070089451377F7032D
:1014D000630CB70C63E7E50A6306071A8545630CDE
:1014E000B7129737000083C7375C3307F60003470E
:1014F00007001377F70F19CB850793F7F70F0D4701
:101500006363F71A17370000A300F75AB787004044
:1015100009472383E700B787004083C77700E207C6
:10152000E18763DE07049737000083C7F757173753
:1015300000001307A7563E9785462300D7001737AC
:101540000000130727563E97930600032300D70099
:10155000173700001307C7543E97A146850723009D
:10156000D70093F7F70F0D476364F71417370000A0
:10157000A30CF752B787004009472383E7007300A5
:101580002030930610026300D70E930620026305F5
:10159000D70693060002E316D7F403C72702137792
:1015A000C70F13672700D5A803C767001377070481
:1015B00065CB03C7A702173800001308A82F1735FB
:1015C00000001305E526134707082385E70203C734
:1015D000A7021377370F136787002385E702814738
:1015E00013070004B305F5008C41B306F80091071A
:1015F0008CC2E399E7FEF5B503C7A70213470704BA
:101600002385E70203C7A7021377C70F13672700D5
:101610002385E702F9B503C767001377070449C3B9
:1016200003C76702173800001308881C173500002D
:101630001305C513134707082383E70203C767028F
:101640001377370F136787002383E7028147130758
:101650000004B305F5008C41B306F80091078CC275
:10166000E399E7FEBDBD03C7670213470704238361
:10167000E70203C767021377C70F136727002383A7
:10168000E70285B503C767001377070411CB03C7CB
:1016900027021377370F136787002381E70291B57D
:1016A000238006003DBD97370000A38F073EB9BDDC
:1016B00097370000A38A073E75BD230304801547B2
:1016C0002303E48001002302A480828083076480D6
:1016D000E3CE07FE23030480828083076480E3CE89
:1016E00007FE03454480828083076480E3CE07FEC3
:1016F0002302A4808280411126C44AC24EC006C67D
:101700001377F50BAD47AA892E899544630CF70032
:10171000194597000000E78080FA97000000E780F5
:1017200020FB8D444E8597000000E78040F9FD596D
:10173000FD1463983401B240A24412498249410128
:101740008280135509011375F50F97000000E7809B
:10175000E0F92209F1BF011126CC06CEB70408003A
:1017600097000000E780C0F6154597000000E7806D
:1017700000F597000000E78080F697000000E78002
:1017800000F62AC697000000E78080F43245937780
:10179000150089EB136515001375F50FF240E2444F
:1017A00005618280FD14E9F00145CDBF397126DC69
:1017B0004ADA4ED852D656D45AD25ED006DE62CE1F
:1017C00066CCB7E700E07D5783AA070022C603AACC
:1017D000470023A0E71823A2E718B7170040130714
:1017E00070052380E704130780FA2380E70483C78A
:1017F0004704930B75FFB684E20793FBFB0F854606
:10180000AA892E8B328937240040E187015763FA79
:1018100076016308D5008946130700026313D500DB
:101820000157D98F93F7F70FB71C00402382FC04B0
:1018300011472303E4801305F00F97000000E780B1
:1018400000E8094C97000000E78080E863657C159C
:10185000B7050700DA9537870700795563FEE50479
:10186000B3879500636AF704370B0800A94733EB89
:1018700065016395F90881E8814497000000E780DD
:1018800020E5268515A8DA85094597000000E78040
:10189000C0E605090345F9FFFD14050B970000009C
:1018A000E780C0E481C49377FB0FE5F79700000061
:1018B000E780A0EA69F17D55B7170040130770056E
:1018C0002380E704130780FA2380E70403C7470453
:1018D000418B2382E704F250B7E700E023A05711C1
:1018E00023A24711E25432445259C259325AA25AE1
:1018F000125B825B724CE24C21618280A547639B44
:10190000F90685691309F00FB3069900B3742B012A
:10191000B6941349F9FFB3749900856B3379690163
:10192000416B9387F9FFB3F7270199E363FC340117
:1019300093D94900C147E3E637FF3DBF0569C16957
:101940007D19D9B71305800D63886901130500025D
:101950006384790113051008CA8597000000E780A9
:10196000C0D997000000E78040DF31D54E99B3849D
:1019700034416DBFDA852D4597000000E780E0D740
:10198000CA94E30B99EE050997000000E78020D583
:10199000A30FA9FEFDB79387F9FF93F7F70F636DC8
:1019A000FC0C83C71C04130730086315F7063707C0
:1019B00008006361EB06B3079B00B706100063FBEA
:1019C000D704334BEB0089476399F9068980D549E1
:1019D000E38404EADA85094597000000E780E0D156
:1019E00011090327C9FF91472320E480030764807E
:1019F000E34E07FE23033481FD17EDFBFD14110BAD
:101A000081C49377FB0FE9FF97000000E780E0D4E3
:101A100061F155B5B717004003C75704B707080071
:101A20001377070219E3B78707007955E376FBE8D8
:101A300033079B00E3F9E7F841B58547E380F9F008
:101A4000DA852D4597000000E78020CB9389F4FFCD
:101A5000E38404E297000000E78060C893F7390050
:101A600091EB832604800327090093074900E3963E
:101A7000E6E03E89CE84D9BFB5476399F9001305E6
:101A8000900B97000000E78080C3FDB3B1471305BA
:101A9000B00AE388F9FE99476397F904B70508008F
:101AA000B365BB002D4597000000E78000C5814469
:101AB0008D4BA14997000000E78060C263967401D6
:101AC000832704802320F9008504E39534FF8327CE
:101AD000048013172B01635507002312F90069BB1B
:101AE0002322F90051BB9D47639FF90281451305ED
:101AF000B00497000000E78040C0BD4423200900E7
:101B000023220900FD5997000000E78040BD93F7AC
:101B10007400CA9703C70700FD14398D2380A700FE
:101B2000E39334FF91BBA1476397F9069700000048
:101B3000E780A0C28144630D0B008D479304C0036E
:101B40006308FB009304000563048B0193044004C5
:101B50001375C507E30295D2194597000000E78089
:101B600000B697000000E780A0B60545970000008A
:101B7000E780E0B4268597000000E78020B709459C
:101B800097000000E78080B697000000E780E0BC87
:101B9000E31405CE0DB39147639FF900130560066A
:101BA00097000000E780A0B197000000E78040B2F6
:101BB00013059009F9B5E38109CCF1547DB9BD66EF
:101BC0000147173600001306660B938606A6854567
:101BD0008347060093F7F70F91C382800507E3F967
:101BE000E6FE97370000238BB708DDB77D16620647
:101BF000618693178601E18763D4070001458280DF
:101C0000931726003307F500AE9718439C4363E70C
:101C1000E7007D16E37FF7FC7D55828005458280D5
:101C2000FD15E205E18513978501618793F7F50FAF
:101C300063480700FD15139725002A97584365D779
:101C4000138517006205618582803308B5021C4246
:101C500083A80600B335B502C29733B50701AE9825
:101C6000469585486367B5006394A50063E3070163
:101C700081480C43C6950CC388C21CC28280814730
:101C80001397870161876343B7008280139727000A
:101C90002A97232007008507E5B7814701479396D8
:101CA0008701E18663C5B6001335170082809396DD
:101CB0002700AA9694428507558FD5B793D75540EC
:101CC0008A07AA979C4305453315B5007D8D828010
:101CD00017F3FFDFE702A33D2A8497000000E780A7
:101CE00060F405C5931725003E940327C4FF814780
:101CF00011EB7D1516053E954205418517F3FFDF73
:101D00006700233D05838507E5B70145C5BF8147CA
:101D10001397870161876343C70082801397270069
:101D2000B386E50094422A97850714C3D5B77D167C
:101D300062066186014793178601E18763D5070034
:101D400013351700828093172600B306F500AE976F
:101D500094429C437D16B58F5D8FF1BF8A05AA958D
:101D600001476363B500828083A6C5FFF11593D751
:101D70001600D98F9CC11397F601E5B72A83014855
:101D8000014701456343D7008280B387050183A8DB
:101D90000700B30706019C43C697AA976384F8001F
:101DA00033B517010507B3080301620723A0F80044
:101DB00061871108C1BF2A8301478147014563C379
:101DC000D70082803388E50083280800330EE600C0
:101DD000032E0E003388A8403308C84163840801ED
:101DE00033B508018507B308E300E20723A0080123
:101DF000E1871107E9B717F3FFDFE702432B011172
:101E0000B286B2842E86AA850A8597000000E780F4
:101E1000C0FA2A84A6850A8597000000E78020E89A
:101E200033348000060413351500018D056117F366
:101E3000FFDF6700032A17F3FFDFE702C324411126
:101E4000AA89AE8A328BB68402C202C402C6014499
:101E5000131C8401135C8C4163499C02939B140006
:101E6000FD1B0549138CF4FFF15C33048901620406
:101E700061846340740792478E04CE9423AEF4FECF
:101E8000410117F3FFDF6700832313192400B30B0D
:101E90002B01014A93172A00D69783A50B0088438C
:101EA00078003400500097000000E78040DA050A0F
:101EB00093178A01E187F11BE35EFCFC92474E9980
:101EC00005042320F900A2473EC2B24702C63EC421
:101ED00041B7131A8901135A8A41131D240093171D
:101EE0008A01E18763CF970092470A044E941CC091
:101EF000A24705091379F90F3EC2B24702C63EC494
:101F0000ADB7B3079A0313152A0056950841780018
:101F100034005000050AEA97DA978C4397000000D6
:101F2000E780E0D26DBF0000197106C212C416C668
:101F30001AC81ECA22CC26CE2AD02ED232D436D6E9
:101F40003AD83EDA42DC46DECAC0CEC2D2C4D6C6D9
:101F5000DAC8DECAE2CCE6CEEAD0EED2F2D4F6D6C9
:101F6000FAD8FEDA971500009385458B8841E70083
:101F7000050092402242B2424243D2436244F244BC
:101F8000025592552256B2564257D2576258F258CD
:101F900006499649264AB64A464BD64B664CF64CFD
:101FA000065D965D265EB65E465FD65F096173008C
:101FB00020300000972100209381C1041751002098
:101FC0001301418417F5FFFF130505049705002051
:101FD00093854503171600201306C6FD63FAC50056
:101FE0008322050023A0550011059105E3EAC5FEF3
:101FF00017050200130545D297150020938585FB30
:10200000171600201306066563FAC5008322050033
:1020100023A0550011059105E3EAC5FE1715002020
:102020001305456397450020938545116377B500F7
:10203000232005001105E36DB5FEFD42739002BC3F
:102040008D4273904280B722000093828288739001
:102050000230970200209382E2FA93E232007390FA
:1020600052309752000093824297739012346FB0AF
:10207000347973002030397101436EC619A039716B
:1020800041536AC866CA62CC5ECE19A03971015349
:102090005AD056D252D44ED64AD826DA22DC06DEA0
:1020A00033016140828241114AC026C222C406C661
:1020B0008282B24D4101024D924C224CB24B410101
:1020C000024B924A224AB2494101024992442244B7
:1020D000B240410182803D432A876373C3029377F4
:1020E000F700BDEFADE5937606FF3D8ABA960CC3C7
:1020F0004CC30CC74CC74107E36BD7FE11E282808B
:10210000B306C3408A069702000096966780A60031
:102110002307B700A306B7002306B700A305B7003F
:102120002305B700A304B7002304B700A303B70037
:102130002303B700A302B7002302B700A301B7002F
:102140002301B700A300B7002300B700828093F5F6
:10215000F50F93968500D58D93960501D58D61B7C2
:10216000939627009702000096968682E78086FA6B
:102170009680C1171D8F3E96E374C3F8A5B73367E9
:10218000B500FD530D8B79E7B7877F7F9387F7F70E
:1021900010419441B372F6003363F600BE92B3E28D
:1021A00062006397720C6318D6065041D441B37233
:1021B000F6003363F600BE92B3E262006398720ADF
:1021C000631BD60410459445B372F6003363F600E2
:1021D000BE92B3E262006391720A631ED60250455A
:1021E000D445B372F6003363F600BE92B3E26200E8
:1021F000639A72086311D60210499449B372F600CB
:102200003363F600BE92B3E2620063937208510535
:10221000D105E30FD6F61317060193970601631C49
:10222000F7001357060193D706013305F74093755E
:10223000F50F91E982804183C1833305F74093759F
:10224000F50F91E182801377F70F93F7F70F3305BE
:10225000F74082800346050083C605000505850515
:102260006313D60065FA3305D640828011059105C7
:10227000E312D6FE014582802105A105E31CD6FCB0
:10228000014582803105B105E316D6FC0145828007
:102290004105C105E310D6FC01458280B717004017
:1022A00003C777051377E70FA38BE704130700F83D
:1022B000A38DE7043D47238CE70413075003A38C49
:1022C000E70403C7A7051377D70F238DE7048280A0
:1022D000B717004003C7E7020D8941111377C70FF5
:1022E000498F93068008F3B6068093F6860836C6B3
:1022F00001000100930670052380D704930680FA3D
:102300002380D704010001002387E702238007040C
:10231000B247F3A70780010001004101828041110B
:102320002A83014E930E407E130F0019930F40062F
:1023300063E56E129308001913034006B378150382
:10234000854E0D4FA14F337365020D89133515006E
:1023500063EFBE121308F6FF7946729842081358CD
:1023600008013307C70213D61700BE07329761462C
:10237000B3F6C60213068070B386C6023697A1660E
:10238000F58F42075D8FB716004083C7F60293F7BB
:102390000708A303F1000346710083C7F60293F711
:1023A0000708E394C7FE83477100B716004093F710
:1023B000F70F6388071293078008F3B7078093F736
:1023C00087083EC401000100B7170040930670055E
:1023D0002380D704930680FA2380D70401000100EC
:1023E00023AA070383C6170393E60608A388D70228
:1023F00023800704A247F3A70780010001001166AC
:10240000B71700407D16D45BC85F93854703A98E3C
:10241000F18EF5FA93068008F3B6068093F68608E7
:1024200036C601000100930670052380D704930689
:1024300080FA2380D7040100010098C103C7170365
:1024400013670704A388E70223800704B247F3A7B2
:10245000078001000100410182807D133368E3039E
:102460009308E016630E08003368F3039308D01650
:10247000630808009378330093B818009388D8163F
:1024800033081E01131E0801135E0E0155B5639338
:10249000E5030548638608000148630303002A88B2
:1024A00071087298FD15131E0801C205135E0E0116
:1024B000C18179BD13F8150063F4BF007908D5B761
:1024C00013381800E5BF83C7F60293F70708A30384
:1024D000F1000346710083C7F60293F70708E394FF
:1024E000C7FE8347710093F7F70FF1DFE9B531714C
:1024F0004AD966CB06DF22DD26DB4ED752D556D32E
:102500005AD15ECF62CD6AC96EC7AA8C02D8971025
:102510000000E78020B12A8993078008F3B707807D
:1025200093F787083EDA01000100B7170040130750
:1025300070052380E704130780FA2380E704010075
:10254000010003C7F7021377770FA387E70203C7DA
:10255000F70213678700A387E70223800704D25797
:10256000F3A7078001000100054597000000E78000
:1025700060D6130780C13347E902116A93070AE85E
:1025800093065002BD69930BA004814A014B1304CA
:102590008008930470057D1AB347F9023307D70208
:1025A0003EC0FD873ECC938709A69309803E334702
:1025B000F7023AC27D873AC4334739038549B39954
:1025C000990193D93940B306D702B30B7703B3C649
:1025D000F602B3CBFB0236C6FD8636C893D6FB4166
:1025E00036CEB7460F00938606243349D902856656
:1025F000938606FAB3969601B389E90213076055EC
:102600003309D90293060010B389E9023349D9028C
:10261000B3C9F9029316390036CA37190040FD864E
:1026200036D0930D090493D7F9413ED2F336048096
:1026300093F6860836DC01000100930770052380BD
:10264000FD00930680FA2380DD000100010083462F
:10265000390593F6860FA309D9048346390593E615
:102660001600A309D90423800D00E256F3A60680C4
:1026700001000100130C80FA116DF336048093F60B
:10268000860836DE01000100930770052380FD00F7
:1026900023808D010100010083463905216693E600
:1026A0000602A309D90483560905B3E6A601231837
:1026B000D90483560905D18E2318D90423800D002F
:1026C000F256F3A60680010001008346390593F611
:1026D00006026381061A03463905218A6DDE081851
:1026E00097100000E7800098733604801376860800
:1026F000B2C20100010023809D0023808D010100F2
:102700000100B717004003C637051376F60DA389FD
:10271000C70403C6370513660602A389C704835698
:1027200009052166B3E6A6012318D90483560905D5
:10273000D18E2318D90423800D009646F3A6068077
:10274000010001008346390593F60602638B0614E7
:1027500083463905A18AEDFE97000020E780A0930B
:10276000AA8636D497000020E780E092A256E30ABA
:10277000D5FE835609054255B3E6A6012318D904B0
:1027800097100000E780C08F83463905A18AEDDEEF
:10279000035609058346290582473376CA00B306E6
:1027A000DA0293D5F641B296B388F640E24733B8E1
:1027B000C6002E983308F840A247B3B61601330876
:1027C000D84063C70701631DF800924763FA1701F9
:1027D000C247634FF80E63950701B24763EAF80EEC
:1027E000894663E9660FF2469315180013D3F80182
:1027F0005E8613951800B365B30042D646D497B0F1
:102800000100E780A07A3258050B137BFB0F63476A
:102810000001631A0838A2586387083813081500A6
:10282000B336A800B69513D6F5013298B336C80072
:10283000AE9613581800FE06B3E606017336048000
:1028400013768608B2C60100010023809D00238014
:102850008D01010001000356C902B296C206C18271
:102860002316D90223800D00B646F3A60680010088
:10287000010021B5F336048093F68608B6C0010046
:10288000010023809D0023808D010100010083460B
:10289000390593E60602A309D90423800D00864674
:1028A0000DB5F336048093F68608B6C40100010026
:1028B00023809D0023808D0101000100834639059E
:1028C00093E60602A309D90423800D00A646BDB5F0
:1028D000E30B0BF0F336048093F68608B6C80100CC
:1028E0000100930680FA23809D002380DD00010013
:1028F00001008346390593F5FC0F93F6860FA30973
:10290000D90483463905CD8EA309D90423800D004F
:10291000C646F3A6068001000100130580FA0346AF
:102920003905930639051D8A631C96297336048080
:1029300013768608B2CC01000100130680FA2380CA
:102940009D002380CD000100010003C60600137620
:10295000F60D2380C60003C6060013660602238018
:10296000C600835609051166D18E2318D9048356F3
:1029700009052166D18E2318D90423800D00E6466F
:10298000F3A6068001000100130680FA834639058C
:1029900093F606026380062683463905130C390533
:1029A000A18AFDDA081897000000E780A06BF336D3
:1029B000048093F68608B6D001000100930680FAE1
:1029C00023809D002380DD000100010083460C0070
:1029D000116693F6F60D2300DC0083460C0093E6A7
:1029E00006022300DC0083560905D18E2318D90482
:1029F000835609052166D18E2318D90423800D0042
:102A00008656F3A6068001000100130680FA83466D
:102A1000390593F60602638A062083463905A18AA2
:102A2000EDFE97F0FF1FE78000672A8C97F0FF1FED
:102A3000E7806066E30C85FF835609051166425501
:102A4000D18E2318D90497000000E7806063834685
:102A5000390513063905A18AFDDAF336048093F6A9
:102A60008608B6D401000100930680FA23809D00F9
:102A70002380DD00010001008346060093F6F60D79
:102A80002300D60023800D00A656F3A60680010081
:102A900001008356090503462905D247B376DA00BB
:102AA0003306CA021305800C9355F6413696330D52
:102AB000F6408257333CD6002E9C3336A601330CA9
:102AC000FC40330CCC403308850392564E86B33518
:102AD000A5033305A503C29597B00100E780004D1B
:102AE00063468001631E0C16630C0D161306150059
:102AF0003335A6002E959356F5013696B335D6009C
:102B0000AA959396F50105828585D18E6346B0001E
:102B1000639D051A638B061A0356C9021582330595
:102B2000D6003336C500B2956348B00063910524E2
:102B30001306F00F637DA622894663F356159307AB
:102B40008008F3B7078093F78708BED6010001001D
:102B500037170040930770052300F704930780FAA6
:102B60002300F704010001008356C702896781171B
:102B7000D58FC207C1832316F70223000704B65777
:102B8000F3A7078001000100FA506A54DA544A5949
:102B9000BA592A5A9A5A0A5BFA4B6A4CDA4C4A4D8D
:102BA000BA4D296182801308F5FF3335A800FD1561
:102BB0002E951356F5013298B336C800AA9695B9EA
:102BC000F336048093F68608B6CA0100010023801C
:102BD0009D002380AD000100010083463905CD8EA4
:102BE000A309D90423800D00D646F3A60680010070
:102BF000010035B3F336048093F68608B6CE0100A3
:102C0000010023809D002380CD0001000100834648
:102C1000390593E60602A309D90423800D00F64680
:102C2000F3A606800100010095B3F336048093F605
:102C30008608B6D20100010023809D002380CD00CC
:102C4000010001008346390593E60602A309D90471
:102C500023800D009656F3A606800100010045BBB7
:102C60009306F5FF33B5A600FD152E959355F50196
:102C7000AE96B3B5B600AA951396F501858269B5EF
:102C8000F336048093F68608B6D801000100930657
:102C900080FA23809D002380DD000100010083561F
:102CA000C9020566011693F6F60FD18EC206C182DF
:102CB0002316D90223800D00C656F3A60680010014
:102CC0000100850A93FAFA0F95B233E6B60045C2C1
:102CD0000356C9023305D0403338A000B305B040D5
:102CE000B385054115826345B000D1E16371A60843
:102CF000894663F0560593078008F3B7078093F77A
:102D00008708BEDA01000100B717004013077005FD
:102D10002380E704130780FA2380E7040100010001
:102D200003D7C7027D8B2396E70223800704D6577B
:102D300081BDF336048093F68608B6DC01000100FD
:102D4000930680FA23809D002380DD0001000100AE
:102D50008356C9020566011693F6F60FD18EC20698
:102D6000C1822316D90223800D00E656B9B7930716
:102D70008008F3B7078093F78708BEDE01000100E3
:102D800037170040930770052300F704930780FA74
:102D90002300F704010001000356C7029397560071
:102DA000B297C207C1832316F70223000704F65720
:102DB000C1BB914763EEB70217D701001307870A1B
:102DC0008A05BA959C41BA978287B717004003A736
:102DD000470B1345F5FF698F23AAE70A03A7070BE3
:102DE000698F23A8E70A03A7070A798D23A0A70AFA
:102DF0008280B717004083A6470B1347F5FFF98E73
:102E000023AAD70A83A6070B558D23A8A70A83A652
:102E1000070A758F23A0E70A8280B717004003A72F
:102E2000470B498F23AAE70A03A7070B1345F5FFB2
:102E300045BFB717004083A6470B1347F5FF758FB3
:102E400023AAE70A03A7070A598D4DB7B717004011
:102E500003A7470B498FEDB7914763EEB70217D72A
:102E60000100130767018A05BA959C41BA978287CA
:102E7000B717004003A7470D1345F5FF698F23AA35
:102E8000E70C03A7070D698F23A8E70C03A7070C1E
:102E9000798D23A0A70C8280B717004083A6470D29
:102EA0001347F5FFF98E23AAD70C83A6070D558D7E
:102EB00023A8A70C83A6070C758F23A0E70C82809C
:102EC000B717004003A7470D498F23AAE70C03A7B4
:102ED000070D1345F5FF45BFB717004083A6470D03
:102EE0001347F5FF758F23AAE70C03A7070C598D2D
:102EF0004DB7B717004003A7470D498FEDB779715C
:102F000022D43714004026D24AD0035924028354D5
:102F1000040206D64209C2044ECE52CC56CA1359F8
:102F20000901C1802DE11379F9F793F4F49F420967
:102F3000C20413590901C18093078008F3B70780C1
:102F400093F787083EC40100010093077005230032
:102F5000F404930780FA2300F40401000100231114
:102F600024032310940223000404A247F3A707803C
:102F700001000100B250225492540259F249624AAF
:102F8000D24A45618280B7F5070081463000B1051D
:102F9000194597000020E7806081A2471397270119
:102FA000E34A07FC1369090893E404409309800885
:102FB000F3B7098093F787083EC001000100930A28
:102FC000700523005405130A80FA2300440501000C
:102FD00001002311240323109402230004048247D8
:102FE000F3A7078001000100294597F0FF1FE78044
:102FF0006034F3B9098093F989084EC201000100D9
:1030000023005405230044050100010083570402F6
:1030100093E707202310F402230004049247B9B772
:10302000B71700408847420541819377050491EB2B
:103030009377F5013755E801130505803345F5020F
:1030400082809377050C130700046397E70093775A
:10305000F50137459C1CCDB72165130505D082804D
:1030600037E700E01C435443A183E206D58F1CC11F
:10307000FD572320F7182322F718828013178500A5
:10308000B7E700E023A0E710618123A2A7108280A8
:10309000B7F700E08847CC47828081473737004048
:1030A000A14663C4C700328582800345B740E38EE2
:1030B000A6FE3385F5000345050085072304A740D8
:1030C000CDB7970700209387E7EE9C431737002082
:1030D0001307C7063E95636EE500173700201307F8
:1030E00067526368A700170700202325A7EC3E85D9
:1030F0008280FD57EDBF8280411122C406C62A841A
:1031000097000000E78000F22947B307E502B240CC
:103110008D83B3D7870222449507B3D7E7023737A9
:103120000040C207C1832316F70041018280378522
:10313000030041111305054006C697000000E78013
:10314000E0FBB7370040130770F82381E7000D4715
:10315000A381E70013070004A380E7000547238746
:10316000E700B240410182803737004083472700A3
:103170001A0593F7F703C98F93F7F70F2301F700A9
:103180008280B737004003C7170019C9D98DA380C3
:10319000B70003C70700136787002380E70082801A
:1031A00093C5F5FFF98DA380B7008280AE872A878B
:1031B000B736004021463738004089E71703000042
:1031C0006700A3F383C8B600E30916FF0507834829
:1031D000F7FFFD17C20723041801C183F9BF41118E
:1031E00022C406C62A8497000000E780A0E329478E
:1031F000B307E502B2408D83B3D787022244950717
:10320000B3D7E70237370040C207C1832316F74020
:1032100041018280716541111305052006C69700A2
:103220000000E78000FCB7370040130770F82381E7
:10323000E7400D47A381E74013070004A380E74060
:1032400005472387E740B24041018280CC414111CC
:1032500006C6328503C6150083C5050022064D8EBD
:1032600042068D654186138875A2630C0611634B77
:10327000C804138845A26300060D634AC8009385FD
:1032800035A26301B6082390060029464DA0138895
:1032900055A26305060D938565A2E316B6FE8D451E
:1032A0001D4663E6E5081146198E63F3C7003E86A6
:1032B000B7E704002390C600FC4797D5010093852B
:1032C000E5BD9DA0138895A263030611634E060D0C
:1032D0001388A5A263000613938505A5E315B6FA26
:1032E00099451D4663E5E504198E63F3C7003E86E4
:1032F000B7E704002390C600FC479705002093859C
:10330000A5D51DA09D451D4663E3E5022146198E06
:1033100063F3C7003E86B7E70400FC472390C6006E
:103320009705002093858533BA9582970146B24070
:10333000328541018280AD451D46E3EAE5FE314616
:10334000198E63F3C7003E86B7E704002390C600DA
:10335000FC4797D501009385E5B6F9B7B1451D4601
:10336000E3E7E5FC3546198E63F3C7003E86B7E711
:1033700004002390C600FC4797D50100938585B5CE
:1033800065B78D451D46E3E4E5FA1146198E63F3F2
:10339000C7003E86B7E704002390C600FC4797D5D8
:1033A0000100938565B049B78D451D46E3E1E5F819
:1033B0001146198E63F3C7003E86B7E704002390D9
:1033C000C600FC4797D50100938585B2B1BFA545DE
:1033D0001D46E3EEE5F42946198E63F3C7003E86E9
:1033E000B7E704002390C600FC4797D501009385FA
:1033F00065AC1DBFB5451D46E3EBE5F23946198EB8
:1034000063F3C7003E86B7E704002390C600FC477D
:1034100097D50100938585A701BFB7E7040003A3F3
:10342000071397060020938626C24146A545170537
:103430000020130565B802832D455DE703C505002F
:103440000947631FE50803A84500411106C6034765
:10345000180032850346080022074168518F9308FF
:1034600028FE6307170563E9E800051863030703EF
:1034700023900600294591A8130648FE630AC70455
:103480001518E31707FF15463E87637BF6001547BF
:1034900001A8130600023E876374F60013070002BA
:1034A000B7E704002390E600FC471316070111A8B4
:1034B0003E8691C30546B7E70400FC472390C6004B
:1034C0004206CC45418282970145B240410182804B
:1034D000130600083E87E375F6FC13070008C9B71A
:1034E0002390060005458280828041677917630436
:1034F000E504411122C406C685472A84639FF5006E
:10350000B7E7040022852244B24003A3871397053E
:1035100000209385E52E4101028389476399F500D8
:10352000B7E7040083A7070B8545829771D9B2409E
:103530002244410182808280797122D452CC2E842F
:103540002A8A97D501009385A59C17D501001305FC
:10355000A59E06D63AC626D24AD0B68432894ECE29
:1035600097B00100E780C0EFA68517D501001305CD
:10357000A59D97B00100E780A0EE294597B0010016
:10358000E780E0F28347840093F70702E1E783498D
:1035900004008947054532476396F908544083C7BC
:1035A000160083C60600A207D58FC166138616FED5
:1035B000638CC7028D16638FD7068D66938626901F
:1035C00029456391D706B7E70400A285225403A3D7
:1035D0004714B250F249A6864A869254025952853F
:1035E000624A8547456102832D450DEF930700022E
:1035F000354563E99702B7E70400FC4748441306E2
:103600000002CA8582978149970700209387072087
:103610009C43014581CB9C4391C74E852686CA8534
:1036200082970145B250225492540259F249624A9B
:10363000456182802D457DF79307700F3545E3E3A3
:1036400097FEB7E70400FC4748441306700FCA858D
:1036500082975DBF2145F9B7411122C437E40400C8
:103660008327841326C2AA84416506C697050020D5
:10367000938505197D1582978327C40A17050000D5
:103680001305E5E68588829795C003230413224439
:10369000B240924497060020938686AD4146C545C8
:1036A000170500201305C59B41010283B240224447
:1036B000924401454101828019C59707002023A744
:1036C000A71401458280454582801147636AA70A95
:1036D00097D60100938686820A05369518414111D6
:1036E00006C63697AE87B28502871307000261458A
:1036F000639DE700B7E70400FC47130600021705C7
:103700000020130525F682970145B24041018280D1
:1037100005476145E39BE7FEB7E70400FC47054624
:1037200017050020130505F6F9BF1307700F614553
:10373000E39DE7FCB7E70400FC471306700F17058D
:103740000020130565F4C1B7130700086145E39E27
:10375000E7FAB7E70400FC47130600081705002046
:10376000130505024DB715476145E390E7FAB7E742
:103770000400FC471546170500201305A50861B78E
:1037800009458280411126C2B7E4040083A7C4130F
:1037900022C44AC006C62E8497050020938545069C
:1037A0002A898297058905C5970700209387478B4B
:1037B00083D7A70BA28503A3440D2310F400224452
:1037C000B24092444A850249014641010283B24017
:1037D00022449244024949454101828097070020D2
:1037E000238807029707002023A60702B717004087
:1037F00003A7070CB706C0FFFD16758F23A0E70CC3
:1038000003A7070DB7064000558F23A8E70C03A7B1
:10381000070C3D9B23A0E70C03A7070D13670701C7
:1038200023A8E70C8280B717004003A5470C83A7A5
:10383000470C598113451500C18B058999E3136520
:1038400025009707002083C7A7FC6380A70297077E
:103850000020238FA7FA11C997070020938787FBC1
:1038600003A307006303030002838280114517F35B
:10387000FFFF670003C8411193962500AA852D45D7
:1038800006C697F0FF1FE78060F2B2400145410194
:103890008280011122CC06CE3714004026CA4AC8C5
:1038A0004EC652C483447405034AB4058349840553
:1038B0000349940597F0FFFFE780809E8347A405A6
:1038C00093F4F40F137AFA0F93E71700230DF4041F
:1038D00093F9F90F1379F90FB717004003C7A7053C
:1038E000058B6DFF03D5C705A38D4705238C3705D1
:1038F000A38C2705A38B9704F2406244D24442492B
:10390000B249224A0561828041119397050122C480
:1039100006C626C2C1872E8463DC0700B7E4040014
:10392000FC54829719C1BC5482972165218D15A83A
:1039300093F7150013C515008DE793F725009DC774
:1039400097000000E78060EEB7E70400BC4F130665
:10395000000A894517050020034545EC8297134569
:103960002400B24022449244410182809397250171
:1039700063D80702B7E4040083A7C41E82979700A8
:103980000000E780E0EEBC4C375607001306063017
:10399000896517050020034565E88297096579B7B1
:1039A000939715010145E3DE07FA17C501001305DA
:1039B000A56197B00100E78080C2B7E70400BC4F63
:1039C00013060064916517050020034525E58297DD
:1039D0001165A9BF2D71232A9110FD74E98C232C48
:1039E000811023282111232631112A84AE8932899E
:1039F000930600100A86A6852D45232E111097F0F8
:103A0000FF1FE780A0DA13154401B7E70400FC4765
:103A100051810A0513962900CA850A958297A685C1
:103A200085660146254597F0FF1FE78020D80A8666
:103A3000A68593060010294597F0FF1FE78000D761
:103A40008320C11103248111832441110329011111
:103A50008329C11015618280B7F7070003C70701EA
:103A6000411106C622C426C24AC0A547631DF700FD
:103A700097000000E78040F6B24022449244024999
:103A800001454101828013942500AA843289A286CF
:103A9000AA850146254597F0FF1FE78020D1A28621
:103AA0004A86A685294597F0FF1FE78020D0E9B711
:103AB0001D71A2CC37E404005C5C485886CE4946B0
:103AC00097C501009385C54B829711E917C5010081
:103AD0001305454C97B00100E78060B001A0B7F630
:103AE00000E0795798CAFD57DCCA0567B7E700E0E0
:103AF00023A0E7101306F00290C223A0E7180100EC
:103B00000100370700201847130600048145970677
:103B1000002023A3E6D04157A38AE7403C4408088D
:103B20008297970700209387276C3EC88567138785
:103B30000740231AE1001D673ACC37070105130738
:103B400007103ACE938757D11307B00F2310E10225
:103B50002312F102054797F7FFFF9387A75323012D
:103B6000E1023ED817070000130727D1970700008E
:103B7000938767D2B7F50700BAC23EDC170700008B
:103B80001307C7ED97070000938787CE8146300063
:103B9000E1051945BAC43EDE97F0FF1FE78000C17A
:103BA00018088147994630003E960346060085076F
:103BB0000507A30BC700E398D7FEC24791C7035779
:103BC000410185676373F70001A0B7E7040083A78D
:103BD000470A08088297AA8511C917C5010013056D
:103BE000A53C97B00100E780A08701A0F64066449D
:103BF00025618280411126C2B7E4040083A704082E
:103C000006C622C417050000130545D08297170485
:103C100000201304A4C02300A40097000000E78044
:103C2000800297000000E780A0BB03450400224407
:103C300003A38405B2409244130600328965410112
:103C40000283797106D622D413078008F3370780E0
:103C500093F787083EC201000100B71700409305A3
:103C600070052380B704130680FA2380C70401007F
:103C7000010083C6F70293F6A60FA387D70223801D
:103C800007049246F3A606800100010073370780FF
:103C9000137787083AC4010001002380B70423800A
:103CA000C7040100010003C7F70213672700A387B9
:103CB000E70223800704A247F3A707800100010061
:103CC000054597E0FFFFE780E06097000000E78090
:103CD00020BA014781468147054685451305407E48
:103CE00097E0FFFFE780E06337E404003C446800AE
:103CF000514681458297B707C0A83EC8B787E803F9
:103D0000938707D03ECA97E7FF1F9387476B3EC64E
:103D10007C5868008297B2502254456182804111DC
:103D200097D501009385859017C501001305C5201F
:103D300006C697A00100E780A07217D50100130501
:103D4000A5A797A00100E780A071B24029454101D5
:103D500017A301006700A375411197D50100938552
:103D6000258E17C501001305251D06C697A0010065
:103D7000E780006F17D501001305C5A297A00100C9
:103D8000E780006EB2402945410117A3010067009A
:103D90000372411122C406C6834705002A849DC7C9
:103DA00097D501009385858F17C501001305C518A8
:103DB00097A00100E780C06A4C4017D501001305A9
:103DC000E5AD97A00100E780A0693DA058410DEF47
:103DD00097D501009385858C17C501001305C5157E
:103DE00097A00100E780C06717D50100130585ACD7
:103DF00097A00100E780C0662244B24029454101F6
:103E000017A301006700A36AA1679386D703631312
:103E1000D70297D501009385658817C50100130562
:103E2000A51197A00100E780A06317D50100130535
:103E300065A97DBFED0797D501009385258617C538
:103E400001001305650F631BF70097A00100E780D1
:103E5000206117D50100130525A859BF97A00100BF
:103E6000E78000604C4017D501001305E5A891BF1D
:103E7000411197C501009385E57D17C50100130524
:103E8000A50B06C697A00100E780805DB2402945DA
:103E9000410117A3010067008361797122D426D202
:103EA0004AD02E842A898145B2844800714606D6BC
:103EB00097E0FFFFE780602297F7FF1F9387074C8B
:103EC000DC4783D70700231421012313F100975007
:103ED0000000E78020819547A305F1009307401F6C
:103EE0003EC6FD572305A100230AF10097500000AC
:103EF000E78080932686A285480097500000E780DF
:103F00004081B250225492540259456182809717E1
:103F10000020239E077C971700202387076CB7E7B4
:103F20000400BC47411106C64146814517050020E3
:103F30001305051A829797200000E78060569720A6
:103F40000000E780C031014597500000E78020263F
:103F5000170700200347C7199307F00A6315F702F4
:103F60009307F0F889451705002013056518170712
:103F70000020230FF71697070020A38B07169750F2
:103F80000000E780604D97500000E780205A81458F
:103F9000370504009707002023AA0712970700207F
:103FA0002394071297070020238107129707002008
:103FB0002392070A970700202390070897070020FD
:103FC0002393071097070020239C071097300000C9
:103FD000E78000C5014597500000E780E05097C595
:103FE00001009385A56917C501001305E5F497A0A5
:103FF0000100E780E04617D501001305259697A03C
:104000000100E780E045B2402945410117A30100C6
:104010006700E349411122C406C626C293F7150082
:104020002E84638F0710814617F6FF1F1306463252
:104030008545170500200355E5FF97C00000E78080
:10404000E0B315C997C501009385056417C5010044
:10405000130585EE97A00100E780804017C5010099
:104060001305450597A00100E780803F294597A0EB
:104070000100E780C04397C501009385E56017C53F
:104080000100130565EB97A00100E780603D17C5AF
:1040900001001305650397A00100E780603C2945F6
:1040A00097A00100E780A04017F5FF1F1305052D1D
:1040B0005C4505472390E70097300100E780606486
:1040C00097C501009385455C17C501001305C5E63A
:1040D00097A00100E780C03817C50100130505004F
:1040E00097A00100E780C037294597A00100E7802D
:1040F000003C930710F817070020230BF7FE9707E3
:10410000002083D7E7F217070020A303F7FE170567
:1041100000201305E5FDA183914517070020230A20
:10412000F7FC97070020A38607FC97500000E78064
:10413000A03213451400B2402244924441018280CF
:1041400093F72500E1C3170700200357E7F745CB96
:1041500097060020938686F7944297D701009387AD
:10416000E78117060020034646F681451705002023
:10417000130505F697700000E780A0BFAA8441C12F
:1041800097C501009385055717C501001305C5DACA
:1041900097A00100E780C02CA68517C50100130574
:1041A00065F597A00100E780A02B294597A00100A5
:1041B000E780E02F97070020239807F0930710F877
:1041C000170700202306F7F29707002083D747E65A
:1041D00017070020A30EF7F0A18317070020230A7A
:1041E000F7F091458D4717050020130565F0170777
:1041F0000020A300F7F097500000E780E02513456A
:10420000240015BF93F74500D1C397C501009385DE
:10421000654E17C50100130525D297A00100E78060
:10422000202417C501001305A5EE97A00100E78023
:104230002023294597A00100E7806027930720F8F5
:10424000170700202306F7EA9707002083D787E0A7
:1042500017070020A30EF7E8A18317070020230A01
:10426000F7E8854717070020A305F7E89740000007
:10427000E780805B17050020130585E7914597507F
:104280000000E780601D1345440075B593F7850075
:10429000A9C797C501009385E54517C5010013051A
:1042A000A5C997A00100E780A01B17C50100130551
:1042B00065E797A00100E780A01A294597A00100B3
:1042C000E780E01E97070020239007E0977000002A
:1042D000E78000BA13458400B9BD93F70501D1C347
:1042E0008545170500200355E5D697500100E78066
:1042F000206C97C501009385E53F17C501001305A4
:10430000A5C397A00100E780A01517C501001305FC
:10431000A5E297A00100E780A014294597A001001D
:10432000E780E018930730F8170700202302F7DC36
:104330009707002083D707D217070020A30AF7DAD0
:10434000170500201305C5DAA1838D451707002046
:104350002301F7DA97500000E780001013450401AD
:10436000D9BB93F70502D1C797C50100938585385E
:1043700017C50100130545BC97A00100E780400E5A
:1043800017C50100130585DD97A00100E780400DEA
:10439000294597A00100E7808011930740F817078F
:1043A00000202307F7D49707002083D7E7C8170713
:1043B0000020A30FF7D2A18317070020230BF7D209
:1043C000854717070020A306F7D2970700202395FB
:1043D00007C697400000E780204517050020130519
:1043E00025D1914597500000E7800007134504024E
:1043F00099B393F70504FDC397C501009385852FF5
:1044000017C50100130545B397A00100E7804005DB
:1044100017C50100130505D697A00100E7804004E9
:10442000294597A00100E78080089707002083C7EF
:1044300027CC1307700A6386E7061307800A638C8C
:10444000E7081307600A6393E704930760F8170708
:104450000020230FF7C89707002083D7C7C6170788
:104460000020A307F7C8A183170700202303F7C87C
:10447000854717070020A302F7C8B145170500209C
:10448000130505C797500000E78000FD9740000026
:10449000E78080391345040497070020239507C25D
:1044A00059B9930770F8170700202303F7C497073B
:1044B000002083D747C117070020A30BF7C2A183B1
:1044C000170700202307F7C2854717070020A3031B
:1044D000F7C2994565B7930780F8F1B793F70508D8
:1044E0000145E38A07C497C501009385A52017C538
:1044F0000100130565A497A00100E78060F617C5C9
:1045000001001305A5C897A00100E78060F52945C3
:1045100097A00100E780A0F99307A0F817070020F3
:104520002308F7BC9707002083D787BB1707002015
:10453000A300F7BCA18317070020230CF7BA854717
:1045400017070020A307F7BA97070020239A07B898
:1045500097400000E780402D17050020130545B95E
:10456000914597500000E78020EF13450408E1B61D
:10457000411122C497C50100938585132A8417C56C
:1045800001001305659B06C697A00100E78040ED7A
:104590004C4017C501001305E52D97A00100E780E9
:1045A00020EC294597A00100E78060F00347040054
:1045B0009307F00F631FF70297C501009385450F1E
:1045C00017C501001305459797A00100E78040E952
:1045D0004C4017C501001305E52A97A00100E780AC
:1045E00020E82244B2402945410117A30100670099
:1045F00003ECB240224441018280B1C1411122C486
:1046000017C50100130545932E8497C501009385B6
:10461000250506C697A00100E78080E4A28517C59E
:1046200001001305653197A00100E78060E3224493
:10463000B2402945410117A30100670043E782808A
:10464000411122C426C22E84AA8497C501009385F5
:10465000E50117C501001305258E06C697A00100C8
:10466000E78000E017C501001305C52D97A00100E4
:10467000E78000DF294597A00100E78040E397C568
:1046800001009385A5FE970700202395979A17C5EB
:1046900001001305658A854497070020239A8798AF
:1046A0009707002023979798971700202391870456
:1046B00097A00100E780C0DA9715002083D5250375
:1046C00017C501001305852897A00100E78040D990
:1046D000294597A00100E78080DD971700202385FA
:1046E00097F097200000E78080B722859750000060
:1046F000E780E0AB054597500000E780E0DE97F7E4
:10470000FF1F9387A7C7DC4703D70700C167FD17C3
:104710006312F7022244B7E70400B240924403A3B5
:10472000870517F5FF1F0345E50F1306000A8545AA
:1047300041010283B240224492444101828001112E
:1047400022CC37E404005C5C06CE354697C50100F8
:104750009385C50717D501001305C5C1829711E9D7
:1047600017C501001305058397A00100E78020E726
:1047700001A097F7FF1F9387A70B3EC4B7F507006B
:10478000856793870780814617F6FF1F1306C609C2
:10479000E10519453EC697E0FF1FE78020017C44F4
:1047A000194697F5FF1F9385250817050020130567
:1047B000A58A8297340017F6FF1F1306E60697C5F1
:1047C00001009385A55217C501001305A5539760F5
:1047D0000000E780002F2A841DCD97C50100938536
:1047E00065F017B501001305257597A00100E78056
:1047F00020C7A28517C50100130545FE97A001003B
:10480000E78000C6294597A00100E78040CAF24032
:1048100062440561828097E00000E780609117C5DF
:1048200001001305A5F297500000E780402397A0F0
:104830000000E780A0E597500100E780204A17F5C7
:10484000FF1F130525B097500100E780C03217C540
:1048500001001305A5F097500100E780A04A2A84C3
:1048600097600000E780808997000100E7800022C0
:1048700097800100E78020BB97700000E780C0E1CF
:1048800097600000E78080FF97300100E78060E3D9
:1048900097C50100938505E517B501001305C569A6
:1048A00019C897A00100E780A0BBA28517C5010029
:1048B000130505F5A1B797A00100E78060BA17C5F9
:1048C0000100130525F697A00100E78060B929458E
:1048D00097A00100E780A0BD97300100E78040BFAE
:1048E00097F00000E78000DE55C9854537050400D4
:1048F00097200000E780C03297C50100938585DED0
:1049000017B501001305456397A00100E78040B586
:1049100017C50100130585F297A00100E78040B498
:10492000294597A00100E78080B897F7FF1F93877C
:10493000A79483D7070017170020231AF7DA8547B3
:10494000171700202302F7CA97200000E780C0AFA6
:1049500097200000E780A09017150020035525D967
:1049600097500000E780A084054597500000E7803D
:10497000A0B797C501009385E5D617B501001305CB
:10498000A55B97A00100E780A0AD17C50100130546
:1049900025ED97A00100E780A0ACADB597C501005B
:1049A000938545D417B501001305055997A001005B
:1049B000E78000AB17C50100130545FA97A0010079
:1049C000E78000AA294597A00100E78040AE014595
:1049D00069BF411122C437E404008327041A06C6C4
:1049E000829797500000E78040808327040817F5DE
:1049F000FFFF13056562829797F7FF1F2384A7E2E5
:104A000017F5FF1F1305859797400000E780601496
:104A10002244B240410117030000670083D2B7E788
:104A20000400FC471171A2DDCAD986DFA6DBCED710
:104A30002E8432892E86AA8517F5FF1F1305456B34
:104A4000829717F7FF1F1307A76A8347070093068C
:104A500080029387E70793F7F70FE3ECF610BA8924
:104A60008A0717B7010013076756BA979C43BA978E
:104A700082878D4797C50100938505C917B5010049
:104A80001305854B630FF40097A00100E780409D5C
:104A900017C501001305058697A00100E780409C1B
:104AA000BDA497A00100E780A09B17C501001305D6
:104AB000E58597A00100E780A09A294597A001000D
:104AC000E780E09E930720F8114697F5FF1F938536
:104AD00025624A8517F7FF1F230CF76097F7FF1F22
:104AE000A389076097F0FFFFE780603B2A841DC918
:104AF00097C50100938545C117B501001305C5434E
:104B000097A00100E780C095A28517C50100130595
:104B1000A58397A00100E780A094294597A00100F4
:104B2000E780E09897C50100938505BE17B50100A1
:104B30001305854097A00100E780809217C501000A
:104B40001305C58197A00100E7808091294597A0B2
:104B50000100E780C0954165930730FA054697F557
:104B6000FF1F9385E5587D1517F7FF1F2302F758A0
:104B700097F0FFFFE780A0322A841DC997C5010086
:104B8000938585B817B501001305053B97A0010073
:104B9000E780008DA28517B501001305E57A97A07F
:104BA0000100E780E08B294597A00100E780209075
:104BB000B7E70400BC4F0566130606C8A14517F504
:104BC000FF1F034525C68297FE506E54DE544E5992
:104BD000BE591161828091476303F40297C50100B9
:104BE000938585B217B501001305053597A001001F
:104BF000E780008717B501001305857971BDB7E718
:104C00000400FC4F914517F5FF1F0345A5C182978E
:104C100097C50100938545AF17B501001305C53150
:104C200097A00100E780C08317B501001305057840
:104C300097A00100E780C082294597A00100E78086
:104C4000008797400000E78020BE914535A4854746
:104C50006303F40297C50100938505AB17B5010006
:104C60001305852D97900100E780807F17B501001F
:104C70001305457515B597F7FF1F239D273DB7E72A
:104C800004000566BC4F130606C8C1450DBF8D471D
:104C90006303F40297C50100938505A717B50100CA
:104CA0001305852997900100E780807B17B50100E7
:104CB00013050573D5B3930740F8114697F5FF1F09
:104CC000938505434A8517F7FF1F2303F74297F79C
:104CD000FF1FA380074297F0FFFFE780401C2A8454
:104CE000E30405EE97C50100938505A217B5010001
:104CF0001305852497900100E7808076A28517B57B
:104D000001001305656497900100E78060752945EF
:104D100097900100E780A07945BD9147E31CF4F628
:104D2000B7E70400FC4F9305000217F5FF1F03458A
:104D300065AF829797C501009385059D17B5010062
:104D40001305851F97900100E780807117B501005A
:104D50001305856AF1BD894763E3870297C50100A2
:104D60009385859A17B501001305051D97900100DD
:104D7000E780006F17B501001305456931BB97F453
:104D8000FF1F83C4043797F7FF1F83C7773697C584
:104D9000010093856597A20417B501001305C51995
:104DA000DD8C97900100E780A06BA28517B501000C
:104DB0001305056797900100E780806AC2042945C2
:104DC00097900100E780A06EC1849305D4FF93966D
:104DD0000401C1824A8693F5F50F17F5FF1F1305ED
:104DE000553197200000E78060E7E35F90DC930790
:104DF00050F817F7FF1F230DF72E83C739002286BF
:104E000097F5FF1F9385C52E85074A8517F7FF1F66
:104E1000A301F72E97F0FFFFE78060082A84E305DF
:104E200005DA97C501009385258E17B50100130596
:104E3000A51097900100E780A062A28517C5010028
:104E4000130585AEC9B5894763E3870297C501009D
:104E50009385858B17B501001305050E979001000A
:104E6000E780006017B501001305455D35B1974037
:104E70000000E780609BA28517F5FF1F13054527FB
:104E800097400000E780405D81B38D476303F402E3
:104E900097C501009385458717B501001305C5091E
:104EA00097900100E780C05B17B501001305C55A54
:104EB000E5B6B76602000146B7750200054597E002
:104EC000FF1FE780A08E930760F817F7FF1F2301ED
:104ED000F72297F7FF1FA38E07209307000617F707
:104EE000FF1F2309F720894717F7FF1FA304F720A7
:104EF00097F7FF1F2381072097F7FF1FA38D071E3A
:104F0000C14717F7FF1F2309F71E930720F917F76B
:104F1000FF1FA303F71E314697F7FF1FA38FA71CA0
:104F200097F5FF1F9385C51C4A8597F7FF1F2386BA
:104F3000071C97F0FFFFE78080F62A84E30605C888
:104F400097B501009385457C17B501001305C5FE93
:104F500097900100E780C050A28517B501001305A6
:104F6000255155B3B1476303F40297B5010093850A
:104F7000A57917B50100130525FC97900100E7807E
:104F8000204E17B501001305655039B6B7E7040088
:104F9000FC4F9305000417F5FF1F0345A588829772
:104FA00097400000E7804088B145F9B5914763E339
:104FB000870297B501009385257517B50100130584
:104FC000A5F797900100E780A04917B501001305E8
:104FD000A54DD9B497F4FF1F83C4C41197F7FF1FE1
:104FE00083C73711A204DD8C8E04B77702006D14DD
:104FF000BE942286A68517B501001305254C97900F
:105000000100E780E045B7E70400FC47228697F5FA
:10501000FF1F9385350E2800829793160401C182E5
:105020003000A685094597D0FF1FE78020782A84A5
:1050300009C917B501001305254A97900100E780BB
:10504000005A930770F8194697F5FF1F9385450A94
:105050004A8517F7FF1F230DF70897F7FF1FA38B4C
:10506000870897F0FFFFE78080E32A84E30E05B40A
:1050700097B501009385456917B501001305C5EB88
:1050800097900100E780C03DA28517B50100130588
:10509000A54595B99947630BF41297B5010093851F
:1050A000A56617B50100130525E997900100E78073
:1050B000203B17B501001305A544F9BA914763E3F6
:1050C000870297B501009385256417B50100130584
:1050D000A5E697900100E780A03817B501001305F9
:1050E000A5435DBA97F4FF1F83C4C40097F7FF1F61
:1050F00083C73700A204DD8C8E04B77702006D14DD
:10510000BE942286A68517B5010013052542979007
:105110000100E780E034B7E70400FC47228697F5FA
:10512000FF1F938535FD2800829793160401C182E5
:105130003000A6850D4597D0FF1FE78020672A84A1
:1051400009C917B501001305254097900100E780B4
:105150000049930780F8194697F5FF1F938545F995
:105160004A8517F7FF1F2305F7F897F7FF1FA3835B
:1051700087F897F0FFFFE78080D22A84E30605A432
:1051800097B501009385455817B501001305C5DA99
:1051900097900100E780C02CA28517B50100130588
:1051A000E53B95B699476303F40297B501009385F3
:1051B000A55517B50100130525D897900100E78084
:1051C000202A17B501001305E53AF9B0B7E7040046
:1051D000FC4F9305000417E5FF1F0345A564829764
:1051E00097300000E7804064994579B18D476303AB
:1051F000F40297B501009385255117B501001305F9
:10520000A5D397900100E780A02517B501001305ED
:10521000E53759B017B501001305453897900100DF
:10522000E780E03B1305C01297D0FF1FE7806011B5
:10523000014597E0FFFFE780E0E20D459710000091
:10524000E780009F294597D0FF1FE780800F97D008
:10525000FF1FE780E0FF8DBA99476303F40297B51B
:1052600001009385654A17B501001305E5CC9790B9
:105270000100E780E01E17B501001305E53229B8EB
:1052800017F7FF1F034717E797F7FF1F83C787E647
:1052900022075D8F9166BA96C2061166C182130617
:1052A000F6EF8D476365D60297E7FF1F9387070DDB
:1052B0009C4B17F6FF1F0346D6E39386C7002DC20B
:1052C00003D6070069CA8907E39CD7FE89471307FD
:1052D000A0F8114697F5FF1F938585E14A8597F65B
:1052E000FF1F2387E6E017F7FF1FA304F7E097F0FF
:1052F000FFFFE780C0BA2A84E308058C97B5010058
:105300009385854017B50100130505C397900100EB
:10531000E7800015A28517B501001305252AE5B21F
:1053200003D60700630EE60A8907E39BF6FE8D4766
:1053300079BF91476304F40297B501009385C53C9A
:1053400017B50100130545BF97900100E780401194
:1053500017B50100130505286FF00FF4B7E7040037
:10536000FC4F9305000817E5FF1F0345A54B8297E7
:10537000C9B897B501009385253917B50100130504
:10538000A5BB97900100E780A00D17B5010013059C
:10539000E5256FF06FF02390E70017E5FF1F130579
:1053A000E5FD97200100E780203897B5010093853F
:1053B000A53517B50100130525B897900100E780C2
:1053C000200A17B501001305652397900100E780B7
:1053D0002009294597900100E780600D8147C5BDF0
:1053E0002390070017E5FF1F130545F997200100DB
:1053F000E780803397B501009385053117B501002B
:10540000130585B397900100E780800517B501006B
:10541000130545205DBF411122C406C68347050020
:105420002A849DC797B501009385C52917B501004A
:10543000130585B097900100E78080024C4017B5B6
:1054400001001305A55497900100E7806001E1A0D9
:105450005841B707CF009387777D631DF70697B54F
:1054600001009385252617B501001305E5AC97903B
:105470000100E780E0FE1C448356E4008355C4002D
:1054800003C6070017B501001305C5519790010029
:10549000E78000FD294597900100E7804001035710
:1054A000E4009707002083D787246309F70083551A
:1054B000C400084497E0FFFFE78080CF0356E40074
:1054C0008355C40008442244B240410117F3FFFF52
:1054D00067002355B707CC009387777D6315F704E2
:1054E00097B501009385051E17B501001305C5A4E6
:1054F00097900100E780C0F61C448356E400835572
:10550000C40003C6070017B501001305A54997900D
:105510000100E780E0F42244B2402945410117939D
:1055200001006700C3F8B707CE009387777D630457
:10553000F70297B501009385E51817B5010013052B
:10554000A59F97900100E780A0F14C4017B501009E
:105550001305853ACDBDB240224441018280B7E7B0
:105560000400FC4741112E8606C622C426C24AC04A
:105570002E842A89AA8517F5FF1F130565B7829720
:1055800097B501009385051A17B501001305C59A53
:1055900097900100E780C0EC97F5FF1F83C545B5E4
:1055A00017B50100130505C097900100E78040EB97
:1055B000294597900100E78080EF97F4FF1F9384BF
:1055C00024B383C7040041479387070693F7F70F77
:1055D000636AF75C17B70100130787A98A07BA97B0
:1055E0009C43BA9782879D476307F40297B50100F1
:1055F0009385451317B50100130505949790010095
:10560000E78000E617B50100130545BA9790010041
:10561000E78000E5ADAC97F7FF1F83C777ADDDCB23
:1056200017F7FF1F0347F7AC97F7FF1F83C767AC58
:1056300022075D8F97F7FF1F83C7C7ABC2075D8F38
:1056400097F7FF1F83C717ABE207D98F17F7FF1F25
:10565000232EF7A683C7640097B501009385850CB8
:1056600017B501001305458D17F7FF1F230FF7A48A
:1056700097900100E780C0DE97F7FF1F938707A58B
:105680008C4317F6FF1F034646A417B50100130508
:10569000A5B397900100E780A0DC29459790010011
:1056A000E780E0E097F7FF1FA38407A42244B240FD
:1056B00092440249930700F817F7FF1F230AF7A245
:1056C0009D4517F5FF1F1305A5A2410117430000D3
:1056D000670083D897600000E780008997F7FF1F75
:1056E0002389A7A09357850017F7FF1FA303F7A0EF
:1056F000935705012A8417F7FF1F230DF79E935731
:105700008501014517F7FF1FA306F79E976000006C
:10571000E780408697F7FF1F238FA79C97B501006E
:105720009385450017B50100130505819790010089
:10573000E78000D317F6FF1F0346E69BA28517B547
:1057400001001305E5A9B1B7CD476303F40297B58E
:105750000100938525FD17A501001305E57D9790B0
:105760000100E780E0CF17B501001305E5A879BD7A
:1057700037E404007C44414697F5FF1F9385559715
:1057800017F5FF1F1305C594829717F5FF1F130523
:10579000259497100000E78040C497100000E78030
:1057A00000AC97F7FF1F83C7C79517F7FF1F034785
:1057B0003795A20703238405D98F17F7FF1F2315F9
:1057C000F7901306000A89452244B24092440249E8
:1057D00017E5FF1F03450505410102838D4763035C
:1057E000F40297B501009385E5F317A501001305B1
:1057F000A57497900100E780A0C617B501001305B6
:1058000065AF29B517F4FF1F0344A48E97F7FF1F58
:1058100083C7178E97B501009385C5F0220417A59D
:105820000100130565715D8C97900100E78040C30E
:10583000A28517B501001305A59D97900100E7808B
:1058400020C2294597900100E78060C60D4697F574
:10585000FF1F9385E589228597E0FFFFE78020649D
:10586000AA8421C197B501009385C5EB17A5010056
:105870001305856C97900100E78080BEA68517B55B
:1058800001001305259A97900100E78060BD22442E
:10589000B240924402492945410117930100670033
:1058A00003C197E7FF1F2397877AB7E704001166C4
:1058B00003A38705130606E8914539B78D476303AF
:1058C000F40297B501009385E5E517A501001305DE
:1058D000A56697900100E780A0B817B501001305F1
:1058E00025B02DB317F4FF1F0344A48097F7FF1FC3
:1058F00083C7178097B501009385C5E2220417A5D9
:105900000100130565635D8C97900100E78040B549
:10591000A28517B501001305259297900100E78035
:1059200020B4294597900100E78060B80D4697E5BF
:10593000FF1F9385E57B228597E0FFFFE7802056D8
:10594000AA841DC197B501009385C5DD17A5010087
:105950001305855E97900100E78080B0A68517B596
:1059600001001305A58E05B797E7FF1F2396876CE7
:10597000B7E70400116603A38705130606E893053D
:10598000000299B5894763E3870297B501009385C3
:1059900065D917A501001305255A97900100E780E6
:1059A00020AC17B50100130565A68DB197E4FF1F64
:1059B00083C4247497E7FF1F83C7977397B50100CB
:1059C000938545D6A20417A501001305E556DD8C85
:1059D00097900100E780C0A8A68517B501001305C0
:1059E000658897900100E780A0A72945979001005E
:1059F000E780E0AB228697E5FF1F9385656F2685DC
:105A000097E0FFFFE780A0492A84630E051A97B547
:105A10000100938525D117A501001305E551979045
:105A20000100E780E0A3A28517B501001305C58436
:105A300099BD854763F98718834519002244B24010
:105A400092440249B335B00097E7FF1F238EB76039
:105A500017B5010013058583410117930100670005
:105A600023A0A2852244B24092444A8502494101C2
:105A7000170300006700032299476303F40297B5F8
:105A80000100938525CA17A501001305E54A9790E3
:105A90000100E780E09C17B501001305E5B0BDB635
:105AA00017E4FF1F0344E46497E7FF1F83C75764AD
:105AB00097B50100938505C7220417A501001305BA
:105AC000A5475D8C97900100E7808099A28517A576
:105AD00001001305257D97900100E7806098294516
:105AE00097900100E780A09C194697E5FF1F9385DA
:105AF0002560228597E0FFFFE780603AAA841DC1F8
:105B000097B50100938505C217A501001305C5428D
:105B100097900100E780C094A68517A501001305A2
:105B2000657995B397E7FF1F239C875AB7E7040071
:105B3000116603A38705130606E89305000869B1FB
:105B4000854797B501009385E5BD17A501001305AD
:105B5000A53E630BF40097900100E780609017A5C5
:105B60000100130565765DB497900100E780408FD2
:105B700017A501001305C57697900100E780408EB8
:105B8000294597900100E78080922244B2409244D8
:105B9000024997E7FF1F239907524101175300005D
:105BA0006700032D97B501009385C5B717A50100C0
:105BB0001305853897900100E780808A17B50100AA
:105BC0001305C5A2A1B4B240224492440249410146
:105BD0008280411106C622C497E0FFFFE780202C97
:105BE0009377F50FA1C32A8497B50100938505B576
:105BF00017A501001305453497900100E780408602
:105C00009375F40F17B50100130505D297900100A5
:105C1000E78000852244B2402945410117930100E5
:105C20006700E388B240224441018280411122C4CE
:105C300091462A8417E6FF1F1306C6599D652D4518
:105C400006C697D0FF1FE78060B6B7F7070003C707
:105C50000701A5476313F70001A093060010014652
:105C60009D65254597D0FF1FE78040B497E7FF1F4C
:105C7000238287562244B240914617E6FF1F13063F
:105C800066559D652945410117D3FF1F670003B283
:105C90005171CAD137E904008327C904A2D52E86E1
:105CA00086D7A6D32E84AA8517E5FF1F1305454482
:105CB000829797E7FF1F83C7A7431307700A63877D
:105CC000E710636CF7001307600A6384E704BE50B3
:105CD0002E549E540E596D6182801307800A63888A
:105CE000E7161307900AE394E7FE8D476309F41C57
:105CF00097B50100938585D617A501001305C52327
:105D000097800100E780C07517B50100130545D2E3
:105D100025A08D47630CF40297B50100938505D447
:105D200017A501001305452197800100E780407306
:105D300017B50100130505C997800100E78040727F
:105D4000294597800100E780807651B7854717B5D0
:105D500001001305E5C817E7FF1F2307F7309790E9
:105D60000100E780C087B7750200B76602000146F0
:105D7000054597D0FF1FE78060A3930760F817E7FA
:105D8000FF1F2307F73697E7FF1FA3840736930704
:105D9000002617E7FF1F232FF734E57793870721A6
:105DA00017E7FF1F231AF734B14597E7FF1F238634
:105DB000073497E7FF1FA382A73417E5FF1F1305DA
:105DC000253397300000E780206911B7914763E3DE
:105DD000870297B50100938565C817A501001305D3
:105DE000A51597800100E780A06717B5010013058E
:105DF00025C199B797E4FF1F83C4C42F97E7FF1FFE
:105E000083C7372FA204DD8C8327C9046D14228633
:105E100097E5FF1F9385152E280082978E04931611
:105E20000401B7750200C1823000A695094597D0DC
:105E3000FF1FE780A097930770F817E7FF1F23095C
:105E4000F72A994597E7FF1FA386A72ABDB7914771
:105E500063E3870297B50100938545C017A501004C
:105E60001305850D97800100E780805F17B501005D
:105E7000130585BAD1B597E4FF1F83C4A42797E71C
:105E8000FF1F83C71727A204DD8C8327C9046D1465
:105E9000228697E5FF1F9385F525280082978E04BB
:105EA00093160401B7750200C1823000A6950D4516
:105EB00097D0FF1FE780808F930780F8BDBF17B58D
:105EC0000100130525B897800100E7804071130594
:105ED000C01297C0FF1FE780C046014597D0FFFF63
:105EE000E78040180D4597000000E78060D4294501
:105EF00097C0FF1FE780E04497C0FF1FE780403551
:105F0000F9B341114AC097F6FF1F83D6467E328906
:105F100017D6FF1F0356A64822C426C206C62A84E7
:105F2000AE8497000000E780805F35C12DC099479F
:105F300063FF97048347140003470400A207D98F27
:105F400013978700A183D98FC2073167C1831307D5
:105F5000C755639EE70297D7FF1F83D74744A30126
:105F6000F400A1832302F40097F7FF1F83D727785B
:105F700091C7A302F400A1832303F400A68517B5FB
:105F800001001305A5B197800100E780604D97F7E8
:105F9000FF1F83C76765B9CF97D5FF1F83D52540FE
:105FA00017B50100130545B197800100E780404B0C
:105FB0002686A28517D5FF1F0355653E9700000072
:105FC000E78060C16301090497E7FF1F83C787214A
:105FD0009DCB95C897E7FF1F83C707098DE72285EB
:105FE0002244B2400249A685924441011733000081
:105FF0006700834617B50100130505AD97800100C2
:10600000E780E05DC1B7B2402244924402494101B9
:106010008280834755008345450017B5010013056D
:10602000A5A6A207DD8D178301006700634317B59E
:106030000100130565A4178301006700435A8D47CB
:1060400063FBB70A011126CA06CE22CC03443500F1
:1060500097E4FF1F83C4141997B50100938585A7A2
:10606000B337800017E7FF1FA30EF71609C497B5D3
:1060700001009385E5A617B501001305E5A69780F5
:106080000100E780E03D97E7FF1F83C7B7156386F0
:10609000970097000000E780402697E7FF1F83C71F
:1060A00077148DC785472306F100B7E7040083A75F
:1060B00047177000854513055030829717B50100CA
:1060C000130585A397800100E78060519967938746
:1060D00057EE2316F100680085479145A30781001C
:1060E0002307F10097300000E7800037F240624458
:1060F000D244056182808280894763F7B708011125
:1061000022CC06CE26CA8344250085472A84639D77
:10611000F404914763F5B704034545008347340011
:1061200022055D8D97D7FF1F239BA72697000000B0
:10613000E780C0479967938767EE2314F100834790
:10614000340023059100A305F100834744009545E1
:1061500028002306F10097300000E780E02FF2408E
:106160006244D24405618280FDF89967938767EEA7
:106170002314F10097D7FF1F83D76722A305F100EF
:1061800023050100A183E1B782800111996722CC28
:10619000D51717F4FF1F130424452314F100834778
:1061A000040026CA97F4FF1F938464542305F1006A
:1061B00083D7040028009545A305F100A18306CEEE
:1061C0002306F10097300000E780002903D6040081
:1061D0008345040017B501001305859397800100DE
:1061E000E7800028F2406244D244056182809D67C6
:1061F0007971D9172316F10097F7FF1F83C7C73EA0
:1062000006D62307F100A9C3B7E70400FC474146BF
:1062100097E5FF1F9385C5EB1305F1008297680092
:10622000CD4597300000E780202397F5FF1F83C5F9
:10623000A53B17B501001305A59097800100E780E5
:106240002022B25045618280B7E70400BC47414636
:1062500081451305F1008297D9B7B76702045D71D4
:10626000938757AA3EC085672312F10097F7FF1F57
:106270009387873783C70700A2C4A30301002303C2
:10628000F10097F7FF1F9387874683D7070037E40E
:10629000040086C62314F10097D7FF1F93872710A9
:1062A00083D70700414668002315F1007C4497E539
:1062B000FF1F9385E5E18297F1450A85970000006D
:1062C000E780E021231EA1007C448A8508107946DE
:1062D00082973C441305E1030946814582971010DB
:1062E00093050002014597D0FFFFE780403EB6408E
:1062F000264461618280B7C7A55A01119387C733CD
:106300003EC497E7FF1F83C7F7ED3EC6B7F7070008
:1063100003C7070106CE22CCA5476313F70001A0EF
:106320001164930504F0930600100146254597C0BB
:10633000FF1FE780A0473000930504F0A1462945E0
:1063400097C0FF1FE780804697E5FF1F83C595E94B
:1063500017B501001305858F97800100E780401075
:10636000F24062440561828001119165A1463000CE
:10637000938505F02D4506CE97C0FF1FE7800043AB
:106380002247B7C7A55A9387C7336314F702B245AC
:1063900017A501001305C57EB335B00097E7FF1FB1
:1063A000A382B7E497800100E780800BF24005618B
:1063B0008280814517A501001305C57E97E7FF1F61
:1063C000A38207E297800100E78080099700000020
:1063D000E780A0F2E1BFB7C7A55A79719387F73577
:1063E0003EC6B7E70400FC47AA8506D622D441463C
:1063F00008088297B7F7070003C70701A54763138B
:10640000F70001A01164930504E89306001001460B
:10641000254597C0FF1FE78060397000930504E8A9
:10642000D146294597C0FF1FE780403817B50100C6
:106430001305858597800100E780601AB2502254C9
:106440004561828079719165D1467000938505E838
:106450002D4506D697C0FF1FE78040353247B7C7A6
:10646000A55A9387F73517A501001305A57B63107F
:10647000F702B7E70400FC4717E5FF1F130545C502
:1064800041460C08829717A501001305A577978050
:106490000100E780C014B25045618280B7F7070061
:1064A00003C70701A5476313F70001A091654111D8
:1064B000930600100146938505E8254506C697C05A
:1064C000FF1FE780A02EB24017A5010013058569C4
:1064D00041011783010067008310C1676976814617
:1064E000FD1705061397060141836364B7003E85D7
:1064F00082803307D50003470700B98F214713F87F
:106500001700858363050800B18FC207C1837D171B
:106510001377F70F6DF78506F1B741C5A547054716
:1065200063F2B70883471500034705003168A207E7
:10653000D98F13978700A183D98FC207C18313080E
:10654000C855054763900707411106C622C426C2F5
:1065500003442500914763F087049307540063ECDC
:10656000F502A301C50021822302C5009304340073
:1065700091C6A302D500A1822303D5002A84A68553
:1065800097000000E780A0F526942300A400218155
:10659000A300A4000147B240224492443A8541013D
:1065A000828005473A858280B7C7A55A0111938733
:1065B000E7343EC42AC6B7F7070003C7070106CE73
:1065C00022CC26CAA5476313F70001A091642A8450
:1065D000938504EE930600100146254597C0FF1FE2
:1065E000E780C01C3000A146938504EE294597C082
:1065F000FF1FE780A01BA28517A5010013050567F3
:1066000097800100E780C0E597000000E78020C583
:10661000F2406244D2440561828001119165A14635
:106620003000938505EE2D4506CE97C0FF1FE7800D
:10663000E0172247B7C7A55A9387E7346318F702D4
:10664000B24517A501001305E55797D7FF1F2398FB
:10665000B7D4C205C18197800100E78060E0970050
:106660000000E780C0BFF24005618280D147D1457C
:1066700017A501001305055717D7FF1F2311F7D2E0
:1066800097800100E780C0DD17D5FF1F035525D196
:1066900097000000E78080F1F9B721C1411126C2BF
:1066A00006C622C4AE848DC52A8497200000E780E8
:1066B00000BC97E7FF1F83C7E7B299CB228522442E
:1066C000B240A68592444101173300006700C3D849
:1066D000B2402244924441018280828079714AD042
:1066E00006D622D426D24ECE93F715002E899DCB06
:1066F000AD67371700409387A7AA1CC3B7E704000C
:10670000BC4F13060019854517D5FF1F034505C962
:10671000829713451900B250225492540259F249FB
:106720004561828093F725006388071E2D4697A553
:10673000010093856559480097800100E780E0C615
:1067400097F6FF1F83C686FA139706014183954784
:1067500063F9E70C014417F5FF1F130525E913063C
:10676000300513085004930810041303B004130EEB
:1067700090059307640063F4F6043A84FD5997F496
:10678000FF1F83C4A4E697F7FF1F83C737E6A20461
:10679000DD8CAD679387B755638CF41463E3970A78
:1067A000A9679387A755638FF414A28517F5FF1F78
:1067B0001305C5E397000000E78060EE39A2B30738
:1067C000850083C50700639AC50483C517006396D7
:1067D000050583C527006392150583C53700639EB1
:1067E000C50283C54700639A650283C75700639655
:1067F000C703A2890DE897F5FF1F83C525EFB38571
:106800003541C20517F5FF1F130545DEC1814E95C1
:1068100097000000E780A0E8E9A005044204418059
:1068200089BF3A84FD598547E3EB87F445C8854520
:1068300017F5FF1F130585DB97000000E78020E6B2
:1068400071A8B1679387C7556380F404B5679387D0
:10685000D755E39CF4F4A28517F5FF1F130505D95E
:1068600097300000E78040BF89476300F406930536
:10687000E4FFC205C18117F5FF1F130545D7972017
:106880000000E780C09E91A00546A28517F5FF1F76
:106890001305C5D597F0FFFFE780E06697F7FF1F68
:1068A00083C787D49DE397E7FF1F83C7A79391CF43
:1068B000480097800100E78040DB93150501C18106
:1068C000480097300000E78020B9A68517A5010091
:1068D0001305853D97800100E78080B8FD57E39C54
:1068E000F9F097F7FF1F238307E01345290025B52B
:1068F000A28517F5FF1F130565CF97F0FFFFE7800F
:106900008071E1B7A28517F5FF1F130525CE97F01B
:10691000FFFFE780007255BF93F745000145E38C08
:1069200007DE17A501001305653997800100E78090
:1069300000CB97300000E78020C113454900E1BB40
:10694000411122C437E404005C5C06C6354697A5B5
:1069500001009385A5E717B501001305A5A182974E
:1069600011E917A501001305E53697800100E780BE
:1069700000C701A08327041C82972A84054597B08D
:106980000000E780407A97600100E78060FF976031
:106990000100E78060D497B00000E780C08B2285BB
:1069A000B2402244410182801567B71700401307A7
:1069B000575598C3D8439D66558FD8C3D843FD76A5
:1069C000758FD8C3D8431367F70FD8C3356713073C
:1069D000C7CC98C382804111054506C622C426C291
:1069E00097C0FFFFE780E0511305800497B0FF1FB9
:1069F000E780E06B757585457D1597C0FFFFE780E3
:106A0000803B7D7585451305F53697C0FFFFE78010
:106A1000E044371400408327840A8D451305002085
:106A200093E707202324F40A97C0FFFFE780A038EC
:106A3000B7E4040097C0FFFFE780007EC858978046
:106A40000100E780C0B917B501001305A592978032
:106A50000100E780C0B88327840C8545414593E752
:106A600007082324F40C97C0FFFFE780203F8D45E3
:106A70001305000897C0FFFFE780403E97C0FFFF67
:106A8000E780206B014597C0FFFFE780206E8545BA
:106A90000545894717F7FF1F230CF7C497C0FFFF71
:106AA000E780606E37070004B7E700E023A0E71037
:106AB00097D0FFFFE780000097D0FFFFE780C0136B
:106AC00097000000E78000E897000000E780008A58
:106AD00097000000E780A0B497E0FFFFE780A0EFF9
:106AE00097000000E780601097000000E780600BCF
:106AF00083A7040817050000130585BE829797D762
:106B0000FF1F238DA788BC4C130600648545829720
:106B100097000000E78080E997C0FF1FE780408D65
:106B200001458280B7F7070003C70701A547AE8676
:106B30006316F7009397450191C301A0AA8501460A
:106B4000254517C3FF1F670063C64111B2862E8615
:106B5000AA852D4506C697C0FF1FE78020C5B24015
:106B60000145410182809307000463E8C7021D715B
:106B7000A2CC2A84080886CE32C697800100E7801E
:106B8000C082B2461008A285294597C0FF1FE78042
:106B9000E0C1F6406644256182803955828041110A
:106BA0000D658D4506C697C0FFFFE780C020B7176B
:106BB00000408D6623A6D70A17F5FF1F130585B37E
:106BC0001387C70A9387870A1CC15CC585668967D6
:106BD0005CC958C114C518C9B7E70400B24003A383
:106BE000871E4101028397F7FF1F83C727B299EFE2
:106BF000411106C697100000E7808061B2408547CA
:106C000017F7FF1F2304F7B041018280828011C56E
:106C100089C517C3FFFF6700A3598280411126C2AF
:106C2000AE848D4522C406C62A8497C0FFFFE78044
:106C3000E022B717004099C803A5C70C418D23A6D1
:106C4000A70CB240224492444101828003A5870CE4
:106C5000418D23A4A70CF5B7834705000347150012
:106C6000A207D98FC2076177C18713072720639ACC
:106C7000E70083452500370504001703000067007F
:106C800023FA828017F6FF1F130686A88147B28673
:106C90001303F00FA9483308F6000348080013F760
:106CA000F70F6307A80C630668008507E39517FFD5
:106CB0002947B387E6002380A70097F7FF1F938734
:106CC000E7A55DA8411113D765001347170006C655
:106CD00093F63500058B954791CA0546994763871A
:106CE000C60009469D476383C600A14713F64500C9
:106CF0003336C00093F68503050685C2A145638B34
:106D0000B604E145638AB604930580026388B6043D
:106D1000930580036393B600914697F5FF1F238484
:106D2000F5C697F5FF1F238FC5C497F5FF1FA38BEB
:106D3000D5C4BE8517A50100130545039770010052
:106D4000E7800072B240854717F7FF1FA30DF7C217
:106D5000410182808546D1B78946C1B78D4675BF4E
:106D600017A5010013050503177301006700436FA2
:106D700017F7FF1F1307879ABA972380B700E147D9
:106D8000E302F5F493077002E30CF5FC82802A8796
:106D900023800500814717F5FF1F1305659713082A
:106DA000F00F2946B306F50083C606006396E60297
:106DB00097F6FF1F93868696B69783C7070005450B
:106DC0002380F5009947636EF7029D4763FDE70056
:106DD000E147630DF7008280638506018507E39331
:106DE000C7FC0145C5B7238005008280B737004046
:106DF00003C7370083C7050093F70704D98F2380A3
:106E0000F5008280797126D24AD097F4FF1F83C49F
:106E100064C917F9FF1F130929C806D622D44ECE1C
:106E200052CC56CA5AC8B307990083C7070093F7D4
:106E3000F70FA5C79387140093F7F70F0D4763610A
:106E4000F70C17F7FF1F230FF7C497F7FF1F938760
:106E500027C5A69783C707001307100293F7F70308
:106E6000638FE7286363F70A054463808720E3891B
:106E7000076E09476389E71413070002E38EE7589A
:106E8000B7E700E03707400023A0E7180100010042
:106E9000CA942380040023A0E710B787004003C7EB
:106EA0006700058BE30F077897F6FF1F83C6A6BF21
:106EB0000547E39AE67629472381E70209472383BA
:106EC000E7022385E70297F7FF1FA38F07AA97F72B
:106ED000FF1FA38A07BCB7870040A381070017F7ED
:106EE000FF1FA30507AA05472383E700B2502254DA
:106EF00092540259F249624AD24A424B4561828019
:106F000097F7FF1F238007BA89B7130730026386FC
:106F1000E70A63E6E71413074002638AE7081307EA
:106F20000003E39FE7F497F7FF1F938727B7A69720
:106F300003C70700A1471377F70FE31AF71C17EAF7
:106F4000FF1F130A6A7E83476A0097F6FF1F238399
:106F5000F6A297E7FF1F83C7977D91C7FD5797F666
:106F6000FF1F2389F6A097E5FF1F83C5F57B97F7E1
:106F7000FF1FA381B7A097E7FF1F83C7E77A93F9A5
:106F800007089306000493F707066393D752930705
:106F9000A009638DF51A63EAB7169307F005638AB3
:106FA000F54E930750096388F52E014479ABFD57E0
:106FB00017F7FF1F230FF79AE1B5FD5717F7FF1FCC
:106FC0002308F79A75BD17A50100130525EE9770E4
:106FD0000100E780C06097F7FF1F938727ACA69753
:106FE00003C40700814917FAFF1F130A6A8C137440
:106FF000F40F97AA0100938AEAEB63C78904294535
:1070000097700100E780A04A854717F7FF1FA30F7D
:10701000F78817F7FF1F230C878817F7FF1F230533
:10702000F79637E700E0B70640002320D7180100A5
:107030000100378600408347A60293F7370F2305E8
:10704000F6022320D7102DBDB3073A0183C50700F0
:107050005685850997700100E780804079BF854794
:1070600017F7FF1F2304F78421BD17A5010013059F
:10707000E5E397700100E780805697F7FF1F93873D
:10708000E7A1A69703C40700814917EAFF1F130A67
:10709000EA751374F40F97AA0100938AAAE163C5F5
:1070A0008904294597700100E7806040854717E70C
:1070B000FF1FA30BF77217E7FF1F2308877217F74D
:1070C000FF1F2303F78C37E700E0B70640002320BB
:1070D000D71801000100378600408347660293F706
:1070E000370F2303F602B1BFB3073A0183C5070088
:1070F0005685850997700100E78080364DB7854732
:1071000017E7FF1F2302F76EA5BB9307400A638DA5
:10711000F5349307200B6388F5369307100AE3963E
:10712000F5E883072A00014463D1074297E7FF1F70
:1071300083C7B75F93F63700638E061A0546638EE2
:10714000C62209466399C61A1D4775A217E5FF1F97
:107150000345A55DC94717EAFF1F034A1A5D97E576
:10716000FF1F83C5A55C17E4FF1F0344345C63194C
:10717000F510CD476316FA1093077008639CF5026B
:107180001307300FB7170E006308E4001307900DC4
:10719000B7B704006314E40817E7FF1F2322F77E44
:1071A000BE8517A50100130565D197700100E78022
:1071B000202BE5BB93078008639DF50033048040D6
:1071C000B77746001374F40F938787CDB3D7870240
:1071D000E1B793079008639AF50033048040916704
:1071E0001374F40F9387C766D5B79307A008639B02
:1071F000F50033048040B7173D001374F40F9387F4
:107200000790E9B79307B008639AF500330480400C
:1072100091671374F40F938797D04DBF93F5F507DB
:107220008D47639BF50033048040B7975B00137470
:10723000F40F938707D859BF8947639BF500330440
:107240008040B7770B001374F40F9387071BBDBF03
:107250008547639AF50033048040DD671374F40FAB
:10726000938767E3A5B789E9330480408D6713747A
:10727000F40F938777DC99BFF1679387072029BFC5
:1072800097000000E78040A0A2855285970000008B
:10729000E780809F19BB9305610017E5FF1F034539
:1072A000C54817E4FF1F0344544897000000E780D7
:1072B00040AE93057100228597000000E78060AD25
:1072C0003C0017E7FF1F2327F77C83476100230457
:1072D000F10083477100A304F100894717E7FF1FFE
:1072E000230AF7688357810017E7FF1F231EF74221
:1072F0000944A1AC154793F64700B336D00093F785
:107300008703850685C32146638BC7066146638A6A
:10731000C706130680026388C706130680036393BB
:10732000C700914717E6FF1F230ED66497E6FF1F9D
:10733000A38AF66497E7FF1F2387E76417E7FF1F19
:107340000347C73E9376070497E7FF1F83C7173E9F
:107350008DEE1377770C93067008630CD7021377C2
:10736000F7078D46631ED70AB307F040B7955B0059
:1073700093F7F70F938505D881A81947ADBF8547C7
:1073800055B7894745B78D4771BF9306700863119C
:10739000D7021307300FB7150E006389E7021307F2
:1073A000900DB7B504006383E7021307700845BF6B
:1073B0009306800C6311D702B307F040B7754600FF
:1073C00093F7F70F938585CDB3D5F50297E7FF1FA8
:1073D00023A8B75AF9B39306900C631AD700B307E2
:1073E000F040916593F7F70F9385C566F1BF93065B
:1073F000A00C631BD700B307F040B7153D0093F70F
:10740000F70F93850590C9B79306B00CE319D7F42D
:10741000B307F040916593F7F70F938595D06DB75B
:107420008946631BD700B307F040B7750B0093F78D
:10743000F70F9385051B49BF8546631AD700B3072D
:10744000F040DD6593F7F70F938565E3B5BF09EB72
:10745000B307F0408D6593F7F70F938575DCADB7F3
:10746000F165938505209DB783472A00C18B99C795
:10747000854717E7FF1F2302F75005BE97E7FF1F59
:10748000238D074E1DB6854717E7FF1FA30DF74E47
:1074900029BE3C0017E7FF1F232EF75E094793071D
:1074A00000032314F10097E6FF1F2385E64C2DBD52
:1074B000639A0758A94763ECB74417A7010013075D
:1074C00027888A05BA959C41BA97828717E4FF1FDF
:1074D0000344B425094A630C440F636C8A0885474A
:1074E0006309F40A9307F00F17E7FF1F0347874864
:1074F00063F6E70017E7FF1F230EF74617EAFF1FA3
:10750000034A4A47930700041374FA0F63F44701D0
:107510001304000497E7FF1F9387C75783AA070048
:10752000228617E5FF1F13052520D685330A8A40DA
:10753000A29A97700100E78040E797E7FF1F238B2F
:10754000474397E7FF1F23A7575597E7FF1F83C7B9
:1075500077421547639AE762B7E700E037074000D4
:1075600023A0E71801000100B786004023808602AF
:107570008DA58D47630CF40A9947E315F4F697A798
:1075800001009387678217E7FF1F2325F750A9475C
:10759000A1BF17E7FF1F0347075197E7FF1F938717
:1075A000673F494697A501009385058963068700D3
:1075B00097A50100938545843E8597700100E7807B
:1075C000C0DE17E7FF1F2327A74CC94731BF97E647
:1075D000FF1F83C6464D054797E7FF1F9387873BED
:1075E0006394E6023E851306700297A50100938519
:1075F000258297700100E78040DB17E7FF1F232BF0
:10760000A74893077002CDB53E85130630049795C1
:1076100001009385257A97700100E78000D917E76C
:10762000FF1F2329A746930730047DBD97E5FF1F61
:1076300083C5A50F17A50100130585899770010063
:10764000E78000E2854A17EBFF1F034BCB4597E528
:10765000FF1F83C5850D17A50100130565876318F6
:107660005B0B97700100E780A0DF97E7FF1F83C7E0
:10767000C70BB5CBE368F4E617A40100130404803C
:10768000638C6701179401001304C47F638647016C
:1076900017A4010013048480228597700100E780FD
:1076A000C0FC1375F50F93071500860717E7FF1F3A
:1076B0002302F72E8D4717E7FF1FA30DF72C97E73F
:1076C000FF1F9387272D0147BE861376F70F890783
:1076D0006365A60297E7FF1F23AED73A97E7FF1F20
:1076E00083C7472B11B5979701009387277217E738
:1076F000FF1F2321F73A9147C5BB3306E400034639
:107700000600A380070005072380C7007DBF977090
:107710000100E780E0D497E7FF1F83C70701E1D7A7
:10772000E362F4DC1794010013044472638C570184
:107730001794010013040472638647011794010033
:107740001304C472228597700100E78000F213755C
:10775000F50F93071500860717E7FF1F230CF72285
:107760008D4717E7FF1FA307F72297E7FF1F9387B0
:1077700067220147BE861376F70F8907E37CA6F4DC
:107780003306E40003460600A380070005072380B4
:10779000C700D5B797E5FF1F83C525F917950100E9
:1077A0001305C57397700100E78080CB97E7FF1F33
:1077B00083C7171E93E7470017E7FF1FA30AF71CAD
:1077C00083472A0017E7FF1FA302F71C6FF0EFFDA6
:1077D000179501001305C57197700100E78020E03F
:1077E00097E7FF1F9387871A83C7070017E7FF1FD5
:1077F000230CF7F217E4FF1F0344C417333480004F
:10780000A9B3179501001305E56F97700100E78094
:1078100000DD97E7FF1F83C7B71793E7070117E757
:10782000FF1FA307F71683472A0017E7FF1F230F41
:10783000F7146FF08FF7179501001305E56D97703A
:107840000100E780C0D903470A007D8B51EFB7875D
:10785000004003C767021377C70B13672700238312
:10786000E70203C7A7021377C70B13672700238517
:10787000E70203C7E7021377C70B136727002387C5
:10788000E70203C727031377C70B13672700238972
:10789000E702854717E7FF1F2308F7F417E7FF1FE5
:1078A0002306F70017E7FF1F2304F70C17E7FF1F56
:1078B0002301F70C97E7FF1FA38807F297E7FF1F45
:1078C000A38607FE97E7FF1FA384070A97E7FF1F1A
:1078D000A381070A97E7FF1FA388070A97E7FF1FFF
:1078E000A383071C6FF06FEC89476312F70297E7D9
:1078F000FF1F83C7A7E39146638CD70863E0F604B4
:10790000638EE70C6369F70A05476380E70EFD574E
:1079100017E7FF1FA300F70637074000B7E700E0AF
:1079200023A0E71801000100B78600401306F0FC11
:107930002381C60223A0E7106FF08FD4130720081D
:107940006382E7086362F70213071008E391E7FC1C
:10795000378700408347670293F7C70B93E72700F9
:107960002303F7026FF06FE4130730086389E7021F
:1079700013074008E39DE7F8378700408347270354
:1079800093F7C70B93E727002309F7026FF0EFE1A6
:10799000378700408347270393F73707F5B73787C3
:1079A00000408347E70293F7C70B93E727002307BD
:1079B000F7026FF08FDF378700408347E70293F7C6
:1079C0003707F5B7378700408347A70293F7C70B00
:1079D00093E727002305F7026FF02FDD378700407C
:1079E0008347A70293F73707F5B7378700408347E8
:1079F000670293F73707ADB7179501001305C55216
:107A000097700100E780A0BD97E7FF1F238E07D086
:107A1000D5B3179501001305255297700100E78033
:107A200000BC97E7FF1F239107D097E7FF1F9387BD
:107A300067F403C40700894763F38700094413749C
:107A4000F40F21B613070002E393E7EC6399090AE8
:107A5000638FF500930720026381F50817950100F5
:107A60001305055197700100E780809F4DB517956C
:107A700001001305254D97700100E78040B60144D1
:107A8000179B0100130B4B4DA14AB3078A0083C516
:107A900007005A85050497700100E780609CE31693
:107AA00054FF179501001305E5AF97700100E780BB
:107AB00000B317E4FF1F034464C711E497E7FF1FF7
:107AC000238707C459B48947E313F4E4854717E7CC
:107AD000FF1F230EF7C26FF04FCD17E6FF1F0346BF
:107AE000D6C497E5FF1F83C545C41795010013054C
:107AF000254797700100E780A0966FF00FCB638F4A
:107B0000F50493071002E39BF5F497E5FF1F83C587
:107B1000E5C1179501001305A54697700100E780A0
:107B2000209497E7FF1F23A747F797E7FF1F938747
:107B300027E5944383D7470017E7FF1F0347A7E4D0
:107B400017E6FF1F2322D6BE1D4497E6FF1F239F83
:107B5000F6BC97E7FF1F238CE7BCC5BA97E5FF1F6C
:107B600083C5C5BC17950100130505439770010037
:107B7000E780008F97E7FF1F238B07B897E7FF1F6A
:107B8000239407BA6FF0CFF62547E387E79C1947A0
:107B90006391E702B786004023808602B7E700E0E2
:107BA0003707400023A0E71801000100130600FC7E
:107BB00041B31307100A6391E702B78600402380A0
:107BC0008602B7E700E03707400023A0E71801006E
:107BD0000100130680FCA9BB1307A009E38FE7FC93
:107BE0001307400AE38BE7FC13072002E386E796BE
:107BF0000547E383E796B7E700E03707400023A097
:107C0000E718E391099601000100B7860040238040
:107C10008602130620FC29BB17E7FF1F034797D5F1
:107C20006308F71E63E7E7029547630EF70E99476F
:107C30006308F704B786004023800602B7E700E038
:107C40003707400023A0E718010001001306A0FC3D
:107C5000C5B19307F005630AF7009307500963065F
:107C6000F70093071002E317F7FCB7E700E03707C8
:107C7000400023A0E71801000100B786004051BF73
:107C800097E9FF1F83C909CF93070004CE8A63F4E5
:107C90003701930A000497E7FF1F9387A7DF03AA22
:107CA000070013F4FA0F2286D28517E5FF1F13058C
:107CB000A5A797600100E780406FB3878940529481
:107CC00017E7FF1F2308F7CA97E7FF1F23A487DCE6
:107CD000638E0902B787004023805703B7E600E0B0
:107CE0003706400023A0C6180100010003C7270281
:107CF000134707042381E70203C727021377C70F3F
:107D00002381E70223A0C6106FF08F97B78600404B
:107D100023800602B7E700E03707400023A0E718FA
:107D200001000100FDB5378700408347370097E623
:107D3000FF1F83C6B6C593F70708D58FA301F700C9
:107D4000B7064000B7E700E023A0D7180100010004
:107D50001306A0FC2301C70223A0D7106FF04F9297
:107D600097E7FF1F938787D3A69783C7070093F7EB
:107D7000F70FD9CF97E7FF1F83C7E7D2D1EB17E7FC
:107D8000FF1F034737BF930700026313F70897E706
:107D9000FF1F9387679903AB070097EAFF1F83CA0A
:107DA000EA9817EAFF1F034A7A9897E9FF1F83C9E9
:107DB0000998D2875687CE865A8697E5FF1F83C5D6
:107DC0000595179501001305A51E97600100E78032
:107DD000206997E7FF1F23A567BB97E7FF1F238352
:107DE00057BB97E7FF1FA38F47B997E7FF1F238C68
:107DF00037B997E7FF1FA38B8790B7E700E03707F6
:107E0000400023A0E71801000100B7860040D1B36D
:107E1000B7E700E03707400023A0E71801000100A2
:107E2000B786004025B529472381E7020947238308
:107E3000E7022385E7022387E7022389E7026FF041
:107E40008F8803C76700118B6302078A83C75700B7
:107E5000918BB5CF17E7FF1F0347E7C4854763132F
:107E6000F70697E7FF1FA380E7B297E7FF1F238D71
:107E7000079697E7FF1F238B07A297E7FF1F23892A
:107E800007AE97E7FF1F238607AE97E7FF1FA38D77
:107E9000079497E7FF1FA38B07A097E7FF1FA3890E
:107EA00007AC97E7FF1FA38607AC97E7FF1FA38DDB
:107EB00007AC97E7FF1FA38807BEB78700401147AD
:107EC0006FF08F8217E7FF1FA302F78479BF854702
:107ED00017E7FF1F230AF79017E7FF1F2308F79CF8
:107EE00017E7FF1F2306F7A817E7FF1F2303F7A8CD
:107EF00069BF854717E7FF1F2308F78E17E7FF1FA6
:107F00002306F79A17E7FF1F2304F7A617E7FF1FBB
:107F10002301F7A617E7FF1FA308078C17E7FF1F2A
:107F2000A306079817E7FF1FA30407A497E7FF1FFF
:107F3000A38107A48280411106C697000000E78054
:107F400080FBB787004023800700130740FC23868F
:107F5000E7001307C004A386E70017D7FF1F130726
:107F6000A77C2398E70017D7FF1F1307E77F239A03
:107F7000E70017E7FF1F1307678B239CE70017E74E
:107F8000FF1F1307E796239EE70029472381E70297
:107F900009472383E7022385E7022387E702238932
:107FA000E702A3810700930600F8A380D700930699
:107FB00090022380D700FD562383D7002381E7005A
:107FC000B706400037E700E02320D71003C71700AB
:107FD00013671700A380E700B24097E7FF1F2397BE
:107FE000079A41018280411106C697000000E78090
:107FF00080F0B787004023800700130700FC23862A
:10800000E7003147A386E70017D7FF1F1307C771A3
:108010002398E70017D7FF1F13070775239AE70078
:1080200017E7FF1F13078780239CE7002947238159
:10803000E70209472383E7022385E702A3810700BC
:10804000930600F8A380D700930690022380D70000
:10805000FD562383D7002381E700B706400037E7AA
:1080600000E02320D71003C7170013671700A38071
:10807000E700B24097E7FF1F239A079041018280F3
:10808000B78703009387074017E7FF1F232AF78E60
:10809000854717E7FF1F2317F78EA14717E7FF1F35
:1080A0002303F78E97E7FF1FA38F078C97E7FF1F28
:1080B000238C078C97D7FF1F238B076497D7FF1F4D
:1080C000A3860764814717D5FF1F13056564FD5517
:1080D00017D6FF1F130686642947B306F5002380D1
:1080E000B600B306F600238006008507E397E7FE97
:1080F00097E7FF1F2382079A97E7FF1FA38E079832
:1081000097E7FF1F238B079897E7FF1FA385078635
:1081100097E7FF1FA383078697E7FF1F238E078438
:1081200097E7FF1F2389078497E7FF1F23880784AA
:1081300097E7FF1FA382078497E7FF1F238F07821C
:1081400097E7FF1FA38B0794828017E7FF1F034762
:10815000879585476316F700170300006700E3E87B
:1081600017030000670063DD411122C406C617E74C
:10817000FF1F0347479385472E8613F4F50FAA8503
:108180006317F70417D5FF1F1305456E97600100AD
:10819000E780A02197D7FF1F238A0770B787004089
:1081A00023848702B7E600E03706400023A0C61804
:1081B0000100010003C7A7021377C70F2385E70259
:1081C000B240224423A0C61001454101828017D548
:1081D000FF1F1305655D97600100E780001D97D7BD
:1081E000FF1F23830760B787004023828702B7E61B
:1081F00000E03706400023A0C6180100010003C7B5
:1082000067021377C70F2383E7025DBF411106C6DC
:1082100097000000E78000E7B2404101170300002B
:108220006700E3F2411106C697F0FFFFE780C0BD8B
:1082300097D7FF1F83C7575B95C797D5FF1F83C588
:10824000C55A89C917D5FF1F1305455A97F0FFFF77
:10825000E780209C97D7FF1FA388075897D7FF1F59
:1082600023840772B2404101828041C9D9C597D7A2
:10827000FF1F83C7A771D1C3011122CC4AC84EC6C4
:1082800056C25AC006CE26CA52C42E89AA890144B3
:10829000930A0004371B030063772403B307894064
:1082A000C207C183BE8463F4FA0093040004C204CD
:1082B000C180130A1BD497D7FF1F83C7E7529DE3E2
:1082C0007D1A631C0A00F2406244D2444249B2491A
:1082D000224A924A024B0561828097F0FFFFE780B5
:1082E000A0B2D1BF338589002694A68542049700A9
:1082F0000000E780A0E7418045B7828097D7FF1F45
:108300009387077E18429C4383D6450003450700A8
:1083100083C5C700035646006396A50083D5E700D2
:10832000638DD502011106CE2386A7002397D700BF
:10833000B705CF00DC4B9385757D05077D162EC2F2
:10834000230001003AC42316C1002317D10099C3AA
:108350000A858297F240056182808280DC4DDC4B89
:1083600081CFB7E70400904503A38705914517D552
:10837000FF1F03452577028382806D713C083EC64E
:10838000B707E500232291103EC8AA843C08328535
:10839000232611103ECA23248110232021112E8967
:1083A00097300000E78020562A8497950100938536
:1083B000A5C317850100130525B897600100E78064
:1083C000200AA28517950100130585D29760010048
:1083D000E7800009294597600100E780400DB70557
:1083E000CB009385757D680097100000E780405FA3
:1083F000A285680097300000E7804043014781462E
:108400007000CA85268597200000E780C08205CDD0
:108410002A8497950100938525BD178501001305D2
:10842000A5B197600100E780A003A2851795010020
:108430001305C5CC97600100E7808002294597604D
:108440000100E780C0068320C1100324811083242B
:108450004110032901105161828097D7FF1F938734
:10846000276818429C43797122D406D60348070036
:1084700083C807012A8483D64500035546006396C6
:10848000080183D82701638DD802238807010507D7
:108490002399D7003708CC00DC4B1308787D3ACC01
:1084A0001307F5FF42CA23080100231EE100231F22
:1084B000D10099C7080832C62EC482973246A24519
:1084C000228597000000E78080EBB250225445617E
:1084D00082806D713C083EC0B707E5003EC23C0893
:1084E0003EC4232611102324811023229110231728
:1084F00001002318010023190100231A0100231B86
:10850000010097B7FF1F83D7E7EB99E3C167FD171A
:108510002316F10097B7FF1F83D7E7EA91EB97D7B0
:10852000FF1F9387E75B9C439C43DC4783D707008F
:1085300017B4FF1F130404E9584C2317F1008357A5
:108540004400484B2318F10031E1979501009385D1
:10855000A5B0178501001305259E97600100E780EF
:1085600020F017950100130565B097600100E780C2
:1085700020EF294597600100E78060F38320C11058
:1085800003248110832441105161828097B7FF1F1B
:1085900083C7B7E389EBB7E70400BC5782975C4C0D
:1085A00023AA0700E1BFFD1797B6FF1FA38FF6E0D0
:1085B00003560701834704014C470A85230BF1004A
:1085C00097300000E780A02397D7FF1F938747517C
:1085D0009C430147814688430A866C00971000003F
:1085E000E7806065AA8429C1979501009385C5A697
:1085F000178501001305459497600100E78040E668
:10860000A68517950100130525A797600100E7804F
:1086100020E5294597600100E78060E9584CB7E7FD
:108620000400BC57484B9DBF97B7FF1F83C7F7D9BE
:10863000F5D7B7E70400BC4F1044854517D5FF1F99
:108640000345454A82971DBF5C4EDC4BB9CFB1CD87
:10865000411122C4178501001305058E2E849795BC
:1086600001009385A59D06C697600100E78040DF65
:10867000A285179501001305E5A297600100E78028
:1086800020DE294597600100E78060E2B7E704003B
:108690002244B24003A3870517D5FF1F0345854435
:1086A000130640069145410102838280411122C494
:1086B00017B4FF1F1304C4CE1C4C06C689C7DC4385
:1086C00099C34C488297584CB7E70400BC57484BB5
:1086D00082975C4CB240224423AA07004101828069
:1086E00017B7FF1F1307C7CD834707009306F00B8B
:1086F000850793F7F70F63E9F60097B6FF1F23810D
:10870000F6CC034507008280930700F8FDB7835736
:1087100045006386071001114AC817B9FF1F1309E6
:1087200069CA52C4032AC90106CE22CC03274A01D2
:1087300026CA4EC656C2F15735E31307D00DFD5772
:10874000636EC704B7E9040083A709072A841305E9
:10875000860042054181B284AE8A8297232AAA000C
:108760000325C9015C49A9E7979501009385058B0D
:10877000177501001305457C97600100E78040CE26
:10878000179501001305459A97600100E78040CDD9
:10879000294597600100E78080D1DD57F2406244AF
:1087A000D2444249B249224A924A3E8505618280BA
:1087B00093874400B705CF002319F5009385757D95
:1087C000310597100000E780A0210325C9018345EA
:1087D0006400310597300000E78040050325C9019A
:1087E0002686D685310597300000E7804001714626
:1087F000A2854A8597600100E78020BB504419CAD2
:1088000083A78905854517D5FF1F0345A52D8297A9
:10881000814769B797000000E780E0CBD5BFFD57DF
:108820003E858280411126C297B4FF1F938484B98C
:10883000D84C22C437E404003C54484B06C6829707
:10884000DC4C0323C4052244B240924423AA07000F
:1088500017D5FF1F034505298545410102834111B5
:1088600026C297D4FF1F9384A4279C4006C622C427
:108870004AC0D5C3DC43C5C35CC12300B5002A840C
:10888000978501009385C574177501001305C56AA6
:1088900097600100E780C0BC294597600100E78030
:1088A00000C19C4023A4070023A2070097B7FF1F25
:1088B000938707AFDC4FDC4B91C729559700000029
:1088C000E78000DF97B7FF1F9387C7AFDC4FDC4B14
:1088D00089C797000000E78020F537E90400832767
:1088E000C905894517D5FF1F0345C51F82978327F3
:1088F000C905914517D5FF1F0345C51E82979C40AA
:1089000003A347016309030022852244B240924435
:10891000024941010283B24022449244024941018A
:1089200082800111328506CE22CC26CA2E84973051
:108930000000E78040FDAA84978501009385856C3F
:10894000177501001305455F97600100E78040B18E
:10895000030784000356640083554400A6861785E8
:1089600001001305257697600100E78060AF294577
:1089700097600100E780A0B397B7FF1F83C7A7A246
:10898000639D9700014597000000E78060D2814514
:108990000A8597000000E780C0ECF2406244D244B0
:1089A000056182806D7123248110232611102322FA
:1089B000911093F745002E84638707143C083EC04E
:1089C000B707E5003EC23C083EC423170100231848
:1089D000010023190100231A0100231B010097B78E
:1089E000FF1F83D7E79B99E3C167FD172316F100AB
:1089F00097B7FF1F83D7E79A91EB97D7FF1F93870E
:108A0000270E9C439C43DC4783D7070017B7FF1F03
:108A1000130707992317F100544F83574700231872
:108A2000F100DC4AA1E7978501009385E5611775A0
:108A300001001305655097600100E78060A217856B
:108A400001001305A56297600100E78060A1294538
:108A500097600100E780A0A5134544008320C11062
:108A600003248110832441105161828097B7FF1F36
:108A700083C777932555D9C3FD1717B6FF1FA304E6
:108A8000F69203D6060183470701CC460A85230BDD
:108A9000F10097300000E78080D697D7FF1F9387BB
:108AA00027049C4317B7FF1F1307878F9786010082
:108AB0009386C65E88430A866C0097100000E780A4
:108AC0008017AA8451D9978501009385E5571775BA
:108AD00001001305654697600100E7806098A68550
:108AE000178501001305455997600100E7804097FD
:108AF000294597600100E780809B2685970000004C
:108B0000E78000BB91BF93F725009DC7B7E704003E
:108B1000BC474146814528088297255597000000AB
:108B2000E78000B928089305F00F97000000E78060
:108B300040D3134524001DB793F71500014599DF75
:108B400097000000E78020991345140001BF5C4D99
:108B5000411106C688C317D7FF1F2323F7F8B7E7CD
:108B6000040083A70708170500001305E5E38297B3
:108B7000B24097D7FF1F2387A7F6014541018280A6
:108B800001113335A000A307A100B7E7040083A7B4
:108B9000471706CE1306F10085451305503082971E
:108BA000F240056182808280411122C406C697D7B7
:108BB000FF1F83C7A7F4014489EF97B7FF1F83C73F
:108BC0007762054499E717D4FF1F0344E4A11344D7
:108BD0001400228597000000E780C0FA1785010085
:108BE0001305456009E4178501001305A5602244BB
:108BF000B24041011763010067008386797122D476
:108C0000A30F010037E404008327841726D24AD03B
:108C100006D6AA842E89130550309305F10132C679
:108C2000829732468347F10193150601C18185CBB6
:108C300001452EC697000000E780C0F48327441743
:108C4000B2454A8626858297054597000000E78051
:108C500060F3B250225492540259456182808327B6
:108C600044174A8626858297EDB7411193970501EF
:108C700022C406C626C2C1872E8463D40702B7E485
:108C80000400FC5417A5FF1F0345C576829719C140
:108C9000BC5482972165218DB24022449244410107
:108CA000828093F715008DC7B7E7040083A7471AA2
:108CB00017A6FF1F1306067397D5FF1F938545E37D
:108CC00017A5FF1F03450573829713451400E9B7E5
:108CD00093F7250099CFB7E70400BC4F1306006453
:108CE000894517A5FF1F0345E570829713452400AA
:108CF00065B793F785009DC7B7E7040003A8871AF7
:108D00001307401F97A7FF1F83C7C76E814613062F
:108D10004006994517D5FF1F035585DE0298134578
:108D200084009DBF93F745000145BDD7B7E404001B
:108D300083A7041817D5FF1F035585DC8297BC4C09
:108D400013060064914517A5FF1F0345A56A829786
:108D50001345440091B797D7FF1F83D767DA63980D
:108D6000A70217D7FF1F231EB7D817D7FF1F231B34
:108D7000C7D817D7FF1F2318D7D82E86178501000D
:108D80001305854CBE85175301006700636D178579
:108D900001001305E54C1763010067004384035786
:108DA000450097D7FF1F83D7A7D5631AF704C1677C
:108DB0004111F91722C417D7FF1F2323F7D437E433
:108DC000040097D7FF1F23AF07D297D7FF1FA387B2
:108DD00007D27C4C06C6894517A5FF1F0345856150
:108DE00082977C4C914517A5FF1F0345A56082978C
:108DF0002244B240410117030000670023DB1785BE
:108E000001001305E545175301006700437D7D15FB
:108E1000954763E2A71C178701001307673A0A0505
:108E20003A951C41011122CC06CEBA972E84828736
:108E3000178501001305454397500100E780207A0C
:108E4000A1A203C7250099476311F7022E85970059
:108E50000000E78000F583456400178501001305D5
:108E6000A54197500100E780A05F97B7FF1F238BB4
:108E70000736178501001305E5417DBF03C72500AF
:108E800095476319F702C16717D7FF1F035747C7F5
:108E9000F91703D5A5006309F702B7E7040083A714
:108EA000C7178297178501001305C53F975001002A
:108EB000E780E072854717B7FF1F2305F732178554
:108EC00001001305A5408DBF97D7FF1F239AA7C2A6
:108ED00083D7E50097D6FF1F2395F6C283D70501F8
:108EE00097D6FF1F2390F6C283D7250197D6FF1F81
:108EF000239BF6C097D7FF1FA38207C0631BE50221
:108F0000B7E70400BC4F096613060690A14517A5F4
:108F1000FF1F0345254E82970356E4008355A400A6
:108F2000178501001305453997500100E78040532C
:108F300051B79307700F2316F100B7E7040083A71A
:108F4000870D17A6FF1F0346E64A6C0082974DF96E
:108F5000854717D7FF1FA303F7BA5DB71785010031
:108F600013058537D1BD83C5250091476392F5026E
:108F7000178501001305C53797500100E78020666B
:108F800097000000E78080C2F24062440561828061
:108F900099476392F502228597000000E78060E020
:108FA00083456400178501001305052D97500100C6
:108FB000E780004BD1BF9547639AF50083471400C3
:108FC000E1F3178501001305E534BDB517850100F0
:108FD0001305C534E1BF82806D71232481102326DF
:108FE000111023229110328401CD8947630AF502C2
:108FF0008320C11003248110832441105161828099
:109000001785010013054532AE8497500100E780B3
:10901000005DA285268597C0FFFFE7808054C9BF09
:10902000B7E70400FC472800829717850100130565
:10903000653097500100E780805A8347810039C42A
:109040001307000B6380E7021387A7051377F70F59
:109050008D4663EDE602A285280097D0FFFFE780EA
:1090600060C379B78547E3F587F8834591001775A5
:1090700001001305A521B335B00097B7FF1F238565
:10908000B7FE97500100E780A03D9DB703479100D0
:10909000A207D98F35671307D7556385E70863683B
:1090A000F7022D671307B7556387E7063167130784
:1090B000C755638AE70429671307A7556394E70236
:1090C000A285280097D0FFFFE780A0F615B7396783
:1090D0009306E765638DD70663E9F6001307E75546
:1090E0006380E706A28528003DB73D679306F755E4
:1090F0006386D7061307F766E396E7FE97D0FFFF70
:10910000E780200FF5B50146A285280097D0FFFF24
:10911000E78060DFF1BDA285280097D0FFFFE780E0
:1091200080EFF9B58947E3F587EC9305E4FFC205C5
:10913000C1811305A10097A0FFFFE78060074DBD27
:10914000A285280097D0FFFFE780A0EF55B5A28544
:10915000280097D0FFFFE78060FA59BD97D0FFFF46
:10916000E780E00271B5411122C417A4FF1F130468
:10917000A429AA8617860100130606062285C14582
:1091800006C697500100E780C0460357440097A7E2
:10919000FF1F938767282393E700035764002394F6
:1091A000E700B240224441018280411106C6970087
:1091B0000000E78080FBB7E7040083A7871417A6A9
:1091C000FF1F13066624D54501458297B2404D46E0
:1091D00097A5FF1F938545241305703041011703A0
:1091E00000006700E3A161712324811A37E40400C1
:1091F000832704082326111A2322911A2320211BD6
:10920000232E311917050000130565A6829717A9AB
:10921000FF1F1309291E994785442300A900231C19
:10922000F10097850100938525FF93074006177588
:109230000100130565D0231CF1082308910097C98C
:10924000FF1F9389C94A97500100E780602183D5A9
:10925000090017850100130525FB97500100E780E1
:109260002020294597500100E780602403D509009C
:10927000856997000000E78040EF832744171008B6
:1092800085451305503082978327441717A6FF1F83
:1092900013068618CD45130570308297832744172F
:1092A00017A6FF1F13064615B545130560308297B4
:1092B0008327441730088945130510318297832787
:1092C00044173009894513052031829783274415B7
:1092D000938509C80D45829783274415938509C84E
:1092E00011458297A3059100230691002308910060
:1092F00002CD230C01008327841630099145130504
:1093000070408297832784161306B10085451305A4
:10931000004082978327841670008545130510400E
:10932000829783278416300885451305204082974D
:10933000832784161008854513055040829783279C
:1093400004157D558297832744137D5582977D555B
:1093500097A0FFFFE78080308327440C829797A077
:10936000FFFFE780C00B8327841417A6FF1F130697
:10937000A609D5450145829789471306700F814597
:1093800028092306F1009790FFFFE78000D58D475D
:109390001306000881452808230CF1089790FFFF69
:1093A000E780A0D39147230CF100977701009387C2
:1093B00027AA984383C747003AC8230AF10097D0E9
:1093C000FFFFE780C0E970008545054597A0FFFFD6
:1093D000E780E02F30099305700F094597A0FFFF44
:1093E000E780E02E3008930500080D4597A0FFFFA9
:1093F000E780E02D10089545114597A0FFFFE78015
:10940000002DC16717C7FF1F1307876FF9171CC30C
:109410002322070017A5FF1F130585FD97A0FFFF57
:10942000E780C0298327C41D17C5FF1F1305C56B1F
:1094300082973C4803450900854582978320C11ADD
:109440000324811A8324411A0329011A8329C1198B
:109450005D618280C16717C8FF1F0358686AF917EA
:109460006301F8083DCDB5CD011126CAB7E404006B
:1094700083A7841222CC2E862315B10006CE2A841F
:1094800001478146ED45428582972AC611ED178531
:109490000100130565D997500100E7804014F240A0
:1094A0006244D24405618280FC440356A100A28537
:1094B00082972C0017C5FF1F0355856497A0FFFFF7
:1094C000E780802C69DD17850100130525D79750AB
:1094D0000100E780C01083A7C412ED4528008297E1
:1094E0007DBF8280411106C61DC9854717A7FF1F92
:1094F000A309F7F0354697A5FF1F9385E5EF130500
:10950000603097A7FF1F238F07EE97F0FFFFE780DC
:10951000206FB240410117F3FFFF6700236997A74F
:10952000FF1FA38007EEF9B7C16717C5FF1F0355DB
:10953000255DF9176307F500B7E7040003A3C71714
:1095400002838280854717C7FF1F2309F75A014509
:1095500017F3FFFF670003631793FFFFE70243B3AF
:109560002A8408452E89B28919C900C197150000BF
:109570009385A586610597300100E78080018144CD
:109580007D5A97100000E780E03963C7A404814446
:1095900097100000E780003A63C8A40497C7FF1F34
:1095A000938787569C43DC47B307F9409187230292
:1095B000F400638309048327C900B307F440958747
:1095C000A302F4001C4C89C79C4799C3228582974B
:1095D0001793FFFF670003AF5C44139714008504E3
:1095E000BA972390470171BF1C4813971400850454
:1095F000BA972390070069BF832789000547B307FF
:10960000F4409587A302F40083570400638EE702B9
:109610008DC309476384E7040D47E395E7FA97870D
:1096200001009387E7231CCC978701009387472489
:1096300011A897870100938727EA1CCC9787010020
:10964000938787EA5CC8BDBF978701009387C7D51A
:109650001CCC97870100938727D6EDB79787010029
:109660009387C7241CCC9787010093872725D9BFF0
:1096700095E51793FFFFE70243A30046184483478D
:10968000940075839D8B6317F70097100000E780A7
:1096900060B448C41793FFFF670063A382801793E9
:1096A000FFFFE702E39E13893500C16442094111BF
:1096B000AA890144F11413590901054A2EC69710CD
:1096C0000000E7802026B2456348A400014541011F
:1096D0001793FFFF6700039F83A709001317140068
:1096E000BA9783D707006388B700639497006374C1
:1096F0002A010504E1B70545D9BF1793FFFFE7022B
:109700004398AA892E89328BB6843A8ABE8A97A05A
:109710000000E78020FB71C9268597200000E780C4
:1097200020098D4763E7A7007D551793FFFF67006A
:10973000C39883DB440097100000E780A0242A84AC
:1097400097100000E78040259307740031443305EB
:10975000850263CDA70297100000E780A022971032
:109760000000E78020222A8497100000E780C022B2
:109770009307740031443305850263C3A70497102F
:109780000000E78020209307450029A897100000DB
:10979000E7808020330585021307F0179307C01771
:1097A000E35FA7FA2D55E3C277F963040B02D6866F
:1097B0005286A6854A8597200100E78020BAB5B772
:1097C00097100000E780401D330585029307C5FF11
:1097D000D1BF832749001385C90083D5270097008F
:1097E0000000E78000EC61F581B769553DBF97C780
:1097F000FF1F239DA73097C7FF1F9387E730904334
:1098000081470C463307F500420741836393B70055
:1098100082805446139847008507C2962390E6003D
:10982000D5B797C7FF1F9387272E9C4303C5870093
:10983000828017C5FF1F0355652D82801793FFFF98
:10984000E702A386C1671387D7FF630BE502636A4C
:10985000A700F1176300F50201451793FFFF6700AA
:1098600003871387E7FF6302E502FD171D8D13359C
:109870001500E5B797500000E780C0267D15C5BFED
:1098800097500000E78040FBD5BF97500000E7806D
:1098900060F9EDB71793FFFFE70223814111AA8416
:1098A00001442EC697100000E780C008B245634807
:1098B000A400014541011793FFFF670043819C48C5
:1098C000131514003E9583570500E385B7FE050484
:1098D000C9BF03485500814693F7F60F63E50701BA
:1098E00081473E858280584593975600BA9703D7A3
:1098F00027006316B70003D70700E304C7FE8506F9
:10990000E1BF8346450001479377F70F63E4D70033
:10991000814711A81C45131657000507B29703D6B7
:109920000700E313B6FE3E8582801783FFFFE70240
:10993000237693170501C18797CAFF1F938ACA1C14
:10994000635BF00883A70A00C0479C4703570400E5
:10995000198D420541816368F50001442285178312
:10996000FFFF6700237612052A94CDBFDC471394CE
:109970004900014A3E94834744006341FA02014A88
:10998000834754006349FA028509C20993D9090142
:1099900083A70A009847E3EBE9FCC1B71C441319FD
:1099A0005A00A6853E994A8597000000E780C0EEE0
:1099B00005E1050AC9B75C4413195A00A6853E990A
:1099C0004A8597000000E78020ED19E1050A4DBFA8
:1099D000E30C09FA61B7AA8481495DBF1783FFFFD1
:1099E000E702A36C1C452A8481E79307C5001CC5C8
:1099F0001C44231204001CC09307F00F63EDB70052
:109A000093F5F50F228597200000E78020E2178369
:109A1000FFFF6700C36B93940501C167C18063F9C1
:109A2000F500A685228597200000E78040E5C5B7B0
:109A3000C18193F5F50F228597200000E78000DFB4
:109A4000A685228597200000E78040E0C9B797C728
:109A5000FF1F9387670B884382801C4599C797C770
:109A6000FF1F23A3A70A014582807D55828097C7E7
:109A7000FF1F93876709984383474500484792072C
:109A80003E9582801783FFFFE702236261710045E4
:109A90001C183EC6B70780013EC81C183ECA835733
:109AA000440002CE02D002CC231EF1008347840082
:109AB0002A8902D22301F1023C083ED402D6970043
:109AC0000000E78000FB835705002316F102975042
:109AD0000000E78060C42307A1025C4003556400D6
:109AE000F18313F717008347F10252055181F99B67
:109AF000D98FA307F10297100100E780807539CD57
:109B0000AA840355050097A00000E78080BC83D796
:109B100004002AD26800231CF10083D72400231DEF
:109B2000F1001C4803D647008C4397200000E780D3
:109B300000CD8347B400CA8617860100130646800D
:109B40008117A305F4006C00481097200100E780FE
:109B5000E0805D611783FFFF670063572155D5BF24
:109B60001C45B1CF03C5A700894613576500630B99
:109B7000D7028D46630ED70285466300D7021307CE
:109B800040063305E50203C7B700418B15CB83C7F9
:109B9000B700BD8B3355F54082801375F50313076D
:109BA000803EC5B709671375F50313070771D1BF69
:109BB000372709001375F5031307077CD9B701454B
:109BC00082801783FFFFE702434E03A98500630CE1
:109BD00009048347B900AE8493F7070E85C3034594
:109BE0009900930520030D810505B305B50288444E
:109BF000610597300100E780E0A935A02E85970028
:109C00000000E78020F62A8419CD97000000E78045
:109C1000605C8325C900B307B54063FA87002E94C2
:109C2000B305A440E9F51783FFFF6700434A854564
:109C30007DBF1783FFFFE70243472A8403D5050052
:109C4000011132C636C43AC22EC002CA02CC02CEBC
:109C500097A00000E780E0A782452ACA22852ECC83
:109C600097000000E780E0E003570500231EE100B5
:109C700097500000E78040AAA24632469247230F41
:109C8000A10036874C08B286228501469700000065
:109C9000E780E0A605611783FFFF67004343178352
:109CA000FFFFE702834061711C183EC6B7078001C1
:109CB0003EC81C183ECA3C0800453ED4AA8402CCCB
:109CC00002CE02D002D202D697000000E78060DA0E
:109CD0008357050035592316F10297500000E7809D
:109CE000A0A32307A10209C48357440081EB215993
:109CF0004A855D611783FFFF6700633D035564007C
:109D00005205518197100100E780A0542A8965D13E
:109D10008347B40093F7070E99C713058401973062
:109D20000100E780609983574400231EF1008347B8
:109D300084002301F1025C4003550900D98313F725
:109D4000070883471102231CA10093F7F707D98F57
:109D5000A300F10283572900231DF1005C40F18329
:109D600013F717008347F102F99BD98FA307F1027C
:109D700097A00000E780E0952AD235D98347940068
:109D80006800139757008347B400FD8BD98FA30554
:109D9000F4001C4803D647008C4397200000E7805E
:109DA00000A6A68717770100130787597400054698
:109DB0004C10268597000000E78060942A890DD911
:109DC0008347B400A685FD8BA305F400970000002F
:109DD000E78060DF31BF1783FFFFE702032D832495
:109DE00085FE2A844111268597000000E78080D7F0
:109DF000834734FF93F7070E8DCB2AC6268597003D
:109E00000000E78060C809CD834734FFB245FD8B71
:109E1000A309F4FE91C5228597300100E780808771
:109E200041011783FFFF6700832A7DD98327C4FF81
:109E30002685829775F5834734FF93F7070E91C700
:109E4000228597300100E7802087032584FE970054
:109E50000000E78000E5E9B71783FFFFE702E32191
:109E60009C4141112A8903C7070089472E849356D4
:109E700067006380F6040D466388C6049307F00705
:109E80006304F7022E8597200000E780C0A7AA840C
:109E90008149C16B130C490097C7FF1F9387C7C641
:109EA0009C43984763E4E90441011783FFFF67007F
:109EB000832003D745008547E3F8E7FE2E859720EA
:109EC0000000E780A0A9E1B703D74500E3FEE7FC67
:109ED0002E8597200000E78000A3AA842285972082
:109EE0000000E78060A4C204C98C5DB7DC4703555D
:109EF000A900139A49003E9A93170501C187635D33
:109F0000F00083570A006397A70263E7740383276F
:109F1000CA00034D5A002DA0A1672167A98F13071E
:109F2000F7EFE374F7FE6397090097000000E780FE
:109F3000209161FD85098DB783278A00034D4A0072
:109F4000835DA90003576900216A138BC7003AC6D5
:109F5000814A33CA4D01631E5D0197C7FF1F938776
:109F600027BB9C43E1DBA2866286814526858297DA
:109F7000D1B7A1679387F7EF930C4BFF63F24703C9
:109F8000B2455A8597F0FFFFE780A0710DC1032706
:109F90008B00104709CE10436382C4023107D5BF3E
:109FA000EE85668597000000E780008F71F9938643
:109FB0001A0093FAF60F130B0B0271BF835644007D
:109FC0005C43E3E9F6F622853AC697100000E78085
:109FD000807DA1679387D7042A8A035D44003247B6
:109FE00063E897008347D90093E707F8A306F900D1
:109FF0001C4766852286E2858297C1670844FD1763
:10A00000337AFA00529508C02312A40125B797C7E6
:10A01000FF1F938767AF9843814715C31447814754
:10A0200063FFD500939745004C47BE9519C903C7F8
:10A03000550081476375E600DC451606B2973E85FC
:10A04000828003C745008147E37BE6FE16069C45F8
:10A05000F5B71783FFFFE702A303AA892E8A81447D
:10A0600097CAFF1F938A4AAA83A70A00984763E604
:10A07000E4001783FFFF6700E304DC471394440008
:10A0800001493E9413BB140083474400634BF9001D
:10A09000014913BB140083475400634FF900850442
:10A0A000E1B70844931759005287DA860146A28522
:10A0B0003E9582990509C9BF4844931759005287B4
:10A0C000DA860546A2853E9582990509E9B7178388
:10A0D000FFFFE70283FD814517F5FFFF13050548E4
:10A0E00097C7FF1F239407A297000000E780A0F600
:10A0F0001783FFFF6700A3FD97C7FF1F9387C7A0C4
:10A100009C4395C31783FFFFE70223FA814517F5A8
:10A11000FFFF1305A54497000000E780C0F31783F5
:10A12000FFFF6700C3FA82801783FFFFE70243F651
:10A1300037E404008327841241112315E100AE891E
:10A140003289368A3A8681460147ED45AA8482974C
:10A150002AC621C90356A100D28597400100E78095
:10A16000C0248327C413CE8526858297058905C917
:10A170008327440D2314210101462C002685829754
:10A180002A8401C9B7E7040083A7C712ED45280058
:10A190008297228541011783FFFF6700A3F249449C
:10A1A000D5B76554FDB75C41FD175CC1828017834C
:10A1B000FFFFE70283EFB7E70400FC5F8297954754
:10A1C0003305F50281450D811783FFFF670023F0FA
:10A1D0001783FFFFE70263EDB7E70400FC5F829798
:10A1E00095473305F5020D811783FFFF670023EEC6
:10A1F0001783FFFFE70263EBB7E7040083A7870B32
:10A200000355050082971783FFFF670043EC178310
:10A21000FFFFE70283E9035505003287AE861796F4
:10A22000FF1F0356862597C5FF1F9385A58E9700B0
:10A230000000E780A0EF1783FFFF670043E9178363
:10A24000FFFFE70283E6B7E7040083A7C7178297FB
:10A250001783FFFF6700A3E71783FFFFE702E3E42D
:10A26000B7E7040083A7871397C5FF1F9385858AE7
:10A27000829701451783FFFF670063E51783FFFFA0
:10A28000E702A3E2B7E7040083A7C71F814517953C
:10A29000FF1F0355851A82971783FFFF670023E38B
:10A2A0001783FFFFE70263E0B7E7040083A7871384
:10A2B00097C5FF1F93850587829701451783FFFF89
:10A2C0006700E3E01783FFFFE70223DEB7E7040040
:10A2D00083A7C71F81451795FF1F0355051C82974C
:10A2E0001783FFFF6700A3DE1783FFFFE702E3DBAF
:10A2F0002E8597800000E780E0AF97800000E78020
:10A30000E0EC1783FFFF670083DC1783FFFFE702A2
:10A31000C3D997800000E780E0F61783FFFF67004E
:10A3200003DB5C49E1175CC95CC583572501A107C4
:10A330002319F50083570501A1072318F500828032
:10A34000F1473305F50297B7FF1F9387A77F9C431B
:10A350003E9582808D476315F60803D746008547F2
:10A3600063F0E7081783FFFFE70223D436853684BE
:10A370002E8997100000E780005929C983574400AF
:10A3800093140501C18063E39704228597100000B0
:10A39000E7806057FD14231294009307A002630026
:10A3A000F5029307B0026307F50293079002631F5B
:10A3B000F500228597000100E780C08501A80146CD
:10A3C000CA85228597A00000E78060B01783FFFF51
:10A3D0006700E3CF228597100000E780C003FDB738
:10A3E000828097B6FF1F938626769C42014599CFBF
:10A3F0009843D44217B6FF1F2328E6746396D7000C
:10A4000097B6FF1F23A4E6741385C7FE82801783C7
:10A41000FFFFE70283C997000000E780A04B71446B
:10A4200033058502914597900000E78020E911E50A
:10A4300065551783FFFF670083C997B7FF1F23A1E7
:10A44000A77097000000E780E0483305850291453A
:10A4500097900000E78080E661DD97B7FF1F23A398
:10A46000A76E97000000E780E04697B7FF1F239391
:10A47000A76C97000000E780E04597B7FF1F239C7B
:10A48000A76A977701009387E7F017B7FF1F232785
:10A49000F76A97070000938707E917B7FF1F232D77
:10A4A000F768014579B71783FFFFE70203C0AA8564
:10A4B00017B5FF1F1305056897100000E780C05B04
:10A4C0001783FFFF6700A3C01783FFFFE702E3BD09
:10A4D00097000000E78060FD97100000E780405B78
:10A4E00097B7FF1F938747669C4391CF1387C7FE9B
:10A4F00019CB83D5C7FF17B5FF1F130565659720D7
:10A500000100E78020191783FFFF670043BC178312
:10A51000FFFFE70283B997000000E780C0EC09CD98
:10A52000834785002A8493F7070499EB0355E500D8
:10A5300097000000E78080F91783FFFF670023B9C9
:10A540008347C5009304450117B9FF1F1309C95F6D
:10A5500085E3832709005CC997B7FF1F23A6975E91
:10A5600083274900F1FB97B7FF1F23A1975EE9B747
:10A57000FD172306F500610597800000E780C0D62F
:10A580008307840063CB07048347840093E707F8BD
:10A590002304F400B7E704009C5F82974205A947B3
:10A5A00041813375F5028347840093F707FCC98F17
:10A5B0002304F4008347D4003E951C402318A400D4
:10A5C00089CF984319CB8347C40050408145850704
:10A5D0003305F502420541810297832709005CC8D3
:10A5E00097B7FF1F23A297568327490089E797B79C
:10A5F000FF1F23AD97548347C4009DDF835504019B
:10A6000017B5FF1F1305C55497200100E780800888
:10A6100025B71783FFFFE70243A997B7FF1F93876B
:10A6200067789C4701448583858B85E3AE84B2853A
:10A630003A8697100000E780804B2A8419C597104E
:10A640000000E780C041829408CC22851783FFFF79
:10A650006700E3A71783FFFFE70283A341112E8959
:10A6600032C6AA8997000000E780C031324713063E
:10A670000502CA86970500009385C5CC17B5FF1F54
:10A680001305454B97000000E780E0F82A8425C9B0
:10A690009304C50097000000E780E0411946AA85B1
:10A6A000268597100000E780801585452685971040
:10A6B0000000E780601117750100130565CB4E950A
:10A6C00083450500268597100000E78020165C482A
:10A6D00031468145A1075CC85CC483572401E1175A
:10A6E0002319F40083570401E1172318F4001C4CCC
:10A6F0003E859780FFFFE780409EA30425012285C9
:10A7000041011783FFFF6700E39B1783FFFFE70209
:10A71000C3994111AA842EC632C497100000E78065
:10A720006036004DB2452246834784000CC050C0BD
:10A7300093F7F70393E707042304F40023180400B6
:10A74000268597100000E780803183479400A94652
:10A750002317A40013D7370005073307D7029D8BB3
:10A7600085072306F400A306E40083C70401D84844
:10A770008507230FF7FE17B7FF1F1307E73C584362
:10A78000232A04009307440129E317B7FF1F232F4F
:10A79000F73A17B7FF1F2329F73A17B4FF1F13041F
:10A7A000243B228597200100E78000E11C44858B33
:10A7B0005D8D19E58145228597200100E78080EDB8
:10A7C00041011783FFFF670083901CC317B7FF1F6A
:10A7D000232EF736D9B71783FFFFE702038D9705BE
:10A7E0000000938565B7014597000000E78000B041
:10A7F00001451783FFFF6700838D1783FFFFE70283
:10A80000C38A97000000E78080B01783FFFF6700CE
:10A81000038C8347C500A5E31783FFFFE702E388A6
:10A820002A840355E50097000000E78000C821C195
:10A830008347840093F7F7FB2304F4001C4091C77F
:10A84000DC4381C74C400145829797000000E780B8
:10A8500080B917B5FF1F1305A52F97200100E780CA
:10A86000A0E50355E40097000000E78020C61783A9
:10A87000FFFF6700C38582801783FFFFE702E38243
:10A8800097B7FF1F9387472C97050000938565C8EE
:10A8900017B5FF1F1305C52B23A0070023A2070030
:10A8A00097200100E780E0CE1783FFFF6700238237
:10A8B0001C4D91CFDC4381CF1773FFFFE702E37E8E
:10A8C0008345070082971783FFFF670043808280DC
:10A8D00097B7FF1F9387072A9C4303C50700828011
:10A8E00097B7FF1F938707299C4303C517008280F2
:10A8F00097B7FF1F938707289C4303C527008280D3
:10A9000097B7FF1F938707279C4303C547008280A3
:10A9100097B7FF1F938707269C4303C537008280A4
:10A9200097B7FF1F938707259C4303C55700828075
:10A9300097B7FF1F938707249C4303C56700828056
:10A9400097B7FF1F938707239C4303C57700828037
:10A9500097B7FF1F938707229C4303C58700828018
:10A9600097B7FF1F938707219C4303C597008280F9
:10A9700097B7FF1F938707209C4303C5A7008280DA
:10A9800097B7FF1F9387071F9C4303C5B70011E1CB
:10A990001D45828097B7FF1F9387C71D9C4303C542
:10A9A000C700828097B7FF1F9387C71C9C4303C5CE
:10A9B000D700828097B7FF1F9387C71B9C4303C5AF
:10A9C000E700828097B7FF1F9387C71A9C4303D580
:10A9D0000701828097B7FF1F9387C7199C4303C560
:10A9E0002701828097B7FF1F9387C7189C4303D521
:10A9F0004701828097B7FF1F9387C7179C4303D5F2
:10AA00006701828097B7FF1F9387C7169C4303D5C2
:10AA10008701828097B7FF1F9387C7159C4303C5A3
:10AA2000A701828097B7FF1F9387C7149C4303C574
:10AA3000B701828097B7FF1F9387C7139C4303C555
:10AA4000C701828097B7FF1F9387C7129C4303C536
:10AA5000D701828097B7FF1F9387C7119C43885700
:10AA6000828097B7FF1F9387E7109C4303D5C702E7
:10AA7000828097B7FF1F9387E70F9C4303D5E702B8
:10AA800019E11305800C828097B7FF1F9387870E0B
:10AA90009C4303C50703828097B7FF1F9387870DE9
:10AAA0009C43C85B828097B7FF1F9387270C88431E
:10AAB000828097B7FF1F9387A70B8843828019E195
:10AAC0007D558280F5DE984265DFFDD917B7FF1FFF
:10AAD0001307472D1847AA877155058B631D072457
:10AAE00003C507001547E37DA7FC03C7370013051F
:10AAF000F0057D171377F70FE364E5FC03C35700F8
:10AB0000E30003FC83C86700E38C08FA03C77700FF
:10AB1000494579171377F70FE364E5FA03C7A700F0
:10AB200011481305F7FF1375F50FE36BA8F803CE73
:10AB300097000D481305FEFF1375F50FE362A8F8A3
:10AB400003C8B7006309080065181378F80F1305E8
:10AB5000600DE36705F703C5C700794879151375DC
:10AB6000F50FE36FA8F403C8D7000D457D181378DF
:10AB7000F80FE36705F503D80701930E4017511846
:10AB8000420813580801E3ED0EF303C8E7007D18EF
:10AB90001378F80FE36605F303C827017D181378CF
:10ABA000F80FE36F05F103C88700C54E75181378D9
:10ABB000F80FE3E70EF103D86701856E938EBEE0D0
:10ABC0006D18420813580801E3EC0EEF03D8470153
:10ABD0006D18420813580801E3E40EEF03D887010B
:10ABE0007918420813580801E36C05ED03C8A70162
:10ABF0007D181378F80FE36505ED03C5B7011D480F
:10AC00007D151375F50FE36DA8EA03C5D7017148EB
:10AC100079151375F50FE365A8EA03D5E701130865
:10AC2000E00F7D1542054181E36CA8E803C50702EA
:10AC3000494879151375F50FE364A8E8C85301C9AD
:10AC400037C834005915130858BFE36BA8E603A8AA
:10AC5000870237C53400130555BF5918E36205E76D
:10AC600017B5FF1F2326C5F003C6050117B5FF1F43
:10AC70002322F5F00545E375C5E403D82501D04945
:10AC800033760603E31E06E203C61501E30A06E275
:10AC900017B6FF1F232CB6EC83C527000146638738
:10ACA000A50003C61700F1453306B60283C70703A4
:10ACB0009305C00272971A071307C70516031A9760
:10ACC00096084697B387B70241553E973297420799
:10ACD00041836362E8061773FFFFE702033D368591
:10ACE00097800000E780A06897000100E780204877
:10ACF0002A8497A00000E780805A2A9497F00000E9
:10AD0000E78060262A9497900000E780A0812A942B
:10AD100097F0FFFFE780E06F2A9497400000E780FC
:10AD200060932A9497700000E780A09C2295177387
:10AD3000FFFF6700C33982801773FFFFE702E33626
:10AD40004111A307A10097A00000E780A0C59305CB
:10AD5000F100170500001305E5B597F0FFFFE78048
:10AD6000802F014541011773FFFF670043361773BA
:10AD7000FFFFE702033117B4FF1F1304A4020328E7
:10AD8000840079599368180097B4FF1F23A0140317
:10AD90001378180063100802BA84BE89368B328A91
:10ADA0002E89AA8A97F0FFFFE780E0A77D152695F8
:10ADB00019E531594A851773FFFF6700033097F093
:10ADC000FFFFE78040A67D152695A167E353F5FEBA
:10ADD00097B7FF1F9387073498433E8C814B01CB75
:10ADE000014597F00000E7802044933B15004A8519
:10ADF000DA865686D28597900000E780C04D2A8972
:10AE000011CD1C44F99B17B7FF1F2321F7FA8327A5
:10AE10000C00CDD3E3800BFA829769BF268597B7E4
:10AE2000FF1F23A307F897F0FFFFE780809C4146B0
:10AE3000CE8517B5FF1F1305650097300100E78029
:10AE4000C05697D00000E78040990325040B97D0A7
:10AE50000000E780009D054597D00000E78000A432
:10AE6000054597000000E78060EDA9B797B7FF1F81
:10AE7000938747F39C47858BEDC71773FFFFE70266
:10AE8000C32217B5FF1F1305A5F997B7FF1F23AB03
:10AE900007F097B7FF1F23A907F097B7FF1F23A756
:10AEA00007F097200100E780208197500000E7809D
:10AEB000E0F597100100E780A04C97100100E780B3
:10AEC000A05297B7FF1F938767EC9C4391C7054536
:10AED00097800000E780402097B7FF1F9387C7D473
:10AEE0009C4399C741657D1597700000E78040A29B
:10AEF00097F00000E780E03D97D00000E780808F6A
:10AF000097B7FF1F938707FF9C431397170163565B
:10AF1000070097F00000E78000AD97B7FF1F23AF51
:10AF200007F097B7FF1F23AD07F097B7FF1F23ABBD
:10AF300007F097B7FF1F23A907F097000000E780ED
:10AF4000008C97000000E780007297F0FFFFE78019
:10AF5000401897F00000E78040D61773FFFF6700A6
:10AF60000317828097B7FF1F9387C7E388438280C8
:10AF70001773FFFFE702631397800000E780607597
:10AF800097800000E780C0771773FFFF67002314E6
:10AF90001773FFFFE702C30F2A8493041402011101
:10AFA0002E85B289A685214636C63A89973001009A
:10AFB000E780403D0DE9B24638082686CE85130568
:10AFC000940497500000E780604121462C084A8590
:10AFD00097300100E780003B1335150005611773BA
:10AFE000FFFF6700230E0145D5BF1773FFFFE70280
:10AFF000C30B9305450617B5FF1F1305E5B797105B
:10B000000100E78020691773FFFF6700430C177387
:10B01000FFFFE702830941112EC697F0FFFFE7808B
:10B02000601BB24588C141011773FFFF6700230A07
:10B030001773FFFFE702C305AA842E8497800000E0
:10B04000E780006CAA898545228597000000E7808B
:10B05000E07D83C7E4011389940899E3138904030D
:10B06000CE85228597000000E780407C214693052D
:10B070001902228597000000E780607897B7FF1FCC
:10B08000938747D28C43228597100000E780C082C7
:10B09000214693858402228597000000E780207670
:10B0A0001773FFFF670003021773FFFFE70263FDDB
:10B0B000397197F00000E780E0B49305400661E93C
:10B0C00097800000E78000606302051497B7FF1FB8
:10B0D00083C747AC13B7170097B6FF1F238CE6AAA8
:10B0E000014499CFC16417B9FF1F1309A9CB930974
:10B0F000400EFD1497000000E780C0866342A40A5A
:10B1000097F0FFFFE780000D4169B7290900096A40
:10B11000FD7A2A8B81447D199389F97B130A0A7180
:10B12000938A8AC797000000E780C08363D7A4048E
:10B130001304400EB387840217B7FF1F130787C697
:10B140000324070B3E948357C4016382270B1840E6
:10B150003307EB4063EAE900834744008507B38780
:10B160004703D6976365F70801468145094597F07F
:10B17000FFFFE780604EAA8B29E597400000E7803B
:10B18000808385476317F50689659385057117B533
:10B19000FF1F1305659E97100100E780A04F95A043
:10B1A000B30734030327090BBA9703D7C701630812
:10B1B000970003C75700A38207002382E700050416
:10B1C00015BF9305C500228597000000E78080E643
:10B1D0005E852286976501009385C51A97F0FFFF6B
:10B1E000E780E0525E8597100000E780608A850462
:10B1F00015BF97B7FF1F9387E7BA9C478D83858B51
:10B20000C1F721611773FFFF670023EB01468545F6
:10B21000094502D002D202D402D697F0FFFFE780A0
:10B22000A043AA8479DD97F00000E780E09C1389B1
:10B23000C4002A8481454A8597000000E780005FAA
:10B240000C4041464A8597000000E780405B832917
:10B2500044006385090C4E8502D802DA02DC02DE66
:10B2600097300100E78060402ACE141005462C0874
:10B2700008184ECC97500000E780E00A1375F50FD0
:10B2800051ED8355840093E525004A859700000021
:10B29000E780E05E11460C104A8597000000E780C9
:10B2A00000560146976501009385450E268597F067
:10B2B000FFFFE780C045268597000000E780407DBE
:10B2C0005C40A1D3014685450D4597F0FFFFE7801F
:10B2D000A038AA841DD548401389C40097300100C6
:10B2E000E780A0382AC64A8597000000E780404CD6
:10B2F0003246636FC5004C404A8597000000E780E6
:10B30000005001468145268597F0FFFFE7802040E9
:10B31000268597000000E780A077E5B58355840077
:10B32000ADB71773FFFFE70243D897B7FF1F9387A7
:10B3300067A79C471DC193E7870017B5FF1F13053B
:10B34000A58317B7FF1F2323F7A697100100E780F7
:10B3500040321773FFFF670083D7DD9B17B7FF1FCE
:10B360002326F7A497300000E780E0647DF117B54D
:10B37000FF1F1305658097100100E780E033D1BF00
:10B380001773FFFFE702E3CF4169AA892E8AB28AC9
:10B39000368BBA8B814417BCFF1F130CACA0930CE7
:10B3A000400E7D1997F0FFFFE780C05B63C4A400E7
:10B3B00001443DA03384940383270C0B3E948357B0
:10B3C000C401638627055A87D6865286CE85130523
:10B3D000040397000000E780E0BB01C923800B0055
:10B3E00022851773FFFF670043CD8347F40185C3B0
:10B3F0005A87D6865286CE8513059408970000009A
:10B40000E78040B909C585472380FB00D1BF85048B
:10B4100051BF835745006380071E1773FFFFE70284
:10B4200023C701112A8497000000E780C04D09C995
:10B4300085476309F50605611773FFFF670083C839
:10B4400097E00000E780007C7DF583574400494782
:10B45000ED9BE392E7FEC145228597000000E7805F
:10B460004033AA84228597000000E780204F0357CD
:10B47000440002CE91472A89631AF700228597007B
:10B480000000E780A0513C082ACC3ECE97E00000A7
:10B49000E78080765C55C5D374084A86A685054545
:10B4A000829751BF03574400D147E3F6E7F8032AD8
:10B4B0000400C169014997BAFF1F938AAA8E130B32
:10B4C000400EFD1997F0FFFFE780C049634FA90EBA
:10B4D0002285032A040097000000E780C042A145AE
:10B4E0002A89228597000000E780A02AAA84228565
:10B4F00097000000E780804A14402A86AA897808CD
:10B500002685CA8597000000E780C0E7AA8405D594
:10B5100003C7F40189476315F7008347C10181DF41
:10B520005546D2851385640097300100E780E0E737
:10B53000014597800000E780C01901C583D7C40189
:10B54000A5E797B7FF1F9387E7859C479355190099
:10B55000858913D73700058B01CF8983858B639944
:10B56000B70001452EC697000000E780C0DBB2455A
:10B570004E8597800000E780601F0346C1012A8442
:10B5800093751900268597900000E780E03935C152
:10B59000268597800000E780E018268511C00145C8
:10B5A00097800000E780004C97300000E780A040C3
:10B5B0008547E312F5E883C754001307F00FE38CC7
:10B5C000E7E68507A382F400BDB5B304690383A74A
:10B5D0000A0BBE9483D7C401638B37015546D285CD
:10B5E0001385640097300100E780C0D955DD050957
:10B5F000D1BD5DD86DB782801773FFFFE70243A905
:10B6000097800000E780000C05C1C164014417A9C0
:10B61000FF1F130929799309400EFD1497F0FFFFCE
:10B62000E7804034634EA40017A5FF1F1305C554DF
:10B6300097100100E780E0031773FFFF670083A8FE
:10B64000330534038327090B3E958357C50163886F
:10B6500097002312050097800000E780A00C0504E6
:10B6600075BF97A7FF1F9387E7739C478D83858BD3
:10B670008DE31773FFFFE70243A317A5FF1F130511
:10B68000A54F97100100E78020031773FFFF6700A5
:10B6900003A482801773FFFFE70223A19705000030
:10B6A0009385C5A017A5FF1F1305054D9710010031
:10B6B000E78020EE1773FFFF670063A11773FFFF9A
:10B6C000E702A39E8841B7E70400BC5B050542057D
:10B6D0004181829709C585472300F5000505177349
:10B6E000FFFF6700C39E83C7F5FF2E858507A38FE5
:10B6F000F5FE828083C7F5FFFD1793F7F70FA38F41
:10B70000F5FE99EF1773FFFFE702239AB7E70400EE
:10B71000BC571385F5FF82971773FFFF6700239BC4
:10B7200082801C41035745008D8FBA951CC123129E
:10B73000B5003E85828093D78500A2051441DD8D3A
:10B74000835745001387E6FF18C189072312F500C8
:10B7500013D685004111238FB6FEA38FC6FE41018B
:10B76000828018419307F7FF1CC183574500850766
:10B770002312F500A30FB7FE8280835745008D8FFB
:10B780002312F5001C41BE950CC12E858280AA872C
:10B7900003D7470008410D8FAA952392E7008CC379
:10B7A0008280184108453305A740828083574500B1
:10B7B000035765001D8F1C4108453385A74033059D
:10B7C000A74082801773FFFFE702238E41112EC628
:10B7D0002A8497000000E780A0FDB2456373B5009E
:10B7E00001A0835744000840BE952312B4003E9543
:10B7F00041011773FFFF6700838D1773FFFFE70297
:10B80000C38A41112E84B28532C697000000E780BA
:10B81000A0FB3246A28597300100E78000B94101C4
:10B820001773FFFF6700A38A1773FFFFE702E38721
:10B830002E84854597000000E78000F923008500ED
:10B840001773FFFF6700A3881773FFFFE702E38505
:10B8500041112317B100894597000000E780C0F629
:10B860008347E1002300F5008347F100A300F500C2
:10B8700041011773FFFF670083851773FFFFE7021E
:10B88000C38293D78500A2054111DD8D2317B10036
:10B89000894597000000E78020F38347E1002300FB
:10B8A000F5008347F100A300F50041011773FFFF86
:10B8B0006700E3811763FFFFE702237F139785018A
:10B8C00093D78501C166938606F0D98F13D785007B
:10B8D000758FD98FA2053707FF00F98D4111DD8DD6
:10B8E0002EC6914597000000E78000EE6C001146DF
:10B8F00097300100E78060AB41011763FFFF6700ED
:10B90000037D1763FFFFE702437A1C41854503C4AB
:10B91000070097000000E78080E622851763FFFF9D
:10B920006700E37A1763FFFFE70223781C414111A8
:10B93000894503C7070083C717002307E100A30752
:10B94000F10097000000E78080E30355E10041012A
:10B950001763FFFF6700A3771763FFFFE702E37436
:10B960001C414111894503C7070083C717002307FE
:10B97000E100A307F10097000000E78040E0835753
:10B98000E100410113D58700A2075D8D4205418189
:10B990001763FFFF6700A3731763FFFFE702E370FE
:10B9A0000C4141112A841146680097300100E7805C
:10B9B000C09F9145228597000000E78040DCB24798
:10B9C000C166938606F01397870113D58701598DB9
:10B9D00013D78700758F598DA2073707FF00F98F9E
:10B9E0005D8D41011763FFFF6700636E1C45BE95C7
:10B9F0000CC18280AE87944391E6584101EF0CC19F
:10BA00005CC1828003C7570013671700A382E70059
:10BA1000B687D5B70CC3EDB7AA87084119CD184131
:10BA2000D44398C36313D500D8C32A87034657006D
:10BA30009376160081E6232007008280944381CA12
:10BA40008C4203A847008CC363930601CCC3799A48
:10BA500014C3A302C7003687D1BF1C45DC471D8D28
:10BA6000B777DBB6938777DB09853305F5024205A7
:10BA700041818280F147B385F50248452E95828049
:10BA80008347450085072302F50082801763FFFF87
:10BA9000E702A3612A8409E41763FFFF67002363B9
:10BAA00083474400F5DBFD1793F7F70F2302F400FB
:10BAB000E5F71C4403D7270005072391E700DC4383
:10BAC00099C3228582974C4889CD83475400898B3E
:10BAD00099E71C4422859C479C439C478297232AD4
:10BAE00004000040232004007DB71763FFFFE70236
:10BAF000C35B8357250041112EC681EB014422858B
:10BB000041011763FFFF6700835C0357050081470E
:10BB1000F146E305F7FEB385D702404585072E942D
:10BB20008345440008C4F5F5B247AA8481E7232A77
:10BB3000040009A81C456C0022859C439C43829705
:10BB400048C84DDD85472312F400B2472320040086
:10BB5000231804002319F4005C485CC483D7240034
:10BB6000FD172391F40061BF1763FFFFE702E35362
:10BB700097A7FF1F938747028843232605002324A6
:10BB80000500410597100100E78000B31763FFFF30
:10BB90006700E3531763FFFFE702235117A4FF1F5A
:10BBA000130484FF1C40411199CF9C472300B5002A
:10BBB0002AC65CC197000000E78040FB1C40DC43C4
:10BBC00099C33245829741011763FFFF67002350F5
:10BBD0000347450029E3584DAA877D551DCF1763BC
:10BBE000FFFFE702834C1CC3DC4797A6FF1F23A57A
:10BBF000E6FAF156130507012390D70097050000D8
:10BC00009385050297100100E780A098014517630E
:10BC1000FFFF6700C34B7D55828082801763FFFF63
:10BC2000E702A34801116146814528009760FFFFA4
:10BC3000E780A04A97A7FF1F938707F69C43280039
:10BC40009305F00FDC473EC697000000E780C0F484
:10BC500005611763FFFF6700834797A7FF1F93875F
:10BC6000A7F39C43D847A1679387C702631EF70ACF
:10BC7000397106DE22DC26DA80004AD84ED652D44C
:10BC800056D23285B28497000000E780C0C7AA89E7
:10BC9000268597000000E78020C92318A4FC26858C
:10BCA00097000000E78040C82319A4FC2685970070
:10BCB0000000E78060C783D744000A8A231AA4FCE7
:10BCC000858393F7F70F230EF4FC8607BD0793F7E0
:10BCD000073F3301F1408A8A01498347C4FD636706
:10BCE000F902CE85130584FC232C54FD9700000037
:10BCF000E78080EA5281130104FCF2506254D2546E
:10BD00004259B259225A925A21618280268597005F
:10BD10000000E78060C193171900D69705092390AA
:10BD2000A7001379F90F55BF828097A7FF1F93874C
:10BD3000A7E69C43D847A1679387A702631AF70A2F
:10BD4000397106DE22DC26DA80004AD84ED652D47B
:10BD500056D23285B28497000000E780C0BAAA8923
:10BD6000268597000000E78020BCFD572318A4FC1F
:10BD700026852319F4FC97000000E780E0BA83D7FA
:10BD800044000A8A231AA4FC858393F7F70F230E35
:10BD9000F4FC8607BD0793F7073F3301F1408A8A19
:10BDA00001498347C4FD6367F902CE85130584FC0E
:10BDB000232C54FD97000000E78000DE5281130120
:10BDC00004FCF2506254D2544259B259225A925A47
:10BDD00021618280268597000000E780E0B49317F8
:10BDE0001900D69705092390A7001379F90F55BFBD
:10BDF000828097A7FF1F938727DA9C43D847A167C4
:10BE000089076310F70A397106DE22DC26DA800022
:10BE10004AD84ED652D456D2328532899700000085
:10BE2000E78060AEAA894A8597000000E780C0AF2E
:10BE3000835749000A8A2318A4FC858393F7F70FD8
:10BE4000230CF4FC8607BD0793F7073F3301F1404D
:10BE50008A8A8144834784FD63E7F402CE85130513
:10BE600084FC232A54FD97000000E780E0D2528131
:10BE7000130104FCF2506254D2544259B259225A6E
:10BE8000925A216182804A8597000000E780C0A90C
:10BE900093971400D69785042390A70093F4F40F8A
:10BEA00055BF828097A7FF1F938707CF9C43D84732
:10BEB000A1679387E704631EF70A397106DE22DC67
:10BEC00026DA80004AD84ED652D456D23285B28471
:10BED00097000000E78020A3AA892685970000002C
:10BEE000E78080A42318A4FC268597000000E78043
:10BEF000A0A3231AA4FC268597000000E780C0A217
:10BF000083D744000A8A2319A4FC858393F7F70F8B
:10BF1000230EF4FC8607BD0793F7073F3301F1407A
:10BF20008A8A01498347C4FD6367F902CE851305F8
:10BF300084FC232C54FD97000000E780E0C552816B
:10BF4000130104FCF2506254D2544259B259225A9D
:10BF5000925A21618280268597000000E780C09C6C
:10BF600093171900D69705092390A7001379F90FA5
:10BF700055BF828097A7FF1F938707C29C43D8476E
:10BF8000A1679387C704631AF70A397106DE22DCBA
:10BF900026DA80004AD84ED652D456D23285B284A0
:10BFA00097000000E7802096AA8926859700000068
:10BFB000E7808097FD572318A4FC2685231AF4FCFC
:10BFC00097000000E780409683D744000A8A23192F
:10BFD000A4FC858393F7F70F230EF4FC8607BD07B7
:10BFE00093F7073F3301F1408A8A01498347C4FD33
:10BFF0006367F902CE85130584FC232C54FD97005A
:10C000000000E78060B95281130104FCF2506254D1
:10C01000D2544259B259225A925A216182802685BD
:10C0200097000000E780409093171900D697050904
:10C030002390A7001379F90F55BF828097A7FF1FA0
:10C04000938787B59C43D847A167DD076317F7043B
:10C050001763FFFFE7026305797132853284970029
:10C060000000E780408A2AC6228597000000E7800A
:10C07000A08B2311A102228597000000E780A088F1
:10C08000B2452300A102280897000000E780C0B055
:10C0900045611763FFFF67008303828097A7FF1F37
:10C0A000938787AF9C43D847A1679387870463171B
:10C0B000F7041763FFFFE70243FF7971328532848B
:10C0C00097000000E78020842AC6228597000000A0
:10C0D000E78080852311A102228597000000E78078
:10C0E0008082B2452300A102280897000000E78063
:10C0F000A0AA45611763FFFF670063FD828097A7D1
:10C10000FF1F938767A99C43D847A1679387A7041C
:10C110006312F7021763FFFFE70223F901112800FA
:10C12000814597000000E78020A705611763FFFFA6
:10C130006700E3F9828097A7FF1F9387E7A59C43D9
:10C14000D847A167938757026319F7021763FFFF68
:10C15000E702A3F50111328597F0FFFFE780A07A8F
:10C160002308A1008145280097000000E780C0A2B5
:10C1700005611763FFFF670083F5828097A7FF1FA4
:10C18000938787A19C43D847A1679387E702631BE6
:10C19000F7041763FFFFE70243F101113285328490
:10C1A00097F0FFFFE7804078AA84228597F0FFFF91
:10C1B000E7808077854709E9228597F0FFFFE780D0
:10C1C00080744205B337A0002800814523189100F0
:10C1D0003ECA97000000E780209C05611763FFFFBF
:10C1E0006700E3EE828097A7FF1F9387E79A9C433F
:10C1F000D84799476313F7081763FFFFE702E3EA9D
:10C2000079713285328497F0FFFFE780C06F2AC6CC
:10C21000228597F0FFFFE78020712310A10222857D
:10C2200097F0FFFFE780206E2301A102228597F09F
:10C23000FFFFE780406DA301A102228597F0FFFF79
:10C24000E780606C2302A102228597F0FFFFE78060
:10C25000806B2313A102228597F0FFFFE780A06A7D
:10C26000B2452314A102280897000000E780C0927D
:10C2700045611763FFFF670083E5828097A7FF1F73
:10C28000938787919C43D847A1679387C70363131C
:10C29000F7081763FFFFE70243E1797132853284C3
:10C2A00097F0FFFFE78020662AC6228597F0FFFF00
:10C2B000E78080672310A102228597F0FFFFE780C7
:10C2C000A0662311A102228597F0FFFFE780A063FB
:10C2D0002302A102228597F0FFFFE780C062A3023C
:10C2E000A102228597F0FFFFE780E0612303A1020E
:10C2F000228597F0FFFFE7800061B245A303A1020A
:10C30000280897000000E780208945611763FFFF38
:10C310006700E3DB82801763FFFFE70203D90111A7
:10C320002A8497F0FFFFE780005EAA84228597F0B9
:10C33000FFFFE780605F228597F0FFFFE780C05E28
:10C34000035744008D4763F7E700228597F0FFFF0E
:10C35000E780805D228597F0FFFFE780E05C2800A2
:10C36000A68597000000E780208305611763FFFF23
:10C370006700E3D597A7FF1F938707829C43D847A1
:10C38000A167FD07631FF7001763FFFFE702E3D113
:10C39000328597000000E78040F81763FFFF6700D1
:10C3A00003D382809797FF1F9387077F9C43D847CB
:10C3B000A167E5076315F7081763FFFFE702E3CE00
:10C3C00079713285328497F0FFFFE780C0532AC627
:10C3D000228597F0FFFFE7802055228597F0FFFF29
:10C3E000E78080542310A102228597F0FFFFE780A9
:10C3F000A053520551812311A1022285230201027B
:10C4000097F0FFFFE7802050A302A102228597F05A
:10C41000FFFFE780404F2303A102228597F0FFFF33
:10C42000E780604EB245A303A102280897F0FFFF02
:10C43000E780807645611763FFFF670043C982800C
:10C440009797FF1F938747759C43D847A1679387AA
:10C45000E703631FF7001763FFFFE70203C5328599
:10C4600097000000E78060EB1763FFFF670023C6BB
:10C4700082809797FF1F938727729C43D847A167B5
:10C4800093874704631EF7021763FFFFE702E3C1C8
:10C4900079713285328497F0FFFFE780C0462AC663
:10C4A000228597F0FFFFE7802048B245280897F0E3
:10C4B000FFFFE780606E45611763FFFF670023C1E0
:10C4C00082809797FF1F9387276D9C43D847A1676A
:10C4D000938787026310F7041763FFFFE702E3BC4B
:10C4E00079713285328497F0FFFFE780C0412AC618
:10C4F000228597F0FFFFE7800041B2452300A102AB
:10C50000280897F0FFFFE780206945611763FFFF68
:10C510006700E3BB82801763FFFFE70203B90111E5
:10C5200097F0FFFFE780203EAA85280097F0FFFFE5
:10C53000E780806605611763FFFF670043B997973F
:10C54000FF1F938767659C43D847A167D107631F87
:10C55000F7001763FFFFE70243B53285970000003D
:10C56000E780A0FB1763FFFF670063B682809797A1
:10C57000FF1F938767629C43D847A167C507631F66
:10C58000F7001763FFFFE70243B232859700000010
:10C59000E780A0F81763FFFF670063B38280979777
:10C5A000FF1F9387675F9C43D847A167B907631F45
:10C5B000F7001763FFFFE70243AF328597000000E3
:10C5C000E780A0F51763FFFF670063B0828097974D
:10C5D000FF1F9387675C9C43D847A167AD07631F24
:10C5E000F7001763FFFFE70243AC328597000000B6
:10C5F000E780A0F21763FFFF670063AD8280979723
:10C60000FF1F938767599C43D84789476318F702F0
:10C610001763FFFFE70263A90111328532C897F063
:10C62000FFFFE780402EAA85280097F0FFFFE780F4
:10C63000A05605611763FFFF670063A98280979783
:10C64000FF1F938767559C43D847A1678D076311E8
:10C65000F7041763FFFFE70243A501113285328417
:10C6600097F0FFFFE780202A13066100AA844C00A0
:10C67000228597300000E780C0232800A68597F028
:10C68000FFFFE780605105611763FFFF670023A488
:10C6900082809797FF1F938767509C4381CFDC432D
:10C6A00091CB1763FFFFE70243A082971763FFFF59
:10C6B0006700E3A182801763FFFFE702039F7971A0
:10C6C0003C08AE843ED2A165B7070A002A843ED456
:10C6D00048103C08DD053ED636C432C63AC297D073
:10C6E000FFFFE780E02F12474810BA8597F0FFFF61
:10C6F000E780C01332464810B28597F0FFFFE7800D
:10C70000E014A2464810B68597F0FFFFE7800012BC
:10C71000501001478146A685228597D0FFFFE7800C
:10C72000805145611763FFFF6700639A1763FFFF3E
:10C73000E702A39701117C000329C501AE843ECA1C
:10C74000A165B70707002A843ECC48087C00C505D0
:10C750003ECE97D0FFFFE780A0288345D900480848
:10C7600097F0FFFFE780800C500801478146A685BF
:10C77000228597D0FFFFE780004C05611763FFFF1C
:10C780006700E3941763FFFFE702239283C79500D6
:10C7900093F7F707A384F50097000000E78040F9BE
:10C7A0001763FFFF6700A3921763FFFFE702E38FA2
:10C7B00079713C08AE843ED2A165B70709002A848E
:10C7C0003ED448103C08938545043ED632C636C454
:10C7D00097D0FFFFE780C020A2464810B68597F0AB
:10C7E000FFFFE780A00432464810B28597F0FFFFB4
:10C7F000E780C005501001478146A685228597D065
:10C80000FFFFE780404345611763FFFF6700238C0C
:10C810001763FFFFE702638983C7950041112A84EC
:10C8200093F7F707A384F50032852EC697F0FFFF34
:10C83000E780800F85672AC46370F5029770000057
:10C84000E78020E92246B24509ED1147814622855D
:10C8500097000000E78060E641011763FFFF670073
:10C86000038701478346F501DDB71763FFFFE70242
:10C87000238201113C003ECAB7070A003ECC3C00AF
:10C880003ECE83C79500AA89328593F7F707A38424
:10C89000F5002E8497F0FFFFE78000098567637D30
:10C8A000F504A165AA8493858504480897D0FFFF05
:10C8B000E7800013268597700000E78080E12A89D1
:10C8C00029E19145480897F0FFFFE78020F6A6850B
:10C8D000480897F0FFFFE78060F7CA85480897F09F
:10C8E000FFFFE780A0F4014781465008A2854E85EE
:10C8F00097D0FFFFE780203405611753FFFF6700E3
:10C90000637C8145480897F0FFFFE78020F20349E8
:10C91000090275BF1753FFFFE702837779711C1077
:10C920003ECAB7070F003ECC404D1C10AA84AE890A
:10C930004808994532C636893ECE97D0FFFFE7803A
:10C94000200A32464808B28597F0FFFFE78000EEE4
:10C95000630C0902A545480897F0FFFFE780C0E691
:10C960002546CA8597200100E78020A4500801478A
:10C970008146CE85268597D0FFFFE780C02B456195
:10C980001753FFFF670003748355C402480897F0EC
:10C99000FFFFE780A0EB0355E402814505C585470D
:10C9A00085456301F502C167FD179305F00F630B21
:10C9B000F5007D1597700000E780208E9305150027
:10C9C00093F5F50F480897F0FFFFE78020E68345D1
:10C9D0000403480897F0FFFFE78040E58345140310
:10C9E000480897F0FFFFE78060E483552403480878
:10C9F00097F0FFFFE78080E583554403480897F0F0
:10CA0000FFFFE780A0E49DB71753FFFFE702E3694C
:10CA100083C795008146014693F7F707A384F50085
:10CA200097000000E78040EF1753FFFF6700236A7D
:10CA30001753FFFFE702636779713E841C103ECAFB
:10CA40002E89B7070F00A1653ECCFD051C10AA84F6
:10CA5000480842C03AC23ECE36C432C697D0FFFF25
:10CA6000E78000F832464808B28597F0FFFFE7807C
:10CA7000E0DBA2464808B68597F0FFFFE78000DDBF
:10CA800012474808BA8597F0FFFFE78020DC02488C
:10CA9000630C08029145480897F0FFFFE780C0D279
:10CAA0001146A28597200100E78020905008014799
:10CAB0008146CA85268597D0FFFFE780C01745616C
:10CAC0001753FFFF6700A3608945480897F0FFFFF1
:10CAD000E78080CF834704002300F50083471400DC
:10CAE000A300F500E1B71753FFFFE702635A83C7BE
:10CAF000950001112A8A93F7F707A384F500328580
:10CB0000AE8432C697F0FFFFE78000E232462A8902
:10CB1000328597F0FFFFE78000DF85676373F902D6
:10CB2000AA894A8597700000E780A0BA2A8419ED87
:10CB3000114781464A86A685528597000000E78006
:10CB4000C0B705611753FFFF6700C3579387E9FF1D
:10CB500093F7F70F0547E366F7FE8347F50195EB7B
:10CB60008947E380F9FE8346F401528501474A86EE
:10CB7000A68597000000E78040B4A167D907480860
:10CB80003ECC230A010002CE97000000E780A0B04F
:10CB90004DBF639EE7008947639EF900930710200D
:10CBA000231FF50097700000E780C0B76DBF0947ED
:10CBB000E39BE7FA8D47E398F9FA22859770000026
:10CBC000E78080DF9797FF1F9387471C9C4399E777
:10CBD0009797FF1F938747059C4399C703D5040088
:10CBE00097800000E780A0CE231F040022855DBF50
:10CBF0001753FFFFE702634B01113C003ECAB70722
:10CC00000B003ECC3C003ECE83C795002A8932857E
:10CC100093F7F707A384F500AE8497F0FFFFE78052
:10CC2000A0D093170501C187635AF006A1652A8435
:10CC30009385E502480897D0FFFFE78060DAA28578
:10CC4000480897F0FFFFE78060C09797FF1F938722
:10CC5000A7FD9C43A9EB01449375F40F480897F096
:10CC6000FFFFE780A0BC9355844093F5F50F48087B
:10CC700097F0FFFFE78080BB9355044193F5F50FD4
:10CC8000480897F0FFFFE78060BA014781465008E7
:10CC9000A6854A8597D0FFFFE780E0F90561175325
:10CCA000FFFF6700C342416585460546A2857D15A5
:10CCB00097500000E78060BD59DD510597000100E5
:10CCC000E780808F130440063344850271B7175301
:10CCD000FFFFE702833D0111B70706003EC683C789
:10CCE000950021642A8993F7F707A384F500AE84A1
:10CCF00028009305A4040AC40AC897D0FFFFE78060
:10CD000020CE300001478146A6854A8597D0FFFF97
:10CD1000E78060F297E0FFFFE7808015130494043A
:10CD2000480822CC230A010002CE97000000E780C9
:10CD3000809605611753FFFF670063391753FFFFA4
:10CD4000E7020335C1642A8901449799FF1F93893B
:10CD50006905130A8002FD1497E0FFFFE78080C198
:10CD60006347A40001451753FFFF6700A335B307CE
:10CD7000440303A7C90ABA9703D7070063069700BD
:10CD800083D72700638427010504F9B70545E1BF70
:10CD90001753FFFFE702C32F2A8A2E8999C123A0C8
:10CDA000050081498144979AFF1F938A6ADF614B8E
:10CDB00097E0FFFFE78040C263C7A4004E8517538A
:10CDC000FFFF670023303384640383A70A003E9487
:10CDD0008357040099E76304090023208900850430
:10CDE000C1BF4146D2851305440097100100E7807A
:10CDF000605975F5A289E5B71753FFFFE70243298C
:10CE000039717C083ED4B7070A003ED67C083ED86C
:10CE100083C795002A8A328593F7F707A384F50024
:10CE20002E8932C697F0FFFFE78000B085676373F5
:10CE3000F5083246AA84328597F0FFFFE780A0AC60
:10CE40008547AA8963E8A706A1659385850428100C
:10CE500097D0FFFFE780C0B8268597700000E78075
:10CE600040872A8429ED9145281097F0FFFFE7803D
:10CE7000E09BA685281097F0FFFFE780209DCE85D8
:10CE8000281097F0FFFFE780609A01478146301035
:10CE9000CA85528597D0FFFFE780E0D9A1679387C5
:10CEA000770448183EDC230A010202DE97F0FFFFF8
:10CEB000E780607E21611753FFFF6700A320814553
:10CEC000281097F0FFFFE7806096A685281097F05E
:10CED000FFFFE780A0979797FF1F938767239C43E7
:10CEE00081CB22856389090097D00000E780402428
:10CEF0008345040271B797D00000E780C022CDBF00
:10CF00001753FFFFE702C31883C795004111AA8991
:10CF100093F7F707A384F5003285AE84328A97F041
:10CF2000FFFFE78060A08567637FF5022A8997602D
:10CF30000000E780007A2A84914631C58347F501D5
:10CF400005476387E70291C70D476366F704AD465F
:10CF50001DA89305050303250A004146971001000B
:10CF6000E78040420DE941011753FFFF6700831539
:10CF70009305950803250A00414697100100E780B4
:10CF80006040814669F54A86A6854E859700000077
:10CF9000E780C081C9BF83250A00130594089770F4
:10CFA0000000E780A02919C1C146F1BF9797FF1F74
:10CFB0009387C7DD9C4399E79797FF1F9387C7C661
:10CFC0009C4399C7228597800000E780208A69FDED
:10CFD0008547A30FF400228597B00000E7806084A6
:10CFE000228597600000E780E0734E8581464A867F
:10CFF000A68597F0FFFFE780607BA16793875704C2
:10D0000048003EC42302010002C697F0FFFFE780FC
:10D01000806891BF1753FFFFE702A30683C79500FF
:10D020004111AA8993F7F707A384F50032852E8969
:10D03000B28A97F0FFFFE780208F85676374F50E53
:10D04000AA8497600000E780C0682A840DED416BD8
:10D05000014A979BFF1F938BEBD4130C400E7D1B53
:10D0600019A833048A0383A70B0B3E948357C4018A
:10D0700063836705050A97E0FFFFE780A08EE34220
:10D08000AAFE95460DA08357C501639697029305A6
:10D09000050303A50A00414697100100E780802E92
:10D0A000994611E181462686CA854E8597F0FFFF95
:10D0B000E780C06F85A883A50A0013050403977055
:10D0C0000000E780A017C14679FD2285231E940049
:10D0D00097A00000E780E074228597600000E78059
:10D0E00060649797FF1F9387A7029C43A9C32300FF
:10D0F0000402228597D00000E78040F04E858146EB
:10D100002686CA8597F0FFFFE780406AA16793876C
:10D11000070448003EC42302010002C697F0FFFF47
:10D12000E780605741011753FFFF670003F9894704
:10D130002300F402E1B7397106DE22DC4AD8800010
:10D1400052D456D25AD026DA4ED65ECE2E8A3289A4
:10D150002A8B97D0FFFFE780E07D06057105419996
:10D160008A8A3301A140232224FC231404FC97D093
:10D17000FFFFE780207C83479A000605350593F77B
:10D18000F7072315A4FCA304FA004A85232624FCF0
:10D1900097E0FFFFE780407993170501C18763405F
:10D1A000F0025681130104FCF2506254D2544259E9
:10D1B000B259225A925A025BF24B21618280AA84B0
:10D1C0004A8597E0FFFFE7802076AA894A8597E0A5
:10D1D000FFFFE7806075A1659385C5022A89130565
:10D1E00044FC97C0FFFFE780A07F268597C0FFFF24
:10D1F000E780E073854511C94A86CE8597C0FFFF59
:10D20000E780606DAA8B21E98945130544FC97E00E
:10D21000FFFFE780A061A685130544FC97E0FFFFB0
:10D22000E780C062CE85130544FC97E0FFFFE780EE
:10D23000E061CA85130544FC97E0FFFFE7800061C9
:10D2400001478146130644FCD2855A8597D0FFFFDB
:10D25000E780609EB9B78145130544FC97E0FFFF66
:10D26000E780C05CA685130544FC97E0FFFFE780DC
:10D27000E05DCE85130544FC97E0FFFFE780005D8D
:10D28000CA85130544FC97E0FFFFE780205C8144DA
:10D2900097D0FFFFE780006AE3D4A4FA83A70B01CD
:10D2A00013971400BA9783D5070099C5130544FC5A
:10D2B00097E0FFFFE78080598504D9BF797106D6D2
:10D2C00022D44AD000184ECE52CC56CA26D25AC8C2
:10D2D000AE893289AA8A97D0FFFFE780A06506054C
:10D2E000690541990A8A3301A140232A24FC231CA1
:10D2F00004FC97D0FFFFE780E06383C79900060531
:10D300002D0593F7F707231DA4FCA384F9004A8594
:10D31000232E24FC97E0FFFFE780006193170501AF
:10D32000C187634FF0005281130104FDB2502254B3
:10D3300092540259F249624AD24A424B4561828074
:10D34000AA844A8597E0FFFFE780005EA165938588
:10D35000A5022A89130544FD97C0FFFFE7804068B6
:10D36000268597C0FFFFE780805C854509C9CA858F
:10D3700097C0FFFFE78020592A8B29E189451305D3
:10D3800044FD97E0FFFFE780604AA685130544FD52
:10D3900097E0FFFFE780804BCA85130544FD97E0C7
:10D3A000FFFFE780A04A01478146130644FDCE8572
:10D3B000568597D0FFFFE7800088B5B781451305F4
:10D3C00044FD97E0FFFFE7806046A685130544FD16
:10D3D00097E0FFFFE7808047CA85130544FD97E08B
:10D3E000FFFFE780A046814497D0FFFFE78080548D
:10D3F000E3DBA4FA83270B0113971400BA9783D5B4
:10D40000070099C5130544FD97E0FFFFE78000443E
:10D410008504D9BF1753FFFFE70223C9834745009F
:10D42000404DD5EFFD575DC48346940009476363C3
:10D43000D70A0346B400854663EEC6088306E400B7
:10D4400063CA06085C45F9562390D7009787FF1FEB
:10D4500083C7477599E3A304E4009787FF1F938769
:10D46000A77C9C4381E78947A306F4009797FF1F99
:10D47000938707CA9C4381E789472306F4009705F1
:10D48000000093854506AA841305040197F0000067
:10D49000E7802010FD57231AF40281471CDC014865
:10D4A0009787FF1F23AC876E9787FF1F9387476F70
:10D4B000232E040304C0804397D0FFFFE780C051B0
:10D4C00061463306C502814522859750FFFFE780FC
:10D4D000C0C081473E851753FFFF670043BFFD571C
:10D4E000D5BF1753FFFFE70243BC2A84035545020B
:10D4F00097600000E780E01D19E5231E0400175324
:10D50000FFFF6700C3BC8357E401F5DB930504FF0D
:10D51000174501001305452197E00000E780E0145E
:10D52000F9BF1753FFFFE70243B82E89A1654111E8
:10D530009385E5032A8436C432C6BE843AC297C0B6
:10D54000FFFFE780E04912472285BA8597E0FFFF99
:10D55000E780C02D32462285B28597E0FFFFE78045
:10D56000E02EA2462285B68597E0FFFFE780002ED9
:10D57000630309029145228597E0FFFFE780C024FD
:10D580001146A68597100100E78020E2410117535C
:10D59000FFFF6700C3B38945228597E0FFFFE7805F
:10D5A000A02283C704002300F50083C71400A30052
:10D5B000F500E9BF1753FFFFE70223AF83C79500CC
:10D5C000444D054793F7F707A384F5001C4241112A
:10D5D00083C707006367F7062E842A89B1C003C793
:10D5E000D400630FF7021787FF1F1307E763184381
:10D5F00005C3A386F40097A00000E780404A83C7D4
:10D60000D40099E741657D1597400000E7804030E0
:10D6100083D72403918B89C797E00000E780C0136C
:10D620004A85A28597F0FFFFE7808010A167C107B8
:10D6300048003EC42302010002C697F0FFFFE780C6
:10D64000800541011753FFFF670063A81753FFFFD1
:10D65000E702A3A503D745008D47AA8441112E8474
:10D6600032892E8563E3E70297E0FFFFE780C02B56
:10D67000AA8523000900268597C0FFFFE780A02820
:10D6800041011753FFFF670083A497E0FFFFE78086
:10D69000A0292AC6228597E0FFFFE780E028B2454F
:10D6A00085472A862300F900268597C0FFFFE7807B
:10D6B0008022F9B7397106DE22DC26DA80004ED6E8
:10D6C00052D456D24AD85AD05ECEAE89B284AA8AF3
:10D6D00097D0FFFFE7800025060513052502419935
:10D6E0000A8A3301A140232224FC231404FC97D08E
:10D6F000FFFFE780202383C7990006054D0593F7B8
:10D70000F7072315A4FCA384F9002685232624FC0F
:10D7100097E0FFFFE780402193170501C187634031
:10D72000F0025281130104FCF2506254D254425967
:10D73000B259225A925A025BF24B21618280AA8B23
:10D7400003AB040097C0FFFFE780601E51E583D75D
:10D75000440001498544F11793B71700A301F4FC75
:10D76000834734FCA165C9C79385E504130544FCD0
:10D7700097C0FFFFE780C026A685130544FC97E00D
:10D78000FFFFE780A00ADE85130544FC97E0FFFF5A
:10D79000E780C00B834734FC114691E30946DA85E4
:10D7A000130544FC97E0FFFFE78060058144630AAE
:10D7B0000900416B7D1B97D0FFFFE780A01663CC6B
:10D7C000A40201478146130644FCCE85568597C0C6
:10D7D000FFFFE7804046B1B7A685130634FC9700EB
:10D7E0000000E780E0E6933415002A8986048DBFA7
:10D7F0009385C504A5BF8327C90013971400BA9762
:10D8000083D5070063886501130544FC97E0FFFF9B
:10D81000E780C003850445B71753FFFFE70263861F
:10D8200079711C103EC4B7070F003EC61C103EC8DD
:10D8300083C79500AA8A328593F7F707A384F5007A
:10D84000AE89328497E0FFFFE780000E9317050151
:10D85000C187635AF0062A8A228597E0FFFFE78096
:10D86000A00C2A895285032B040097C0FFFFE78094
:10D87000000C39ED8357440081440544F11793B7F8
:10D880001700A303F10083457100DA872287CA8657
:10D890005286280097000000E780E0C801478146D3
:10D8A0003000CE85568597C0FFFFE780C038A1675E
:10D8B0009387D70348083ECC230A810026CE97F0F1
:10D8C000FFFFE78040DD45611743FFFF6700E37E10
:10D8D000A2851306710097000000E78060D7AA8434
:10D8E000094455D13544E30055FB4A8597F0FFFFC5
:10D8F000E78000450D4441D9014497D0FFFFE78000
:10D900006002634DA400C16B0144FD1B97D0FFFF73
:10D91000E7804001634EA4001544B5B7DC441317FB
:10D920001400BA9783D70700638327030504F1B770
:10D93000D84493171400BA9703D70700631B7701E5
:10D9400023902701268597A00000E78080DB014413
:10D950001DBF050465BF1743FFFFE702637383C75D
:10D96000950041112A8A93F7F707A384F5003285C1
:10D970002E89328497E0FFFFE78000FB93170501B3
:10D98000C1876353F006AA89228597E0FFFFE780ED
:10D99000A0F92311A1004E85832A040097C0FFFF40
:10D9A000E780E0F839E58357440085440144F117E6
:10D9B00093B71700A300F10003481100035721009B
:10D9C000D6875285CE862686CA8597F0FFFFE780E8
:10D9D0006006A167F10748003EC42302910022C6F9
:10D9E00097F0FFFFE78020CB41011743FFFF67005F
:10D9F000636DA2851306110097000000E78040C503
:10DA00002A84894455D98357210011678544BA97E0
:10DA1000C2071167C1831307F7EFE36FF7F8978722
:10DA2000FF1F9387A7369C4381CB854513052100B3
:10DA300097500000E780207583552100228581449E
:10DA400097C0FFFFE78040E525D923100500228518
:10DA500097A00000E78040CD85B71743FFFFE7029E
:10DA6000436283C7950041112A8B93F7F707A3847C
:10DA7000F50032852E8A328497E0FFFFE780C0EA06
:10DA800093170501C1876351F006AA8A228597E0A2
:10DA9000FFFFE78060E92A895685832B040097C041
:10DAA000FFFFE780C0E831E5835744008144054427
:10DAB000F11793B71700A301F10003483100DE8787
:10DAC0005A854A87D6862286D28597F0FFFFE7805F
:10DAD00060F6A167ED0748003EC42302810026C618
:10DAE00097F0FFFFE78020BB41011743FFFF67006E
:10DAF000C35CA2851306310097000000E78040B5A3
:10DB0000AA8409445DD99167CA97C2071167C18386
:10DB10001307F7EF0544E362F7FACA8597C0FFFFE2
:10DB2000E78080D7014451F9814997D0FFFFE78012
:10DB300060E063DBA900984893971900BA9703D770
:10DB4000070005EF2390270197D0FFFFE78080DED5
:10DB50001544E384A9F6268597A00000E780C0BCA1
:10DB60009787FF1F938787229C430144B9D74A8533
:10DB700097500000E780C05889B785097DB71743E3
:10DB8000FFFFE702E35079713E847C083EC82E8A8D
:10DB9000B7071400A1653ECAE5057C08AA890808F4
:10DBA00036C4428932C6BA8AC6843ECC97C0FFFFCB
:10DBB000E78000E3CA85080897E0FFFFE78000C719
:10DBC00032460808B28597E0FFFFE78020C8A246EA
:10DBD000630A09049D45080897E0FFFFE780C0BE7F
:10DBE0001D4681459740FFFFE780204F63890A0863
:10DBF0009145080897E0FFFFE78000BD1146A68524
:10DC000097000100E780607A100801478146D285BD
:10DC10004E8597C0FFFFE780000245611743FFFF75
:10DC20006700434AB685080897E0FFFFE78000C217
:10DC30001C400808D8439355C701858912075183B2
:10DC4000B205D98D97E0FFFFE78040C01C4008086F
:10DC500083C5870097E0FFFFE78040BD1C400808B0
:10DC600083C5A70097E0FFFFE78040BC1C40080881
:10DC700083C5970097E0FFFFE78040BB85BF8945DC
:10DC8000080897E0FFFFE78020B483C70400230063
:10DC9000F50083C71400A300F500BDB71743FFFFCD
:10DCA000E702033F83C795004111AA8993F7F7075D
:10DCB000A384F5003285AE84328497E0FFFFE780CD
:10DCC000A0C693170501C187635DF0042A89032A62
:10DCD000040097C0FFFFE78080C519E9835744001F
:10DCE0000548F11793B71700A307F100814631A843
:10DCF0001306F100A28597000000E78060951DC51E
:10DD00001C459DC783D6470001480347F100930790
:10DD10008500D2884A86A6854E8597000000E78058
:10DD200040E641011743FFFF6700C33909487DBF43
:10DD30001D486DBF1743FFFFE702833565715C081F
:10DD40003EC4B7077B013EC65C083EC883C795004A
:10DD50002A8A328593F7F707A384F500AE8997E006
:10DD6000FFFFE78040BA8357E100E1C789452800FB
:10DD700097C0FFFFE780C0C68145280097E0FFFFFE
:10DD8000E780C0AA97C0FFFFE780A0CC9787FF1F5E
:10DD9000938707389C431784FF1F0344A4E0AA8499
:10DDA0003334800099C3136424009787FF1F93873F
:10DDB000A7E79C4399C3136444009787FF1F938789
:10DDC000E7FC9C4399C31364840083D504002800B6
:10DDD000014997E0FFFFE78060A783D52400280072
:10DDE00097E0FFFFE78080A683D54400280097E0F6
:10DDF000FFFFE780A0A597D0FFFFE780A0AE9315B7
:10DE00000501C181280097E0FFFFE78020A4A285DB
:10DE1000280097E0FFFFE78060A39C446360F9025D
:10DE2000014781463000CE85528597C0FFFFE780CD
:10DE300080E059611743FFFF6700C328DC441314D7
:10DE4000490028003E9497E0FFFFE78060968347F3
:10DE500044000347540089070607BA978607E36A18
:10DE6000F5FC835524002800814A97E0FFFFE780F6
:10DE7000E09D83454400280097E0FFFFE780009B7A
:10DE800083455400280097E0FFFFE780209A8347EE
:10DE9000440063C9FA00814A8347540063C1FA020F
:10DEA0000509A5BF1C4413975A002800BA9783D5CB
:10DEB0000700850A97E0FFFFE7804099C9BF032B61
:10DEC000C40093975A0028003E9B83552B00850A77
:10DED00097E0FFFFE780809783550B00280097E0CD
:10DEE000FFFFE780A0964DBF1743FFFFE702E31B4C
:10DEF0005C4993E717005CC997A00000E78020B653
:10DF00001743FFFF6700A31C1743FFFFE702E31956
:10DF10002E84814597F0FFFFE780C0E705C5835752
:10DF20000500FD172310F50009C4835725002310B1
:10DF3000F40097000000E78060FB01451743FFFFF6
:10DF40006700E31831457DD823100400C5BF17438F
:10DF5000FFFFE702E31383C7950041112A8A93F775
:10DF6000F707A384F50032852E89328497E0FFFFFE
:10DF7000E780809B93170501C1876356F006AA8945
:10DF8000C145228597E0FFFFE780A0802A8B4E8560
:10DF9000832A040097C0FFFFE780609931E9835727
:10DFA0004400231101000544F11793B71700A300A3
:10DFB000F10081440348110003572100D6875285A0
:10DFC000CE862286CA8597F0FFFFE780A0A6A167CC
:10DFD0009387170248003EC42302810026C697E0BB
:10DFE000FFFFE780406B41011743FFFF6700830D90
:10DFF00013061100A28597F0FFFFE7806065AA84F1
:10E0000009E523110100094475B7930521005A85DC
:10E0100097000000E78080EF835721002A84D9DB36
:10E020009787FF1F938787D69C4381CB8545130530
:10E03000210097500000E7800015835521002685B8
:10E04000314497C0FFFFE78020852DD523100500C0
:10E05000268597900000E780206D0144A1BF1743FB
:10E06000FFFFE702830441112E896C00AA8402C6D7
:10E0700097F0FFFFE78000D20DC1035705000507A9
:10E080002310E50097000000E78040E681473E85C9
:10E0900041011743FFFF670083033247954765DB64
:10E0A000CA85268597300000E780400DC147E340D0
:10E0B00005FE3244854741462310F400835709008A
:10E0C000A685130544002311F40097000100E780A2
:10E0D000C02D228545BF1743FFFFE70263FB83C7BF
:10E0E00095004111AA8A93F7F707A384F5003285BA
:10E0F000AE89328497E0FFFFE78000839317050124
:10E10000C1876356F0062A8AC145228597D0FFFF52
:10E11000E7802068AA845285032B040097C0FFFF84
:10E12000E780E08031E983574400231101008544F2
:10E13000F11793B71700A300F10001440348110041
:10E1400003572100DA875685D2862686CE8597F03A
:10E15000FFFFE780208EA1679387070248003EC437
:10E160002302910022C697E0FFFFE780C0524101E1
:10E170001743FFFF670003F5A2851306110097F010
:10E18000FFFFE780E04C2A8409E523110100894460
:10E1900075B726859305210097000000E78060ECA5
:10E1A000AA8449FD83552100228597B0FFFFE780AF
:10E1B000A06E49F5014997C0FFFFE780A077635D36
:10E1C000A900184893171900BA9703D707000DEF55
:10E1D000035721002390E70097C0FFFFE780807579
:10E1E000630625039787FF1F938747BA9C4399C708
:10E1F0000355210097500000E78080F0228597901A
:10E200000000E78060521DBF050975B795443DB712
:10E2100005C19307F00F630FF500C547630CF500C8
:10E220009307F5FF05453315F500420541818280CE
:10E230000145828041657D158280B9E91743FFFF62
:10E24000E702A3E603450603328497000000E78057
:10E2500060FC9305803EB305B502C205C18181CD46
:10E260000357E402854763F8E7001305040197E0CC
:10E270000000E78020428357E40241677D176385F1
:10E28000E700FD172317F4021743FFFF670023E49D
:10E2900082801743FFFFE702C3DE004283C7950079
:10E2A000444D0349140093F7F707A384F50083470F
:10E2B0000400220911673369F900A167B347F90027
:10E2C00041112A8BAE8A63ECE70E834724001307C3
:10E2D000C00EB91793F7F70F6373F71003473400B5
:10E2E000C14763EEE70E834744001307E00793C777
:10E2F00007086371F70C8349840083477400A209FF
:10E30000B3E9F900856763F7F90A034A64008347B4
:10E3100054004E85220A336AFA0097500000E780C5
:10E32000403B61C123962403834B3400137AFA00E7
:10E33000239A3403238874032399440393890401A3
:10E34000631C090023A60402239804024E8597E06B
:10E350000000E78060363DA0034924004A8597000D
:10E360000000E78020EB2397A402834744004E85FA
:10E37000A388F402E38D0BFCE30B09FC97E000009B
:10E38000E780202F97900000E780007381460146C8
:10E39000D6855A8597E0FFFFE7800058A1679387ED
:10E3A00097033EC423020100480002C697E0FFFF26
:10E3B000E780602E41011743FFFF670003D08544CB
:10E3C000A2862686D6855A8597E0FFFFE780C0544F
:10E3D000A167938797033EC423029100F1B7BD4420
:10E3E000C5B79144F1BF1743FFFFE70263CA0111AC
:10E3F0001C08404D3EC2B7070F003EC41C083EC675
:10E400002A89AE8997C0FFFFE780A0DA585C1C5CC0
:10E410006346B70E6394E50063E2A70E3385A74019
:10E42000B3B7A700B305B7401306803E81469D8D64
:10E4300097000100E78080B793140501C180A165B2
:10E440009385C503480097B0FFFFE7806059814579
:10E45000480097D0FFFFE780603D835504044800E3
:10E4600097D0FFFFE780803E83552404480097D073
:10E47000FFFFE780A03D814589CCC167FD1793056B
:10E48000F00F6388F400268597500000E780E0E0F5
:10E49000AA85480097D0FFFFE78040390355440420
:10E4A000814501CDC167FD179305F00F6307F500A6
:10E4B00097500000E78060DEAA85480097D0FFFFF4
:10E4C000E780C03683456404480097D0FFFFE780AB
:10E4D000E03583457404480097D0FFFFE78000359E
:10E4E000500001478146CE854A8597B0FFFFE780FF
:10E4F000807405611743FFFF6700C3BC814481B787
:10E500001743FFFFE70263BA83C7950093F7F70746
:10E51000A384F50097000000E78020ED1743FFFF7C
:10E520006700E3BA1743FFFFE70283B683C795008E
:10E530004111404D93F7F707A384F5002A8A3285ED
:10E54000B284AE8997D0FFFFE780003E2A8B2685F4
:10E5500097D0FFFFE780403D2A89268597D0FFFFAF
:10E56000E780603A93170B0163CA0702E177CA9705
:10E57000C207C183116763E3E70293070910C2076B
:10E58000C1831307B00F637BF70093170901C1879D
:10E59000AA8A634AF000C54763FE57014101174349
:10E5A000FFFF670023B297B0FFFFE780C028E317A3
:10E5B00025FFD5B763080B0263060902814463890E
:10E5C0000A02B7077F0023106405231124057CC0CD
:10E5D000568597000000E780E0C39304803EB304B3
:10E5E000950239A0B7077F00232004047CC0814432
:10E5F0000355240497E00000E780A0A3A1C497C0BE
:10E60000FFFFE78000BB269593D7F4413337950091
:10E61000AE97BA9708DC5CDCCE8552859700000087
:10E62000E780A0DC99E023220404A1679387B70365
:10E6300048003EC42302010002C697E0FFFFE780C6
:10E640008005A9BF814701481CDC232E0403E9B7DC
:10E650001743FFFFE70263A597C0FFFFE780C037BE
:10E66000E1473305F502914597500000E78000C56A
:10E67000E55711C59777FF1F23A4A75281473E8511
:10E680001743FFFF6700A3A485471777FF1F230BDE
:10E69000F75082801743FFFFE70223A19777FF1F00
:10E6A0009387C74F80433DC0835704046390A706F8
:10E6B00083572404639CB7043689B28497C0FFFF54
:10E6C000E78020AF5C5C63C3B7046395B7001C5C54
:10E6D00063EEA7028347640463F3F400A687230371
:10E6E000F4048347740463F39700A687A303F40438
:10E6F0008357440441677D176385E700850723122C
:10E70000F4043C4481C7CA85268582971743FFFFDE
:10E710006700E39B9777FF1F938747489C4301451A
:10E7200099C303C5870082801743FFFFE702E39781
:10E730000111B70707003EC683C79500584D0AC4AC
:10E7400093F7F7070AC8A384F5002A89AE8411CB92
:10E750001C4283C707002304F70097900000E7805E
:10E760000034216493055402280097B0FFFFE7802E
:10E77000202797000000E78020FAAA85280097D07C
:10E78000FFFFE780A00A300001478146A6854A8541
:10E7900097B0FFFFE780204A13044402480822CCC8
:10E7A000230A010002CE97E0FFFFE780C0EE05617B
:10E7B0001743FFFF6700A3911743FFFFE702E38EB4
:10E7C00001117C003ECAB70707003ECC7C003ECE5C
:10E7D00083C795002E84AA8493F7F707A384F500D6
:10E7E000A16593855502480897B0FFFFE780401F59
:10E7F00097000000E78040F2AA85480897D0FFFF05
:10E80000E780C002500801478146A285268597B05F
:10E81000FFFFE780404205611743FFFF6700238B3E
:10E820009777FF1F938787379C43094599C303C593
:10E83000970082809777FF1F938747369C4309454F
:10E8400099C303C5D70082809777FF1F9387073549
:10E850009C43014599C303C5A70082801743FFFF6E
:10E86000E70203830111B70708003EC683C795007E
:10E87000404D0AC493F7F7070AC8A384F5002A8914
:10E88000AE8429C41442854703C7060063E0E70A43
:10E8900083479400094681496380C702B307F74064
:10E8A000A304E400B339F00083C716002305F40085
:10E8B00097900000E780A01E03572403058B19C71B
:10E8C0006386090097D00000E78000E92164930582
:10E8D0008402280097B0FFFFE780801097000000B7
:10E8E000E78040F4AA85280097D0FFFFE78000F476
:10E8F00097000000E78080F5AA85280097D0FFFFE9
:10E90000E780C0F2014781463000A6854A8597B06E
:10E91000FFFFE780403213047402480822CC230A28
:10E92000010002CE97E0FFFFE780E0D605611733D4
:10E93000FFFF670023791733FFFFE7020377011119
:10E940007C003ECAB70708003ECC7C003ECE83C7A1
:10E9500095002E84AA8493F7F707A384F500A16598
:10E9600093858502480897B0FFFFE780600797000E
:10E970000000E78020EBAA85480897D0FFFFE780DA
:10E98000E0EA97000000E78060ECAA85480897D08D
:10E99000FFFFE780A0E9500801478146A285268550
:10E9A00097B0FFFFE780202905611733FFFF67005D
:10E9B00003729777FF1F9387671E9C43014599C396
:10E9C00003C5B70082801733FFFFE702036E011112
:10E9D000B70707003EC683C79500404D0AC493F7AA
:10E9E000F7070AC8A384F5002A89AE8405C81C422B
:10E9F000054783C707006368F7060347B400630F42
:10EA0000F700A305F40097900000E78040098347D2
:10EA1000B400B9CF97D0FFFFE78040BE21649305D3
:10EA2000B400280097B0FFFFE78080FB970000004C
:10EA3000E78060F8AA85280097D0FFFFE78000DF15
:10EA4000014781463000A6854A8597B0FFFFE780E1
:10EA5000801E2904480822CC230A010002CE97E038
:10EA6000FFFFE78040C305611733FFFF67002366A0
:10EA700097D0FFFFE78020BF55B71733FFFFE702AE
:10EA8000C36201117C003ECAB70707003ECC7C0080
:10EA90003ECE83C795002E84AA8493F7F707A384FC
:10EAA000F500A165AD05480897B0FFFFE78040F38A
:10EAB00097000000E78020F0AA85480897D0FFFF64
:10EAC000E780C0D6500801478146A285268597B0C9
:10EAD000FFFFE780401605611733FFFF6700235FE4
:10EAE0009777FF1F9387870B9C43094599C303C5FD
:10EAF000C70082801733FFFFE702235B01117C0010
:10EB0000AE843ECAA165B70707002A843ECCD10572
:10EB10007C0048083ECE97B0FFFFE78060EC97008E
:10EB20000000E78020FCAA85480897D0FFFFE78017
:10EB3000E0CF500801478146A685228597B0FFFFA8
:10EB4000E780600F05611733FFFF670043581733F5
:10EB5000FFFFE702835583C7950093F7F707A38468
:10EB6000F50097000000E78020F91733FFFF6700EA
:10EB700003561733FFFFE702A35183C7950003290C
:10EB8000C501411193F7F707A384F5001C4283C91F
:10EB90000700854763E637079777FF1F9387475737
:10EBA0009C432E84AA8485CF97000000E78080F3E1
:10EBB00089476306F502630409028347C90063803D
:10EBC00037032306390197900000E78040ED835713
:10EBD0002903898B89C797D00000E780E0B7268595
:10EBE000A28597000000E78020F1A167CD074800CB
:10EBF0003EC42302010002C697E0FFFFE780A0A900
:10EC000041011733FFFF6700E34B9777FF1F93879F
:10EC1000E7F89C431D4599C303C5E700828017337D
:10EC2000FFFFE70283480111B70707003EC683C70D
:10EC30009500584D0AC493F7F7070AC8A384F50056
:10EC40002A89AE8415C71C4283C7070093968701A3
:10EC5000E18663C4060685466381D7068346E700DE
:10EC60006388F6002307F70097900000E78020E311
:10EC700021649305E400280097B0FFFFE78040D6A9
:10EC800097000000E780A0F8AA85280097D0FFFF32
:10EC9000E780C0B9014781463000A6854A8597B014
:10ECA000FFFFE78040F93504480822CC230A010021
:10ECB00002CE97E0FFFFE780009E05611733FFFF5C
:10ECC0006700E3401733FFFFE702233E01117C009A
:10ECD0003ECAB70707003ECC7C003ECE83C79500F6
:10ECE0002E84AA8493F7F707A384F500A165B905DC
:10ECF000480897B0FFFFE780A0CE97000000E780AC
:10ED000000F1AA85480897D0FFFFE78020B250089D
:10ED100001478146A285268597B0FFFFE780A0F1D5
:10ED200005611733FFFF6700833A1733FFFFE702E0
:10ED30002336AA8401441779FF1F130969E6E149C4
:10ED400097C0FFFFE78040C96344A400014519A8AC
:10ED500033053403832709003E95835725006397C5
:10ED6000970011051733FFFF6700C3350504C9BFBE
:10ED7000032E8500630A0E121773FF1F130303018E
:10ED80000323030063150300294363900612032342
:10ED90004E01631503001D43639907101733FFFFEE
:10EDA000E702232EC689428A3E89BA8AB684328B0C
:10EDB000AE8B2A84B5E103554E0019E501431A854F
:10EDC0001733FFFF6700632FA167A98F116763FBEC
:10EDD000E70097000000E78080F5814597F0FFFF8E
:10EDE000E780C0120844B70700E05841F98F184582
:10EDF0005CC1B707001FF98F1CC55C4991C761054D
:10EE000097E00000E780408BE38A09FA228597901B
:10EE10000000E78060C65DB7328597C00000E780DC
:10EE200040430D4349DD1C44116703D54700A167EA
:10EE3000A98F63FBE70097000000E78040EF814562
:10EE400097F0FFFFE780800C0323840093164B01AB
:10EE5000D1828347B300035663008588FD8BA305E9
:10EE6000F300FD777D8E558EFD76FD16B204F18E92
:10EE700083274301C58E231273012313D300230478
:10EE8000530123052301A3044301BDDF228597B06D
:10EE9000FFFFE78020CDAA850844B5D1610597D052
:10EEA0000000E780207F8DB71D431A8582801733CD
:10EEB000FFFFE702E31D0569AA84AE89328A014497
:10EEC000FD5A7D1997C0FFFFE780C0A56347A400E6
:10EED00001451733FFFF6700E31ED8449317140062
:10EEE000BA9703D70700631F3703239057016307BF
:10EEF0000A00268597900000E780A0809C449DC36F
:10EF000083D76700B3F72701639E3701D288014892
:10EF100081470147814601468145268597000000CB
:10EF2000E78040E5050479BF1733FFFFE70243168A
:10EF300079711C103EC4B7070F003EC61C103EC8B6
:10EF400083C79500AA8A328593F7F707A384F50053
:10EF50002E89328497D0FFFFE780009D931705012B
:10EF6000C187635AF006AA89228597D0FFFFE78000
:10EF7000A09B2A8A4E85032B040097B0FFFFE780F1
:10EF8000009B39ED8357440081440544F11793B742
:10EF90001700A303F10083457100DA872287D28628
:10EFA0004E86280097E0FFFFE780E0570147814643
:10EFB0003000CA85568597B0FFFFE780C0C7A167BC
:10EFC0009387F70348083ECC230A810026CE97D0CA
:10EFD000FFFFE780406C45611733FFFF6700830E3A
:10EFE000A2851306710097E0FFFFE7806066AA84A0
:10EFF000094455D1528597E0FFFFE78060D40D4466
:10F0000059D90546D285268597000000E78060EA39
:10F010002A8451B71733FFFFE702230983550700FE
:10F020000346270041112A842E8532C62EC497E05C
:10F03000FFFFE780E0D001C93246A2452285970054
:10F040000000E78000E741011733FFFF6700230856
:10F050001733FFFFE702E30283C795004111AA8A35
:10F0600093F7F707A384F5003285AE89328497D0F1
:10F07000FFFFE780608B93170501C1876357F00A94
:10F08000C1452A8A228597C0FFFFE78080702A8DBC
:10F09000228597D0FFFFE78020892A89228597D093
:10F0A000FFFFE7804086930705F893F7F70F1307F4
:10F0B000E007AA8B637BF706228597D0FFFFE780E6
:10F0C00080842A8C228597D0FFFFE780C083AA8C9A
:10F0D0005285032B040097B0FFFFE780408539E994
:10F0E00083574400231101008144F11793B717009F
:10F0F000A300F100054403471100835621009387C4
:10F1000084005685DA8822885286CE8597F0FFFFE4
:10F11000E78020A7A167E90748003EC423028100D9
:10F1200026C697D0FFFFE780005741011733FFFF46
:10F130006700A3F813061100A28597E0FFFFE780A0
:10F140002051AA8409E52311010009446DB79305F4
:10F1500021006A8597F0FFFFE780A0F02A8441FD37
:10F16000835521009356C9001316490185486688C6
:10F17000E2875E87858A5182268597000000E780B6
:10F1800060BF2A848DBF1733FFFFE70283EF83C779
:10F19000950041112A8B93F7F707A384F500328578
:10F1A000AE89328497C0FFFFE7800078931705018E
:10F1B000C1876352F00A2A8A228597C0FFFFE78041
:10F1C000A076AA8A228597C0FFFFE780E0752A898A
:10F1D000228597C0FFFFE7800073930705F893F738
:10F1E000F70F1307E0072A8C6377F706228597C08D
:10F1F000FFFFE7804071AA8C228597C0FFFFE78060
:10F2000080702A8D5285832B040097A0FFFFE78032
:10F21000007239E58357440085440144F11793B7E0
:10F220001700A301F10003473100930784005A85BA
:10F23000DE882688D6865286CE8597F0FFFFE78047
:10F2400040948D4748003EC42302910022C697D0C7
:10F25000FFFFE780404441011733FFFF6700E3E50C
:10F26000A2851306310097E0FFFFE780603E2A8405
:10F27000894455D99356C9001316490185486A88AF
:10F28000E6876287858A5182D68597000000E780ED
:10F2900060AEAA8449BF1733FFFFE70263DF2A8904
:10F2A00081440144617A916A177BFF1F130B0BAEF7
:10F2B00097B0FFFFE780006863C7A400228517337B
:10F2C000FFFF670023E08327090093991400CE977E
:10F2D00003D50700330745014207418363645703A1
:10F2E00005C103270B0019C785453E8597400000DF
:10F2F000E78060E9832709000504CE972390070083
:10F3000085047DB797000000E78060A2832709008D
:10F310000504CE972390070065D5814597F0FFFF40
:10F32000E780C0BEF1BF1733FFFFE70263D683C794
:10F33000950041112A8A93F7F707A384F5003285D7
:10F340002E89328497C0FFFFE780005E9317050186
:10F35000C187635AF004AA89832A040097A0FFFF9B
:10F36000E780E05C31E58357440085440144F117B0
:10F3700093B71700A301F10003483100D6875285E7
:10F380000147CE862686CA8597D0FFFFE780806A30
:10F39000A167F50748003EC42302910022C697D01A
:10F3A000FFFFE780402F41011733FFFF670083D144
:10F3B000A2851306310097E0FFFFE78060292A84C9
:10F3C00089445DD99777FF1F9387479C9C4381CFE2
:10F3D000044997B0FFFFE780E055AA85268597404E
:10F3E0000000E78040DA1305040197000000E78081
:10F3F000C0EA228597800000E78000338144ADBFDA
:10F400001733FFFFE702E3C783C795004111AA8ABC
:10F4100093F7F707A384F5003285AE893284231170
:10F42000010097C0FFFFE780205093170501C187B7
:10F430006354F0062A8AC145228597C0FFFFE78002
:10F440004035AA8B5285032B040097A0FFFFE7806D
:10F45000004E21E98357440085440144F11793B7D6
:10F460001700A300F1000348110003572100DA87B9
:10F470005685D2862686CE8597D0FFFFE780805BB3
:10F48000A1679387270248003EC42302910022C649
:10F4900097D0FFFFE780202041011733FFFF67006F
:10F4A000C3C1A2851306110097E0FFFFE780401A51
:10F4B0002A8489444DD99777FF1F9387278D9843D6
:10F4C0003E8901CF044997B0FFFFE780A046AA8597
:10F4D000268597400000E78000CB130504019700C4
:10F4E0000000E78080DB97B0FFFFE780A0449544F1
:10F4F0003DD9930521005E8597F0FFFFE78060B658
:10F50000AA8435F11C480357210022852390E70087
:10F5100097800000E780402183270900A9D7035581
:10F52000210097400000E780A0BD35BF1733FFFFE3
:10F53000E70223B583C795004111AA8A93F7F7071D
:10F54000A384F5003285AE89328497C0FFFFE7803F
:10F55000A03D93170501C1876351F0062A8A2285D1
:10F5600097C0FFFFE780403C2A895285032B0400A7
:10F5700097A0FFFFE780A03B31E583574400854417
:10F580000144F11793B71700A301F10003483100BC
:10F59000DA8756854A87D2862686CE8597D0FFFFA2
:10F5A000E7804049A167F90748003EC42302910063
:10F5B00022C697D0FFFFE780000E41011733FFFFFF
:10F5C0006700A3AFA2851306310097E0FFFFE78035
:10F5D00020082A8489445DD99167CA97C2071167B8
:10F5E000C1831307F7EF8544E362F7FA9767FF1FBC
:10F5F0009387C7799843BE8B01CF044997B0FFFF2B
:10F60000E7804033AA85268597400000E780A0B7B1
:10F610001305040197000000E78020C897B0FFFFA2
:10F62000E780403195443DD11C4822858144239098
:10F63000270197800000E780200F83A70B00B9D730
:10F640004A8597400000E780A0AB89B71733FFFFDA
:10F65000E702A3A52A844105B28497000000E78051
:10F66000C0C311C5228597800000E780E00B81466A
:10F670000146A685228597800000E780C04E1C4C7D
:10F6800089C7DC4799C3228582971733FFFF67003C
:10F6900003A49767FF1F938767509C43014599C355
:10F6A0001385070182809767FF1F9387274F884341
:10F6B00082801733FFFFE702439F9317C600DD8D5B
:10F6C000C2054111C1812A8432C697C0FFFFE7807D
:10F6D000E0173246228511829375F60F97C0FFFF1F
:10F6E000E780C01441011733FFFF6700439E1733C3
:10F6F000FFFFE702E39979713C083ED2B7070C009F
:10F700003ED43C083ED683C79500AE842A8993F741
:10F71000F707A384F500A16593853504481097A0E9
:10F72000FFFFE780E02BC165FD150144176AFF1F4D
:10F73000130A4A67930A400EAE892E8B2EC697B0E5
:10F74000FFFFE78020224205931704014181C18316
:10F75000B24563E9A702C167FD176387F50048104A
:10F7600097C0FFFFE780800E501001478146A685B5
:10F770004A8597A0FFFFE780004C45611733FFFFE4
:10F78000670043943307540383270A0BBA9703D6C1
:10F79000C701630A3601638A3501481097000000EB
:10F7A000E78060F1DA85050451BFB285EDBF1733FC
:10F7B000FFFFE702038D79717C083EC8B70711008F
:10F7C0003ECA7C083ECC83C79500AA89328593F750
:10F7D000F707A384F5002E8997C0FFFFE780C014C8
:10F7E00085676378F504A165AA848905080897A050
:10F7F000FFFFE780E01E268597400000E78060ED70
:10F80000133415000A04A285080897C0FFFFE7809B
:10F81000E001A685080897C0FFFFE780200325CCFC
:10F82000014781461008CA854E8597A0FFFFE780F3
:10F83000804045611733FFFF67002388B3075403F7
:10F840000327CA0ABA9703D70700631C970003D699
:10F85000270063806505080897000000E780A0E5A1
:10F86000DE8505042EC697B0FFFFE780A010420595
:10F87000931704014181C183B245E3E1A7FCC1674D
:10F88000FD17E38FF5F8080897C0FFFFE78000FC3D
:10F8900041BFB285F9B7C165FD150144176AFF1F65
:10F8A000130A4A50930A80022E8BAE8B65BF172332
:10F8B000FFFFE702837F1841834717008346070055
:10F8C000A207D58FD207D1832390F5008347270065
:10F8D000034717008D45A207D98F91832310F600A7
:10F8E00097C0FFFFE780A0E91723FFFF6700237E93
:10F8F0001723FFFFE702C379C16401441769FF1FA3
:10F900001309494A93098002FD1497B0FFFFE7806D
:10F9100060066347A40001451723FFFF6700837A51
:10F92000330534038327C90A3E9583570500E385D1
:10F9300097FE0504D9BF1723FFFFE70263752A8AE4
:10F94000AE89B284B68A97400000E78080D819E576
:10F9500091473E851723FFFF6700C3762A894E85AE
:10F9600097C00000E780E08E2A84638E0A048D47EA
:10F970006DD103570500C547E31D47FD0347F90156
:10F980008546AD47E317D7FC8347450081CF414605
:10F99000A6855D0597F00000E780C09E814755D998
:10F9A000AD4745BF130965012302E500CA852685D9
:10F9B00097100000E780606231C1A547E38B0AF829
:10F9C0002302040079B705C183570500E39247F984
:10F9D0004146A685190597F00000E780A09A814767
:10F9E0002DD99947BDB74E8597000000E78080F07C
:10F9F0002A84954739DD130955004DBF4146A68538
:10FA000023104401231134011305190097F000005D
:10FA1000E780A099228597800000E780A0EA8147CF
:10FA20000DBF1723FFFFE702436879717C003ECCCE
:10FA3000B7070A003ECE7C003ED083C79500B28453
:10FA40002E8493F7F707A384F5001306A1002A89F3
:10FA50002C00268597000000E780A0E5A165280816
:10FA60008D0597A0FFFFE780A0F790408355A10088
:10FA700003558100854697000000E78000ECAA84CA
:10FA8000AA85280897C0FFFFE78040DA0356A10047
:10FA900083558100280897000000E780C0C1300826
:10FAA00001478146A2854A8597A0FFFFE780A018FD
:10FAB000854748103ED42302910202D697D0FFFF1B
:10FAC000E78060BD45611723FFFF67004360172390
:10FAD000FFFFE702835D79717C003ECCB7070A0027
:10FAE0003ECE7C003ED083C79500B2842E8493F72F
:10FAF000F707A384F5001306A1002A892C002685A8
:10FB000097000000E780E0DAA16528088D0597A03E
:10FB1000FFFFE780E0EC90408355A1000355810092
:10FB2000814697000000E78040E1AA84AA85280862
:10FB300097C0FFFFE78080CF0356A1008355810067
:10FB4000280897000000E78000B730080147814689
:10FB5000A2854A8597A0FFFFE780E00D48102302A9
:10FB6000910202D402D697D0FFFFE780C0B2456170
:10FB70001723FFFF6700A3551723FFFFE702E35298
:10FB800097000000E78060DB1723FFFF6700235426
:10FB90009767FF1F9387C700884382801723FFFF63
:10FBA000E702A350835725004111AE842A8423071E
:10FBB000B10017F5FFFF130525466C002316F10071
:10FBC00097A0FFFFE780204991C42285978000001D
:10FBD000E780E0D6FD572310F4001306200281458C
:10FBE000130554009720FFFFE780204F41011723A2
:10FBF000FFFF6700C34D1723FFFFE70263497971D9
:10FC00007C003ECCB7070A003ECE7C003ED083C7C6
:10FC10009500AA89AE8493F7F7073285A384F5008F
:10FC20001306A1002C0097000000E78080C8035550
:10FC30008100114497400000E780A0A915C5035535
:10FC4000A100014497B00000E780A06011CD0357E8
:10FC500005008357810045446318F70085459700E8
:10FC60000000E780E0F3014421699305390028088A
:10FC700097A0FFFFE780C0D6A285280897C0FFFFA6
:10FC8000E780C0BA0356A100835581002808970079
:10FC90000000E78040A2300801478146A6854E85D6
:10FCA00097A0FFFFE78020F948104AD42302810281
:10FCB00002D697D0FFFFE780009E45611723FFFF24
:10FCC000670043401723FFFFE702833C9767FF1F4E
:10FCD0009387C7EC2A8488432E8915C503574503AB
:10FCE0008357C4016311F702232605022318050276
:10FCF000410597D00000E780209C630609009780AB
:10FD00000000E78060DB81449769FF1F93898909C0
:10FD1000130A800297B0FFFFE780C0C563C4A40444
:10FD20009767FF1F938747F09C4399C70355C4010A
:10FD300097200000E780C0BD6307090022859780F7
:10FD40000000E780C0A01306400E81452285972061
:10FD5000FFFFE7808038FD57231EF4001723FFFFC5
:10FD6000670043363385440383A7C90A3E9503578A
:10FD700005008357C4016317F700CA859700000088
:10FD8000E78000E2850479B71723FFFFE7024330DD
:10FD900083C795004111AA8993F7F707A384F5005B
:10FDA0003285AE8497C0FFFFE78000B8856763782F
:10FDB000F5042A8997400000E780A091014401CD15
:10FDC00083D70400314463882701854597000000EC
:10FDD000E78080EF01444E85A2864A86A68597D0AB
:10FDE000FFFFE780A09CA1679387170448003EC4EB
:10FDF0002302810002C697D0FFFFE780C08941013E
:10FE00001723FFFF6700032C1723FFFFE702432898
:10FE10009767FF1F938787D8804329C4014597C000
:10FE20000000E780002181470148C1641CDC232ECB
:10FE30000403232004041769FF1F1309A9F60144D2
:10FE40009309400EFD1497B0FFFFE780A0B1634F08
:10FE5000A400814517F5FFFF1305857F97A0FFFFDD
:10FE6000E780601F1723FFFF6700C32533053403B6
:10FE70008327090B3E958357C50163879700854506
:10FE800097000000E78040E4050475BF9357050123
:10FE900013D78700A380F50093170501C183A183C1
:10FEA0002380E5002381F500A381A500828017232C
:10FEB000FFFFE702831F2300050083C71500A3008F
:10FEC000F50083C725002301F50083C73500A30192
:10FED000F50083C745002302F50083C75500A30240
:10FEE000F50083C7650093059500A3030500230370
:10FEF000F50023040500328597000000E78040F9F3
:10FF00001723FFFF6700A31C1723FFFFE702431817
:10FF10004111E9540DCD85CD93F9C5FF2E842A8971
:10FF2000AA84338AA900B7EA040063189A020D88EC
:10FF3000854411CCB7E704009C5F82972AC62286CD
:10FF40006C003305390197E00000E7800046268504
:10FF500041011723FFFF6700E31683A78A0391047B
:10FF6000829793170501C183A183A38EF4FE935753
:10FF70000501238FF4FEA183238EA4FEA38FF4FE3C
:10FF80006DB763E6D5021723FFFFE7020312B287BE
:10FF900041113686BE8536C697E00000E780E04016
:10FFA000B246410136851723FFFF670043128146A1
:10FFB00036858280838705001387F5003D05FD8720
:10FFC00093F77708834607007D158606B58FA30053
:10FFD000F5006307B7007D17834717009D83DDB7E2
:10FFE00082801723FFFFE702430CB7E7040083A7D3
:10FFF000070932872A863A85829713351500172319
:020000040001F9
:10000000FFFF6700C30C15C181478DC11723FFFF98
:10001000E702A309414697E00000E78000398547E1
:100020003E851723FFFF6700830A81473E85828054
:100030001DCD1723FFFFE7024307414681452A8470
:100040009720FFFFE78060094146814513050403BF
:100050009720FFFFE78060080147C167232204045F
:1000600038C87CC805451723FFFF670043060145D4
:10007000828081473DCDB5CD1723FFFFE702E30224
:10008000B2842E891306800581452A849720FFFFBC
:10009000E780A004CA8524C4268597000000E78075
:1000A000C0F64146814522859720FFFFE780E002A8
:1000B0003044A285228597000000E780C0F29304B7
:1000C0000401A285268597000000E780E0EEA68562
:1000D0001305040297000000E78000EE22859700D8
:1000E0000000E78020F585473E851723FFFF670066
:1000F00003FE3E8582801723FFFFE70263F941116B
:10010000E9540DCD85CD93F9C5FF2E842A89AA84A3
:10011000338AA900B7EA0400639844030D88814438
:1001200011CCB7E704009C5F82972AC622866C0038
:100130003305390197E00000E7802027268541013B
:100140001723FFFF670003F883A78A0391048297B0
:1001500093170501C183A183A38EF4FE9357050174
:10016000238FF4FEA183238EA4FEA38FF4FE6DB72C
:1001700065CD1723FFFFE702A3F1B28411E6054521
:100180001723FFFF670003F42A842E890145EDD968
:100190003C487848B3E6E700E5D69386F7FFB3B767
:1001A000F6007D17032A4404BA9734C87CC8630557
:1001B0000A06C14913050A03B38949412295637DA3
:1001C0003601B2862E86A68597000000E780A0DB68
:1001D0007C40BE9464C065B7CE862E86CE859700DF
:1001E0000000E78040DAC114D2944E99232204041F
:1001F000A2879306040103C7070003C60703850708
:10020000318FA38FE7FEE398F6FE3044A285228566
:1002100097000000E78020DD2699C1493306994008
:1002200063EC9900A9DCA686A68513050403970054
:100230000000E78040D579BF8147B306F40033075B
:10024000F6000347070083C5060085072D8F23802E
:10025000E600E39437FF3044A28522859700000032
:10026000E78060D8C1145DBF014582800DC11723AE
:10027000FFFFE70283E31306800581459720FFFF18
:10028000E780A0E505451723FFFF670043E401452C
:100290008280814749C5C1C51723FFFFE702E3E01C
:1002A000FC4141462E84AA846399C7041386050144
:1002B000A2878146C14503C7070003C50703850719
:1002C000298F3305D600034505008506298FA38FA6
:1002D000E7FEE392B6FE3044A28526859700000033
:1002E000E78060D0228597000000E78060F88547AE
:1002F0003E851723FFFF670083DD138507031D8EEF
:10030000814522959720FFFFE78020DD7C40130781
:1003100000F813060402A2972388E70251BF3E8526
:1003200082801723FFFFE70243D86D712E84B284C9
:10033000AA8590102800368997000000E780A0D396
:1003400009EDD55725A050400C402800970000002B
:10035000E78040E27DD5FD142104F5F42C004A85A8
:1003600097000000E78020F3814761DD3E85516101
:100370001723FFFF6700A3D51723FFFFE702E3D290
:1003800041112EC432C62C00054697000000E780BC
:1003900080F941011723FFFF670063D31723FFFF95
:1003A000E702A3D001112A842EC602C802CA02CCD9
:1003B00002CE97E00000E780402BB2462A86A28555
:1003C000080897000000E78060FB1375F50F0561D2
:1003D0001723FFFF6700A3CF1723FFFFE702E3CC3C
:1003E0007971B2872A8421462308B10013051101CF
:1003F000BE853AC436C697E00000E78000FBB246EF
:1004000093059101368597000000E78060A822855A
:10041000141035460C0897000000E78020F62A8467
:10042000224701E921460C103A8597E00000E78059
:10043000C0F7228545611723FFFF670043C91723D3
:10044000FFFFE70283C67171AE84AA850A853284F4
:1004500097000000E78060BB11C90A86A685228547
:1004600097000000E78020B8814711E1C5473E852D
:100470004D611723FFFF670083C51723FFFFE702C6
:10048000C3BF1D712A8AB289BE84354685471305CC
:1004900011012E8CB68A3A8BC28C468D2308F1004E
:1004A00097E00000E78060F010100C085285231FD1
:1004B000010097000000E780C0F82A843DEDA147C5
:1004C0006313FD089307900591E0E5473546E28503
:1004D0001305110113990A012308F10013590901A9
:1004E00097E00000E78060EC1357890093978A003B
:1004F000D98F90080C085285231FF1009700000047
:10050000E78020F42A8415E9A1E49387FA00918317
:100510001379F9003EC6631309004149668B814493
:10052000C14B854DB247639F970C6A868C0033851B
:100530005C0197E00000E78040E7228525611723F2
:10054000FFFF670043B793079004C9F0A547BDBFFD
:10055000834701050947C14B2308F1008347110573
:10056000A58FA308F10093872400814463E1FB0475
:10057000014714083386E6008C08B386E400BA9578
:10058000DA9683C6060083C505000507AD8E2300F5
:10059000D600E390E7FE4147639CE70490080C080F
:1005A000528597000000E780C0E925D181A0B306FD
:1005B0009B00BA871008B305F60090083E9603C565
:1005C00006000346060085078506298E2380C500A0
:1005D000E39277FF998F90080C085285BE9497009C
:1005E0000000E78000E68947014749D12A84B1B776
:1005F00090083E96034606001408BE962380C60067
:10060000850759BFB2478504638797148147180847
:10061000B306F70098083E973386F90003470700B2
:10062000034606008507318F2380E600E39177FFBC
:1006300090080C08528597000000E78080E05DF587
:100640003546E285130511012308B10197E000004A
:10065000E780A0D5139704014183939784002183F9
:10066000D98F10180C085285231FF1009700000045
:10067000E78020DD25FD814710183387F9003E967D
:100680000347070003460600B306FB008507318FCA
:100690002380E600E39277FF65A81808B306F70009
:1006A00098083E973386F900034707000346060083
:1006B0008507318F2380E600E3E127FFCA87639E29
:1006C000770990080C08528597000000E78060D7F2
:1006D00011FD81479800B306F700900818103E9767
:1006E0003E9603470700034606008507318F2380A7
:1006F000E600E39177FF3546E285130511012308F3
:10070000B10197E00000E78040CA139704014183DC
:10071000939784002183D98F10180C085285231FCA
:10072000F10097000000E780C0D1E31105EC81479C
:1007300010183387F9003E9603470700034606006A
:10074000B306FB008507318F2380E600E3E227FF35
:10075000C109410BC1BB814785B79408BE9683C6CA
:10076000060018083E972300D700850789BF6380DD
:1007700006321723FFFFE702439059712A84BE898E
:10078000B28B85473546130511022E8B468C428964
:10079000BA8A368A2300F10297E00000E780E0C0C1
:1007A00010180C1022852317010297000000E78023
:1007B00040C963180512A147631FFC069307900503
:1007C00063930900E5473546DA8513051102931452
:1007D0000A012300F102C18097E00000E780E0BC3D
:1007E00093178A0013D78400D98F90080C102285A4
:1007F0002317F10297000000E780A0C47DE1639217
:1008000009049307FA00BD88918391E0C144C207AF
:10081000C183DE8C814A3EC6414DB24763E2FA0E87
:100820006286B3854B01881097E00000E78080B5B1
:100830004DC93D557DA093079004E39609F8A5475F
:1008400059B7834701050947C14C2300F10283478B
:100850001105B3C7F900A300F1029387290081496C
:1008600063E1FC04814618103306D7008C083387F7
:10087000D900B69556970347070083C5050085063E
:100880002D8F2300E600E390D7FE41476390E706F3
:1008900090080C10228597000000E78080BA35D1BF
:1008A00089A0B3863A01BA871010B305F600900804
:1008B0003E9603C506000346060085078506298E79
:1008C0002380C500E39297FF3387EC4090080C101B
:1008D0002285BA9997000000E780A0B689470147B2
:1008E00041D165611713FFFF6700E37C90083E96D6
:1008F000034606001410BE962380C600850779B70C
:10090000B247850A93990A01939D8A0093D90901F8
:100910006391570F85473546DA8513051102230089
:10092000F10293D9890097E00000E78000A8B3EDB9
:100930003D0190000C1022852317B10397000000A1
:10094000E78020B059FD8147A68963EA970626868D
:100950000C084A8597E00000E78020A58147181021
:10096000B306F700100898083E973E960347070025
:10097000034606008507318F2380E600E3E197FEFA
:10098000639FA90590080C10228597000000E7805E
:1009900040AB21F981479810B306F700900818186A
:1009A0003E973E9603470700034606008507318FB2
:1009B0002380E600E391A7FF4109C10CB9BD1808E7
:1009C0009000B306F7003E963387FC00034707000C
:1009D000034606008507318F2380E600B5B79808E7
:1009E0004E97034707001C10CE972380E700850928
:1009F00041BF85473546DA85130511022300F10210
:100A000093D9890097E00000E780209AB3ED3D017B
:100A100090000C1022852317B10397000000E78097
:100A200040A2E31005EC814718089000B306F700D8
:100A30003E963387FC000347070003460600850700
:100A4000318F2380E600E391A7FF41460C084A85D9
:100A500097E00000E780609581471810B306F70023
:100A6000100898083E973E96034707000346060085
:100A70008507318F2380E600E391A7FF90080C10D3
:100A8000228597000000E780C09B1DD599BD7D554C
:100A900082801713FFFFE702436101112A842E852C
:100AA00093055100328902C002C202C402C69304F7
:100AB000740097F0FFFFE780A03D1D46A685130553
:100AC000910097E00000E780408E10088A854A85F3
:100AD00097000000E780E09619ED930714001808CE
:100AE00083C607000346070085070507B18EA38F5D
:100AF000D7FEE397F4FE05611713FFFF6700235D40
:100B00001713FFFFE702C3582E848C414111AA89B5
:100B1000838715003289914463D30700A144975716
:100B2000FF1F9387E75E9C43A1C7C1CA8D4723106F
:100B3000F10083C725004A852301F10083C73500F2
:100B4000A301F10083C745002302F10083C75500CC
:100B5000A302F10083C7650093059100A303010080
:100B60002303F1002304010097F0FFFFE7804032E8
:100B70000C404A860A8597F0FFFFE7808033032800
:100B8000040083564400A6881D0881470147E516E6
:100B900042868A854E8597000000E780408E2A892C
:100BA00019E5A685228597B0FFFFE780E0C14A8559
:100BB00041011713FFFF6700E3504A860A8597F04B
:100BC000FFFFE780002F6DB71713FFFFE702434CCD
:100BD0002E848C414111AA89838715003289914462
:100BE00063D30700A1449757FF1F938767529C4325
:100BF000A1C7C1C68D472310F10083C725004A85D0
:100C00002301F10083C73500A301F10083C745002C
:100C10002302F10083C75500A302F10083C76500DA
:100C200093059100A30301002303F10023040100B5
:100C300097F0FFFFE780C0250C404A860A8597F0B1
:100C4000FFFFE780002783564400032804008A85BD
:100C5000858EC2061D08C1822312D400A688814752
:100C60000147E51642864E8597000000E78060B098
:100C700041011713FFFF6700E3444A860A8597F096
:100C8000FFFFE78000234DBF1713FFFFE702E3419B
:100C9000B335B000011185052A891315F6013365B6
:100CA00015012308B1009305110136843AC632C0FC
:100CB0003EC442C297F0FFFFE780801DA247124862
:100CC000425593D68700230BF1009305910193576A
:100CD0008800A30AD100A30BF100230C010197F0B7
:100CE000FFFFE780E01A3247024603280400B337CB
:100CF000E000835644009207914411C2A1444A8502
:100D0000A68842860C0897F0FFFFE78040772A8983
:100D100019E5A685228597B0FFFFE780E0AA4A85FE
:100D200005611713FFFF6700833A1713FFFFE70200
:100D3000233601113EC68647B335B0008505AA8922
:100D40001315F6015D8D2308B1009305110136845A
:100D50003A89B28442C446C297F0FFFFE78040134D
:100D600022489248164593578800A30AF10093053C
:100D7000910193D78800230B0101A30BF100230CF1
:100D8000110197F0FFFFE780A01032471040835613
:100D90004400B337E000920703280900914891C04E
:100DA000A1480C084E8597000000E780809CAA842B
:100DB00001E9835544004A8597B0FFFFE780C0A052
:100DC000268505611713FFFF6700C32FAA959307B8
:100DD000F00F171701001307A7986317B50013C585
:100DE000F7FF1375F50F828005058346F5FFB58F74
:100DF000BA9783C70700D5B7035745001441930737
:100E0000F00F171601001306A69536974207418387
:100E1000139506014181631BE500AD8FB29703C5B1
:100E20000700130515F3133515008280850603C5E9
:100E3000F6FFA98FB29783C70700D9BF1713FFFF2B
:100E4000E702A326B28736842E86BA86AA853E8517
:100E5000BA8497F0FFFFE7806052634F0500228558
:100E600097E00000E78060802A86A686A285268516
:100E700097F0FFFFE78080501713FFFF67002325DF
:100E80001713FFFFE702C3205D712A8BAE8A171587
:100E900001001305658A2C00B284368ABA893E891E
:100EA00097F0FFFFE780C04F2A845DE13410414690
:100EB000DA85280097F0FFFFE780404C2A8449E953
:100EC0008547A303F100A6C2930771002408BEC49E
:100ED000A68685470D462C18281002DC02DED6C0F7
:100EE000BEC697F0FFFFE78000442A8435E18347C0
:100EF0007102A6860D4693F7F7072300FA00C14753
:100F00003EDE2C188947281026DCA303F10097F059
:100F1000FFFFE78040412A8405ED4146A6854E85C6
:100F200097D00000E78060488D47A6860D462C18B4
:100F30002810A303F10097F0FFFFE780C03E2A844A
:100F400001E94146A6854A8597D00000E780E04543
:100F5000228561611713FFFF6700C3161713FFFF98
:100F6000E702A31497F70000938707EF984383C71E
:100F7000470079712A89AE84170501001305457C65
:100F80000C083AC42306F10097F0FFFFE7804041C8
:100F90002A8405ED14104146CA85080897F0FFFF22
:100FA000E780C03D2A8415E1140815462C0008107E
:100FB00097F0FFFFE780803C2A8401E921462C0856
:100FC000268597D00000E780403E228545611713B3
:100FD000FFFF6700C30F1713FFFFE702030D97F72B
:100FE0000000938767E79C477971AA842E841705D0
:100FF0000100130565750C083EC697F0FFFFE780FA
:10100000203A0DE914104146A685080897F0FFFF25
:10101000E780C03605E1140811466C00081097F00F
:10102000FFFFE780A03519E58347F10193F7F70348
:101030002300F40045611713FFFF670043091713EE
:10104000FFFFE70283063688A14881470147E5464E
:1010500097F0FFFFE780A0421713FFFF6700230709
:101060001713FFFFE70263043688A1488147014751
:10107000E54697F0FFFFE780C06F1713FFFF67009B
:1010800003051713FFFFE702430201112A842E858F
:101090000C0832C697F0FFFFE780803009ED324739
:1010A000970601009386C6681008C14522859700FF
:1010B0000000E780E0D805611713FFFF67002301F8
:1010C0001713FFFFE70263FE4111C1472EC032C470
:1010D0008A8509463EC23EC697F0FFFFE780A024FE
:1010E00041011713FFFF670083FE1713FFFFE7029D
:1010F000C3FB4111AE8613061009AA850A8502C0FA
:1011000002C202C402C697F0FFFFE7802027410118
:101110001713FFFF6700A3FB1713FFFFE702E3F8B6
:101120003287970601009386A6622E8693050002F9
:1011300097000000E780C0D01713FFFF670023F976
:101140001713FFFFE70263F67971C1472ACC2ED04F
:1011500032D42C080D4628003ECE3ED23ED602C4E4
:1011600002C602C802CA97F0FFFFE780C01B4561B4
:101170001713FFFF6700A3F51713FFFFE702E3F262
:101180000111AA842E84170501001305E55C8A85E8
:1011900097F0FFFFE780C02015E514084146A685BB
:1011A0000A8597F0FFFFE780601D09ED8347E101A5
:1011B0000347F101A207D98FCA07C9836177D98F85
:1011C0002310F40005611713FFFF670043F015CDEE
:1011D0001713FFFFE70263ED9757FF1F9387C7A021
:1011E00090439755FF1F938565A01755FF1F130563
:1011F000A59B97D00000E78000C51755FF1F13057A
:10120000A59A1713FFFF670083EC1755FF1F1305FF
:10121000A59982808DCD1713FFFFE70203E9975749
:10122000FF1F9387679C944301112E840A8697556C
:10123000FF1F9385A59B97D00000E78040C60A85D5
:101240000294014505611713FFFF670043E87D55D0
:1012500082801713FFFFE70243E597D00000E78085
:1012600080D19757FF1F23A1A79817F5FFFF1305FC
:10127000E5C997B00000E780C0741713FFFF67004F
:1012800003E51757FF1F13076798931715000843C7
:101290003E95FD572310F50082801713FFFFE702EC
:1012A000C3E02A84084009E51713FFFF670023E223
:1012B0001C4158401CC06313E5005CC083475500C7
:1012C00023200500F99BA302F50097A0FFFFE7800C
:1012D000207CC9BF1713FFFFE70283DB9757FF1F6F
:1012E0009387C79498432A8411CB8347350093F79B
:1012F000070289C703550500894502971305440174
:1013000097B00000E780403B835504000355E4009C
:1013100097300000E780A00C485819C597A0FFFF40
:10132000E7800077232A0402130584039700000056
:10133000E780E0F68144B1499790FFFFE780C06DF8
:1013400063CBA402834734002320040493F727FCD3
:10135000A301F40000489790FFFFE780E06C1316AC
:101360001500814522859710FFFFE78000D71713EE
:10137000FFFF670023D5B3873403032904038504E3
:101380003E994A8597000000E78060F12304090038
:1013900065B78347350093F7070299E301458280DB
:1013A0008357E500E39CB7FEC167FD176316F6009F
:1013B00005458280054599A81713FFFFE702E3CE94
:1013C00093170601C187B2842A8401496359F00248
:1013D000835705009DCB01456367F60003458400F4
:1013E0003E953325A6001375F50F0DA01C48131765
:1013F0001900BA9783D70700E38E97FA05099790EB
:10140000FFFFE7806062E343A9FE01451713FFFF7A
:101410006700E3CB1713FFFFE70283C7AE89AA84F7
:101420009790FFFFE78000562A8497D0FFFFE78060
:10143000A02EAA8601471306840197050000938514
:1014400085E41745FF1F1305A57C9790FFFFE780F4
:10145000801C2A8925C98C441304C50022859E0559
:1014600093F5050897A0FFFFE780403CCC408387B9
:101470007400E18163DD070493E50508228597A0E8
:10148000FFFFE780A03A0D4693854400228597A090
:10149000FFFFE780C03683D50400228597A0FFFFB9
:1014A000E780E03D83D52400228597A0FFFFE780F9
:1014B000003D03D6490083A50900228597A0FFFFC0
:1014C000E780E0334A851713FFFF6700A3BF93F55A
:1014D000F5076DB71713FFFFE70223BD01112A843B
:1014E000328532C697A0FFFFE780E0279780FFFF95
:1014F000E7806034835704001757FF1F1307878A5C
:101500003246231BF100930700F8A30DF1001C479E
:101510001843231AA1008983858BB307F740B2854E
:1015200048083ECE231C0100230D01009700000057
:10153000E78080EE05611713FFFF670043B91713BB
:10154000FFFFE702E3B4004101453DC49304C4003A
:1015500026853289AE8997A0FFFFE780C024954594
:101560002A8A2685035B040197A0FFFFE7802021DC
:10157000268597A0FFFFE780603E8D45AA8A2685D5
:1015800097A0FFFFE780A01F268597A0FFFFE780B9
:10159000E03C5C48420A135A0A01D2975CC4231803
:1015A0006401814763983A0146054D813306254120
:1015B0009337160013F5F70F1713FFFF670083B07B
:1015C0001713FFFFE702E3AB89692A8BAE8B328AE0
:1015D000B68A81440144314CFD199790FFFFE780A2
:1015E000A04363CDA4009790FFFFE780E045018D05
:1015F00033B5AA001713FFFF670023AC33898403B8
:1016000083270B003E9963170A00834789008504EE
:101610003E94E1B703560A00DE854A8533F6C900D9
:1016200097000000E780E0F16DD10545E1B71713A1
:10163000FFFFE70283A701112A847C000355E50020
:101640003ECAB70707003ECC7C003ECE9720000084
:10165000E78020082A898545480897A0FFFFE78092
:1016600020399945480897A0FFFFE780E015AA8434
:101670004A8597200000E780A0082380A4009747B0
:10168000FF1F938727729C434166130606F09396CB
:10169000870113D78701558F93D68700F18E558F19
:1016A000A207B706FF00F58FD98F11462C001385CE
:1016B00014003EC497D00000E78020CF5008A382DA
:1016C00004008945228597000000E780E0E019C901
:1016D000AA851305840397A0FFFFE780E0313C4013
:1016E00085073CC005611713FFFF6700439E171372
:1016F000FFFFE702839B9790FFFFE780E0342A8497
:1017000005049790FFFFE78020333305A402F147DB
:1017100091453305F50297200000E78020BA11E5D6
:1017200065551713FFFF6700839A9747FF1F23A78D
:10173000A74E9790FFFFE78020312A8405049790F9
:10174000FFFFE780602F3305A40289450605972037
:101750000000E780A0B669D59747FF1F23A8A74AD6
:101760009790FFFFE780402E2A8405049790FFFFA3
:10177000E780802C3304A4029747FF1F239A8748F1
:101780009790FFFFE780402C2A849790FFFFE78027
:10179000A02A930714003385A7029747FF1F239AB7
:1017A000A746970701009387E7BE1747FF1F23252A
:1017B000F7460145BDB71713FFFFE702638DAA8403
:1017C0002E8901449749FF1F9389C95D130A80063A
:1017D0009790FFFFE78040266347A4000145171359
:1017E000FFFF6700238E3305440383A709024A865F
:1017F000A6853E9597000000E780E0B919E1050451
:10180000C1BF0545E9BF1713FFFFE7028387AA8A17
:101810002E8BB28B368C3A8A814401448149974C95
:10182000FF1F938C2C58130D80069790FFFFE780C5
:10183000A02063C9A40011E085494E851713FFFF5E
:101840006700A3873389A40383A70C025E86D6852D
:101850003E994A8597000000E780E0B31DC197904C
:10186000FFFFE780601E0544636D4501D2866286F6
:10187000DA851305090397000000E780A0D411C1A1
:10188000854985045DB71713FFFFE7026380C164D4
:1018900041112A8901449749FF1F9389A950130ACE
:1018A0008006FD1436C632C42EC29790FFFFE78033
:1018B000A01892452246B2466348A4000145410162
:1018C0001713FFFF670003803305440383A7090252
:1018D0003E9509C683473500C18B9DC791C6834796
:1018E000350093F707028DC3630699008357E5001F
:1018F000639C27010357050001CB63E7E50083479D
:101900008500BA97E3CDF5FA050469BF1703FFFF19
:10191000E7020378C1642A8901449749FF1F93892C
:101920006948130A8006FD149790FFFFE780C010F6
:101930006346A4001703FFFF6700C3783305440321
:1019400083A709023E958357E500638A97006304E5
:1019500099006396270197000000E780E09705044F
:10196000E1B71703FFFFE702437189692A8AAE8A4C
:10197000328BB68B8144174CFF1F130CAC42930C77
:101980008006314DFD199790FFFFE780E00A63C69E
:10199000A4001703FFFF67000372338994038327B2
:1019A0000C028355CA015A863E994A859700000069
:1019B000E780609E31C1814D15A03384AD0383273C
:1019C000090303D60B00D68533F6C9003E94228561
:1019D00097000000E780E0B609E9850D9790FFFFCA
:1019E000E7808003E3CBADFC01A8228597000000CF
:1019F000E780E08A23040400850471B71703FFFF22
:101A0000E70223684169AA8A014A174BFF1F130B9B
:101A10006B397D19C14B054C9790FFFFE780C001E2
:101A20006346AA001703FFFF670023699309800636
:101A3000B3073A0383290B02BE9983D7E900638E6B
:101A4000270163842A01639A570103A4890301E8EB
:101A50004E8597000000E780C0BD050A75BF83571B
:101A60000401639977099304C400268597A0FFFFBA
:101A7000E78060D385452A8D2685835C040197A085
:101A8000FFFFE780C0CF268597A0FFFFE780A0E794
:101A900062056185635905048D45268597A0FFFF82
:101AA000E780E0CD8945268597A0FFFFE78020CD20
:101AB0008945268597A0FFFFE78060CC8545268570
:101AC00097A0FFFFE780E0CC83470500094793F725
:101AD000F707639AE7009945268597A0FFFFE780FF
:101AE00040CBA30285014848337D2D012318940182
:101AF0006A9548C40040A1BF1703FFFFE702E35AFD
:101B000037E404008327041D82979747FF1F83C78C
:101B100067161725FF1F1305A59DA300F500832752
:101B2000441C82978327841C81461306F00F81454D
:101B3000014582971703FFFF670063591747FF1F8F
:101B40001307470318439745FF1F83C5A5129747FF
:101B5000FF1F9387A7108346870303469703639766
:101B6000D5009747FF1F2387C710828083C5870151
:101B70000347A7036317B6009747FF1F238CE70EA1
:101B8000828003C687016317C7009747FF1F23831F
:101B9000D70E828083C68701130750026319D700CE
:101BA000930760021747FF1F2306F70C828083C646
:101BB0008701130660026315D60093077002DDB734
:101BC00083C7870155BF9747FF1F93872709D44BCA
:101BD0000947638DE6081703FFFFE702034D174926
:101BE000FF1F1309E9043E8483470900918B9DCFB1
:101BF000B7E4040083A7041D829783A7441C1745FC
:101C0000FF1F13056503829783A7841C814617462F
:101C1000FF1F0346660481450145829721C583471E
:101C20000900ED9B1747FF1F2304F70083470400BB
:101C300093F7F70F85CB91471747FF1F232AF7022A
:101C400097000000E78080EB97000000E78040EFFE
:101C5000B7E70400BC4F414691451745FF1F0345B8
:101C6000650082971703FFFF6700634682801703B2
:101C7000FFFFE70283438D4741116306F504C54723
:101C80006308F50285476310F5029747FF1F238518
:101C9000A7FEB7E70400BC4B930500101745FF1FD4
:101CA000034545FC829741011703FFFF670023426C
:101CB00085471747FF1F2301F7FCB7E70400BC4B1C
:101CC00093050020E1BF9747FF1F938727F9D44B67
:101CD0001147638DE600B7E7040083A7071D8297CD
:101CE000B7E70400BC4B930500044DBF05491747F7
:101CF000FF1F232F27F783C7070032C62E8493F7D1
:101D0000F70FD5D3B7E4040083A7041D7D14137423
:101D1000F40F8297E37689FCB245994703C6150014
:101D2000E3F0C7FCFC4409061745FF1F130505F542
:101D30008297BC48930500081745FF1F034585F2AD
:101D4000829779BF1703FFFFE70223361747FF1F6C
:101D50001307C7F04047184B1C409746FF1F23A5A9
:101D6000F6F06316E4001747FF1F2321F7F0130571
:101D700084FE9790FFFFE78000AA035564FF9780D9
:101D8000FFFFE780807297A0FFFFE78060D0170316
:101D9000FFFF6700C3331703FFFFE70203319747D5
:101DA000FF1F9387A7EBD84BDC4789C7970000003C
:101DB000E78080F985471747FF1F232BF7EA9747EE
:101DC000FF1F938727DB9C43930500021745FF1FE6
:101DD000034545E983C787031747FF1F230CF7E82F
:101DE000B7E70400BC4B82971703FFFF6700232E61
:101DF0009747FF1F23A6A7E682801703FFFFE7028E
:101E0000232937E404007C4CA1451745FF1F0345F7
:101E100065E582977C48A1451745FF1F034585E48A
:101E20009744FF1F938484E38297DC4489EB9700F7
:101E30000000E78080D91703FFFF6700A32803D5C0
:101E400067FF9780FFFFE7804066AA896DD1D84879
:101E500091476310F7027C4C91451745FF1F0345DE
:101E600065E082977C4891451745FF1F034585DF54
:101E7000829703A9490103D409018947B7E90400FE
:101E80001747FF1F2326F7DE83A7091D21044204FD
:101E9000829783C784011715FF1F130565656119B4
:101EA0001717FF1FA306F76483A7491C4180829779
:101EB0009747FF1F238207DC83A7C91C8146094679
:101EC0009375F40F4A85829711E99747FF1F83C7DF
:101ED000E7EA89C79710FF1FE78060CEB7E70400E5
:101EE000BC4F2146A1451745FF1F0345A5D7829743
:101EF00099B71703FFFFE702431B93F70520011172
:101F00002E8481CF97000000E78020E9134504204C
:101F100005611703FFFF6700831B93F70510A9CF27
:101F20009744FF1F938484D3DC4897000000E78028
:101F300020C11747FF1F1307E7C3184383C7840156
:101F4000034787036318F700DC4489C79700000044
:101F5000E78080DF85471747FF1F232BF7D0B7E7C0
:101F60000400BC4B930500021745FF1F034585CFB6
:101F700082971345041069BF93F70508BDC79747BB
:101F8000FF1F83C7B7CFE91719469745FF1F9385F2
:101F900005CF1305D10093F4F70F1749FF1F03492D
:101FA000E9CD97C00000E780404093970401C183CA
:101FB0001747FF1F130707CD231DF100231CF10056
:101FC0009747FF1F938787C93ACE3ACAD84323065B
:101FD000010009CBDC439315890154080D46E185C6
:101FE000680082971345040825B793F72500A5C319
:101FF0009747FF1F938787C6D84B89476306F70229
:102000009747FF1F83C7C7C213F7270011EF918BB4
:1020100099CFB7E70400BC4F1306000A894517455E
:10202000FF1F034525C4829713452400D5B5974764
:10203000FF1F938727B49C4383C787031747FF1F5E
:10204000230AF7C297000000E78060DBF1BF93F737
:10205000050281CB97000000E78060DA1345040297
:1020600045BD93F7850081CB97000000E780E0D263
:102070001345840071BD93F7150081CB97000000D4
:10208000E780A0B41345140061B593F7450081CBF8
:1020900097000000E78060B31345440095BD93F7B7
:1020A000050495C39747FF1F83C747BB91CB970094
:1020B0000000E780A0A491471747FF1F232AF7BA23
:1020C00013450404B1B593F705010145E38207E424
:1020D0009747FF1F938787B8D84B91476310F70442
:1020E0009747FF1F9387C7B49C4313D72700858367
:1020F000D98F858B91E7B7E7040083A7071D8297E7
:10210000B7E70400FC4F91451745FF1F034585B510
:10211000829785471747FF1F232CF7B41345040107
:10212000C5BB9747FF1F238BA7C482801703FFFF00
:10213000E702A3F79747FF1F23A807B29747FF1FA0
:1021400023A607B285471744FF1F1304A4A217470D
:10215000FF1F232FF7B01C4083C787031747FF1FBC
:10216000230AF7B09790FFFFE780409329C59717A0
:10217000FF1F23A3A7381C40170500001305A5D790
:1021800083C787031747FF1F2306F7AE1717FF1FE5
:10219000A300F7369747FF1FA38207ACB7E70400F9
:1021A00083A7070882979747FF1F238DA7AA1703C6
:1021B000FFFF6700C3F1B7C7898E938767ED1717D5
:1021C000FF1F232BF73245BF1747FF1F034707A900
:1021D000795555E79747FF1F938747A803C717000F
:1021E00005079746FF1FA38BE6A603C717008D467A
:1021F0003377D7029746FF1FA382E6A683C6170050
:102200001747FF1F13070797184393F6F60FA9EE1A
:10221000834787031747FF1F230EF7A485471747F8
:10222000FF1F230DF7A29747FF1F938767A09C43CB
:102230000145998BA9E71703FFFFE70203E737E49E
:1022400004007C48C1451745FF1F0345A5A182979F
:102250003C4885451745FF1F0345C5A082970145AA
:102260001703FFFF6700A3E683C717008546639542
:10227000F6008347970379BF8347A70361BF828036
:102280009747FF1F83C7879DA1CF1703FFFFE70273
:10229000C3E137E404009747FF1F2381079C7C4874
:1022A00085451745FF1F0345E59B82977C4C91456B
:1022B0001745FF1F0345059B82977C4891451745AD
:1022C000FF1F0345259A82973C48C1451745FF1FCC
:1022D00003454599829701451703FFFF670023DFF8
:1022E000795582801703FFFFE70223DC2A84035518
:1022F00065FF9780FFFFE780401B9747FF1F93878D
:10230000E795D847BE841DEF9790FFFFE780807761
:102310009C48232004009DEB9747FF1F23A8879428
:102320009747FF1F23A28794B7E70400BC4B89455A
:102330001745FF1F03450593829701451703FFFFCC
:102340006700E3D8630A8700184375BF80C39747C7
:10235000FF1F23AD8790C9BF7955CDB71703FFFF86
:10236000E702A3D49747FF1F938787A188432326BB
:10237000050023240500510597A00000E780C03325
:102380001703FFFF6700A3D41703FFFFE702E3D1A2
:102390001744FF1F1304C49E1C40411199CF9C4752
:1023A0002302B5002AC61CC197000000E78040FB4D
:1023B0001C409C4B99C33245829741011703FFFF94
:1023C0006700E3D01703FFFFE70223CE4111444D1E
:1023D000328532842EC69790FFFFE780C0522AC410
:1023E00022859790FFFFE780205403A84400630CE8
:1023F0000800B245835744001840224683D5450063
:10240000AA862685029841011703FFFF670023CCA7
:102410001703FFFFE70263C9404D1DC808C09705B9
:102420000000938565031305440197A00000E78031
:1024300040169747FF1F9387A7949C43014589E760
:102440009747FF1F23AE87921703FFFF670023C83C
:102450007D55DDBF1703FFFFE70223C501116800AB
:102460009305F00F02C602C802CA02CC02CE970042
:102470000000E780A0F105611703FFFF670023C597
:102480009747FF1F9387C78F9C43D847A1679D0736
:102490006319F7021703FFFFE70223C10111328519
:1024A0009790FFFFE7802046230AA100814568003E
:1024B00097000000E78080ED05611703FFFF6700CC
:1024C00003C182809747FF1F9387878B9C43D84720
:1024D000A167938777036319F7021703FFFFE702EA
:1024E000C3BC011132859790FFFFE780C041230AEA
:1024F000A1008145680097000000E78020E90561A0
:102500001703FFFF6700A3BC82809747FF1F9387D5
:1025100027879C43D84795476316F7041703FFFFA7
:10252000E702A3B80111328532849790FFFFE7805C
:10253000803D230AA10022859790FFFFE780C03EDF
:1025400083574400231BA10081453ECC1C406800FA
:102550003ECE97000000E78060E305611703FFFFB0
:102560006700E3B68280930785FF8DC38327C5FF8D
:1025700091CFDC4B81CF1703FFFFE70203B30325A5
:1025800085FF82971703FFFF670063B482801703FC
:10259000FFFFE70283B12A8432859790FFFFE7802F
:1025A0008036BD4763EBA70018449377F5000345D9
:1025B000B70041995D8DA305A7001703FFFF6700D2
:1025C00003B11703FFFFE70243AE01117C003ECACF
:1025D000B70707003ECC7C003ECE5C4DA9C72A84DD
:1025E00013858700AE8497A00000E780E0FCA1651A
:1025F0002A899D0548089770FFFFE780603E930594
:10260000803EB345B902480893F5F50F9790FFFF58
:10261000E780C021014781465008A6852285977032
:10262000FFFFE780406105611703FFFF670023AAF2
:102630001703FFFFE70263A797000000E780A0F8F9
:102640001703FFFF6700A3A81703FFFFE702E3A537
:1026500001117C00AE843ECAA165B70707002A8439
:102660003ECC48087C00938575033ECE9770FFFFF3
:10267000E78000371C44480883C5B700BD899790A0
:10268000FFFFE780A01A500801478146A6852285F2
:102690009770FFFFE780205A05611703FFFF67006F
:1026A00003A31703FFFFE70243A02A84AE84970029
:1026B0000000E78000EEA685228597000000E780F5
:1026C000E0F81703FFFF670083A01703FFFFE7028F
:1026D000C39D97000000E78060F71703FFFF6700C6
:1026E000039F1703FFFFE702439C0329C501411124
:1026F000630809022A843285B2849790FFFFE7803D
:1027000080202AC626859790FFFFE780E021832757
:1027100049002A8691C7DC4781C7B2452285829746
:1027200041011703FFFF6700839A1703FFFFE702CA
:10273000C397444D91CC2A8432859790FFFFE78060
:10274000A01EDC40AA8589C79C4799C32285829731
:102750001703FFFF6700A3971703FFFFE7024393E9
:10276000032AC5014111630D0A062E89AA849545E5
:10277000328532849770FFFFE78080268545228569
:102780009790FFFFE7804004AA89CA852285979029
:10279000FFFFE780A00B83274A008DCBDC439DC75A
:1027A00022859790FFFFE780A00083274A00104012
:1027B00083564400DC437115A307A100B2961307AA
:1027C000F1004E86CA852685829701C523800900BF
:1027D00001A88345F10022859790FFFFE780C0FEA6
:1027E00041011703FFFF6700E38D1703FFFFE702B7
:1027F000C38B65711C083EC2B70780013EC41C082C
:1028000032893EC62A84AE8497000000E780A0ED9E
:102810004A859790FFFFE78020118357A1008DC361
:10282000AA855000228597000000E78020F3014729
:1028300081465000A68522859770FFFFE780A03F64
:1028400059611703FFFF670083881703FFFFE70243
:10285000238465711C088329C5013EC2B707800126
:102860003EC41C082A84AE8432893EC6970000000C
:10287000E780E0EB638A09024A859790FFFFE780D3
:10288000A00A8357A100AA8585C35000228597001E
:102890000000E780A0EC014781465000A685228514
:1028A0009770FFFFE780203959611703FFFF67002A
:1028B000638117F3FEFFE702437F65711C083EC288
:1028C000B70780013EC42A841C0832853EC6AE8408
:1028D0009790FFFFE78040058357A1008DC3AA852D
:1028E0005000228597000000E78040E701478146BD
:1028F0005000A68522859770FFFFE780C03359619D
:1029000017F3FEFF6700A37C17F3FEFFE702E379EE
:10291000444D81EC8347450093B71700B307F0405F
:102920003E8517F3FEFF6700837A1845FD576DDB80
:1029300097070000938747032A845CCB9705000024
:102940009385A5C21385840097A00000E78060C42A
:1029500080C003474400814761F71737FF1F2323D7
:1029600097427DBF17F3FEFFE70283728329C501FB
:1029700041110329850081476387090A032409015E
:1029800091452A8A22859770FFFFE780600585457B
:1029900022859790FFFFE78020E38945AA8A228558
:1029A0009790FFFFE78040E2AA849770FFFFE780DF
:1029B000400A83A749002A8B8DCB9C439DC7228563
:1029C0009790FFFFE780C0DE83A74900A306A10020
:1029D0001040835644009C431307D100B296D6851D
:1029E0001306E1005285829709CD83570B0023809F
:1029F000F400A183A380F40023800A00A306010051
:102A000039A88357E10022852380F4008345D10053
:102A1000A183A380F4009790FFFFE780E0DA83476B
:102A2000D100B337F0000347B900920701453D9B41
:102A3000D98FA305F900410117F3FEFF67008368F2
:102A400017F3FEFFE702636641110DED9737FF1F95
:102A500093874733804315C80440130984009DC9F8
:102A60005C4099C79C4B89C726852EC68297B24584
:102A70009307803EB385F5024A8597A00000E78062
:102A800060C121A0404DAA8469F8410117F3FEFFFF
:102A90006700E3634A8597A00000E780E0C15C40DF
:102AA000EDD7DC4BFDD326858297C5B717F3FEFF24
:102AB000E702A35F2A8432859790FFFFE780A0E4B6
:102AC000AA85228597000000E780C0F717F3FEFF74
:102AD0006700E35F17F3FEFFE702235D2A84AE84FD
:102AE00097000000E780C0FCA685228597000000C3
:102AF000E78060AD17F3FEFF6700635D0841335563
:102B0000B5000589828017F3FEFFE702035A1734E8
:102B1000FF1F130424291C5C0111231701008D835E
:102B2000858BA303F1008327040B231801002319CD
:102B3000010003D7C7013ECA3C002314E1007D57C2
:102B40002315E1000357C4023ECC02CE2316E10058
:102B50009770FFFFE78020CE8357E101231EA1007D
:102B600093F707E093E71710231FF1009737FF1F34
:102B700083C7E72595C305470145638AE700834777
:102B8000840393E727001737FF1F2309F724056104
:102B900017F3FEFF6700A353814717F700001307E1
:102BA00067DB85461306710085454808979000004D
:102BB000E780408F69FD83478403F59B1737FF1F2C
:102BC000230EF72085471737FF1F2302F720C1B7D1
:102BD00017F3FEFFE702634A973DFF1F938D8D1C9D
:102BE00003A6CD0639712A898147814493060002E4
:102BF0003357F600058B01C7850493F4F40F85075E
